:020000040800F2
:10000000205F01206D02000825C30008A5A9000893
:1000100005C10008C1340008F1FA00080000000022
:1000200000000000000000000000000011D00008E7
:10003000C95100080000000091C80008FDE2000856
:10004000870200088702000887020008870200086C
:100050008702000887020008195500088702000877
:10006000870200088702000825550008870200085B
:10007000814F0008870200088702000887020008F5
:10008000870200088702000887020008870200082C
:10009000C5340008D534000887020008315500082F
:1000A000870200088702000887020008870200080C
:1000B00087020008870200088702000887020008FC
:1000C00087020008870200088702000887020008EC
:1000D000870200089DFA000887020008B9FA0008A4
:1000E00087020008870200088702000887020008CC
:1000F00087020008870200088702000887020008BC
:1001000087020008870200088702000887020008AB
:10011000870200088702000887020008870200089B
:1001200087020008914F0008A14F0008B14F000856
:10013000870200088702000887020008870200087B
:10014000E5340008F534000887020008870200083B
:10015000C14F0008D14F000887020008D5FA0008F7
:10016000870200088702000887020008870200084B
:1001700087020008870200088702000800000000CC
:10018000870200088702000800F002F800F05EF81D
:100190000AA090E8000C82448344AAF10107DA45E2
:1001A00001D100F053F8AFF2090EBAE80F0013F0D6
:1001B000010F18BFFB1A43F00103184754810100D7
:1001C000748101000A444FF0000C10F8013B13F059
:1001D000070408BF10F8014B1D1108BF10F8015BA0
:1001E000641E05D010F8016B641E01F8016BF9D193
:1001F00013F0080F1EBF10F8014BAD1C0C1B09D1EA
:100200006D1E58BF01F801CBFAD505E014F8016B5B
:1002100001F8016B6D1EF9D59142D6D370470000ED
:100220000023002400250026103A28BF78C1FBD8FF
:10023000520728BF30C148BF0B6070471FB517F089
:10024000AEFD00F0C0F81FBD10B510BD00F080F984
:100250001146FFF7F3FF0FF03FFF00F09EF903B4E4
:10026000FFF7F2FF03BC00F0A1F900000948804746
:1002700009480047FEE7FEE7FEE7FEE7FEE7FEE788
:10028000FEE7FEE7FEE7FEE704480549054A064BA0
:1002900070470000D1E3000889010008202F0120E9
:1002A000205F0120203F0120203F012053EA020C63
:1002B00000F069802DE9F04B4FF00006002B1FBFC6
:1002C000B3FA83F503FA05F424FA05F65E4012BF8B
:1002D0001643B2FA82F502FA05F4C5F120051EBFF5
:1002E00022FA05FC44EA0C04203556EA044C4FEA95
:1002F000144418BF641C4FF000084FF000099042EE
:1003000071EB030C39D3002919BFB1FA81F701FA57
:1003100007F6B0FA80F700FA07F6C7F120071EBF0C
:1003200020FA07FC46EA0C062037B6FBF4FCA7EBE4
:100330000507103F07F01F0BCBF120062CFA06F63D
:100340000CFA0BFB44BFB3460026202FA4BF5E4629
:100350004FF0000B5BEA060C08BF4FF0010B19EBE6
:100360000B0948EB0608ABFB027C06FB02CC0BFB3F
:1003700003CCC01B71EB0C01C1E70B4602464146A2
:100380004846BDE8F08B13B5084318BF4FF0FF3067
:100390000146AFF30080BDE81C4070470B4910B523
:1003A000A1F17C020A4CC2E93712372106E000EBCA
:1003B000104342F82130074B00FB03400B1EA1F114
:1003C0000101F4DC10BD0120E8E70000CC030020AF
:1003D000E119D666CD0D0100032A40F2308010F0FD
:1003E000030C00F0158011F8013BBCF1020F6244D0
:1003F00098BF11F801CB00F8013B38BF11F8013B61
:10040000A2F1040298BF00F801CB38BF00F8013B0D
:1004100011F0030300F02580083AC0F0088051F87D
:10042000043B083A51F804CBA0E80810F5E7121D88
:100430005CBF51F8043B40F8043BAFF30080D207A7
:1004400024BF11F8013B11F801CB48BF11F8012B73
:1004500024BF00F8013B00F801CB48BF00F8012B96
:10046000704710B5203AC0F00B80B1E81850A0E8F2
:100470001850B1E81850A0E81850203ABFF4F5AF72
:100480005FEA027C24BFB1E81850A0E8185044BFCE
:1004900018C918C0BDE810405FEA827C24BF51F83B
:1004A000043B40F8043B08BF7047D20728BF31F82F
:1004B000023B48BF11F8012B28BF20F8023B48BF80
:1004C00000F8012B704702F0FF0343EA032242EADF
:1004D000024200F002B84FF0000200B51346944605
:1004E0009646203922BFA0E80C50A0E80C50B1F18C
:1004F0002001BFF4F7AF090728BFA0E80C5048BFA0
:100500000CC05DF804EB890028BF40F8042B08BF3D
:10051000704748BF20F8022B11F0804F18BF00F839
:10052000012B704770477047704710B500F008F80E
:10053000006810BD10B5044600F002F8046010BD5C
:1005400000487047340400200048704734040020FD
:100550007546FFF7F9FFAE4605006946534620F0A1
:100560000700854618B020B5FFF78EFEBDE8204095
:100570004FF000064FF000074FF000084FF0000B5F
:10058000AC46ACE8C009ACE8C009ACE8C009ACE8CE
:10059000C00921F007018D46704710B50446AFF33E
:1005A00000802046BDE81040FFF759BE01491820E1
:1005B000ABBEFEE7260002007047000080B58AB09F
:1005C00008900791089820B9FFE7FF208DF82700D1
:1005D0009BE0079820B9FFE7FF208DF8270094E003
:1005E000079890ED000A90ED013A90ED021A90ED17
:1005F000032A20EE030A21EE021A30EE010A30EE41
:10060000000A8DED060A079890ED010A90ED021A96
:1006100020EE000A21EE011A30EE010A30EE001A37
:10062000B7EE000A8DED010A30EE410A8DED050AA4
:100630009DED060ADDED050A14F006FB9DED011A9D
:10064000089880ED010A079890ED000A90ED013AB4
:1006500090ED024A90ED032A20EE040A22EE032ACE
:1006600030EE420A30EE000A8DED040A9DED040AD8
:10067000B0EEC00AB4EE410AF1EE10FA0ADBFFE771
:10068000DDED040A9FED230A0FF06EFC089880ED63
:10069000020A07E09DED040A13F0D4FF089880EDEC
:1006A000020AFFE7079890ED000A90ED011A90ED1D
:1006B000022A90ED033A20EE030A21EE021A30EEF0
:1006C000010A30EE000A8DED030A079890ED020A48
:1006D00090ED031A20EE000A21EE011A30EE010A15
:1006E00030EE001AB7EE000A30EE410A8DED020A34
:1006F0009DED030ADDED020A14F0A6FA089880EDDC
:10070000000A00208DF82700FFE79DF927000AB0B6
:1007100080BD00BFDB0FC93F80B58CB00A90099146
:100720008DED080A0A9820B9FFE7FF208DF82F0009
:1007300029E19DED081AB7EE000A80EE010A0A9839
:1007400080ED040A0A994FF07E5008600A99002053
:1007500048600A9988600A99C8600998002800F0E2
:100760000E81FFE7099801680091406817F04CFA84
:100770000246009801920A46019942EC101B8DED49
:10078000020B17F041FA9DED020B41EC110B14F036
:100790005BF98DED040B9DF8170080F080008DF85B
:1007A00017000498059916F009FB0790099890ED39
:1007B000000AB5EE400AF1EE10FA2BD1FFE70998D6
:1007C00090ED010AB5EE400AF1EE10FA22D1FFE7F2
:1007D000099890ED020AB5EE400AF1EE10FA19D12F
:1007E000FFE70A9940F2C560C3F64D7008600A99A8
:1007F00044F62D20C3F60D4048600A994AF256404F
:10080000CBF6393088600A9944F2AD70C3F619709E
:10081000C860B3E09DED070A9FED5D1AB4EE410A92
:10082000F1EE10FA08DBFFE79DED070AB5EE400A8E
:10083000F1EE10FA19DDFFE70A9945F66E10C3F6DE
:100840007F7008600A9945F20C30C3F6B01048601A
:100850000A9948F6AB00CBF6BB3088600A9949F29A
:100860008550C3F69750C86087E09DED070A9FED5D
:10087000491AB4EE410AF1EE10FA0ADBFFE79DEDEA
:10088000070A9FED431AB4EE410AF1EE10FA19DDA2
:10089000FFE70A9940F2C560C3F64D7008600A99F7
:1008A00044F62D20C3F60D4048600A994AF256409E
:1008B000CBF6393088600A9944F2AD70C3F61970EE
:1008C000C86059E09DED070A9FED331AB4EE410A66
:1008D000F1EE10FA0ADBFFE79DED070A9FED2D1AF6
:1008E000B4EE410AF1EE10FA19DDFFE70A9940F281
:1008F000C560C3F64D7008600A9944F62D20C3F612
:100900000D4048600A994AF25640CBF6393088606B
:100910000A9944F2AD70C3F61970C8602BE09DEDE2
:10092000070A9FED1D1AB4EE410AF1EE10FA08DB3A
:10093000FFE79DED070AB5EE400AF1EE10FA19DD6A
:10094000FFE70A9940F2C560C3F64D7008600A9946
:1009500044F62D20C3F60D4048600A994AF25640ED
:10096000CBF6393088600A9944F2AD70C3F619703D
:10097000C860FFE7FFE7FFE7FFE7FFE7FFE70020CB
:100980008DF82F00FFE79DF92F000CB080BD00BF50
:10099000DB0FC93FDB0F49400000B44281B000903B
:1009A0000099002088604860086001B0704700002E
:1009B00080B52DED048BB2B030902F912E922D93F7
:1009C000309828B9FFE7FF208DF8C70000F0F7BD89
:1009D0002F9828B9FFE7FF208DF8C70000F0EFBD82
:1009E0002E9828B9FFE7FF208DF8C70000F0E7BD7B
:1009F00040F20401C2F200014EF69E70C3F6275089
:100A000008602D9848B9FFE730982F992E9A00F08A
:100A1000DDFD8DF8C70000F0D2BD2D98006809906B
:100A20002D98406808902D98806807909DED090AE0
:100A3000B5EE400AF1EE10FA19D1FFE79DED080A74
:100A4000B5EE400AF1EE10FA11D1FFE79DED070A6D
:100A5000B5EE400AF1EE10FA09D1FFE730982F9970
:100A60002E9A00F0B3FD8DF8C70000F0A8BD2F98B6
:100A7000006806902F98406805902F988068049031
:100A80002E98006803902E98406802902E988068F7
:100A9000019030989DED033A90ED010A90ED022A05
:100AA00090ED031A20EE430A9DED023A22EE032A4E
:100AB00030EE420A9DED012A21EE021A30EE410A83
:100AC000B6EE001A20EE010A8DED270A30989DED52
:100AD000034A90ED000A90ED023A90ED032A20EED1
:100AE000040A9DED014A23EE043A30EE030A9DED1F
:100AF000023A22EE032A30EE420A20EE010A8DED80
:100B0000260A30989DED024A90ED000A90ED013AD8
:100B100090ED032A20EE040A9DED014A23EE043AEB
:100B200030EE430A9DED033A22EE032A30EE020A2C
:100B300020EE010A8DED250A30989DED014A90EDD9
:100B4000000A90ED013A90ED022A20EE040A9DED94
:100B5000024A23EE043A30EE030A9DED033A22EEF8
:100B6000032A30EE420A20EE010A8DED240A9DEDA3
:100B7000060AB5EE400AF1EE10FA11D1FFE79DED3D
:100B8000050AB5EE400AF1EE10FA09D1FFE79DED36
:100B9000040AB5EE400AF1EE10FA00F09984FFE77E
:100BA0009DED060A20EE000A9DED051A21EE011AC0
:100BB00030EE010A9DED041A21EE011A30EE010A11
:100BC00009F0F2FE8DED2C0A9DED2C1A9DED060A22
:100BD00020EE010A8DED060A9DED2C1A9DED050A09
:100BE00020EE010A8DED050A9DED2C1A9DED040AFB
:100BF00020EE010A8DED040A9DED090A20EE000A9F
:100C00009DED081A21EE011A30EE010A9DED071A3A
:100C100021EE011A30EE010A09F0C6FE8DED2C0A14
:100C20009DED2C1A9DED090A20EE010A8DED090AB1
:100C30009DED2C1A9DED080A20EE010A8DED080AA3
:100C40009DED2C1A9DED070A20EE010A8DED070A95
:100C5000309890ED000A30EE000A9DED091A20EE62
:100C6000010A8DED210A309890ED000A30EE000A5D
:100C70009DED081A20EE010A8DED200A309890EDC6
:100C8000000A30EE000A9DED071A20EE010A8DEDF4
:100C90001F0A309890ED010A30EE000A9DED091A06
:100CA00020EE010A8DED1E0A309890ED000A30EE1C
:100CB000000A8DED190A309890ED010A30EE000A15
:100CC0008DED180A309890ED020A30EE000A8DED95
:100CD000170A309890ED030A30EE000A8DED160ADF
:100CE000309890ED000A90ED021A30EE000A20EEE6
:100CF000010A8DED150A309890ED020A90ED031A65
:100D000030EE000A20EE010A8DED140A309890EDC5
:100D1000000A20EE000A8DED130A309890ED000ACB
:100D200090ED011A20EE010A8DED120A309890ED37
:100D3000000A90ED021A20EE010A8DED110A30989A
:100D400090ED000A90ED031A20EE010A8DED100AD5
:100D5000309890ED010A20EE000A8DED0F0A3098D0
:100D600090ED010A90ED021A20EE010A8DED0E0AB7
:100D7000309890ED010A90ED031A20EE010A8DEDF6
:100D80000D0A309890ED020A20EE000A8DED0C0A53
:100D9000309890ED020A90ED031A20EE010A8DEDD5
:100DA0000B0A309890ED030A20EE000A8DED0A0A36
:100DB0009DED091A9DED130A21EE000A9DED202AF2
:100DC000309890ED025A90ED033A22EE032A30EE6D
:100DD000420A9DED1F2A22EE052A30EE020A9DED01
:100DE0000F2A21EE022A30EE020A9DED182A9DED0F
:100DF000084A22EE044A24EE054A30EE040A9DED2C
:100E0000074A22EE042A22EE032A30EE020A9DED62
:100E10000C2A21EE022A30EE420A9DED0A2A21EE2A
:100E2000021A30EE410A8DED230A9DED210A309819
:100E300090ED015A90ED024A90ED033A20EE030A3C
:100E40009DED081A9DED132A21EE022A30EE020ACA
:100E50009DED1F2A22EE052A30EE420A9DED1E2A44
:100E600022EE042A30EE020A9DED0F2A21EE022A1C
:100E700030EE420A9DED0C2A21EE022A30EE020AE3
:100E80009DED172A9DED074A22EE042A22EE032A41
:100E900030EE020A9DED0A2A21EE021A30EE410AD6
:100EA0008DED220A9DED230A20EE000A9DED221A07
:100EB00021EE011A30EE010A09F076FDB7EE006A64
:100EC00086EE000A8DED1D0A9DED210A309890ED09
:100ED000012A90ED021A90ED033A20EE011A9DEDE1
:100EE000200A20EE020A30EE412A9DED071A9DED00
:100EF000130A21EE000A30EE022A9DED1E0A20EEB2
:100F0000030A30EE020A9DED0F2A21EE022A30EE8E
:100F1000420A9DED172A9DED084A22EE042A22EE90
:100F2000032A30EE020A9DED0C2A21EE022A30EE51
:100F3000420A9DED0A2A21EE021A30EE010A8DEDD9
:100F40001C0A9DED1D0A30EE000A8DED1B0A9DED79
:100F50001C0A30EE000A8DED1A0A9DED170ADDED30
:100F60000D0A30EEA02A9DED151A31EE422A9DEDB4
:100F7000061A31EE021A20EE010A9DED181ADDED77
:100F8000123A33EEA32A9DED143A32EE032A9DED78
:100F9000053A32EE432A21EE021A70EE014A9DED27
:100FA0001C3A309890ED011A90ED020AD0ED032A18
:100FB00063EE001A9DED1D2A9DED0C7AB6EE004AF7
:100FC0008DED004A77EE445A9DED0A5A35EE255ACA
:100FD00062EE055A9DED115A75EE606A63EE266A5F
:100FE00075EEA66ADDED095A75EEA65A61EEA51AF0
:100FF00071EEA41A62EE222A23EE011A31EE621A71
:10100000DDED0E2ADDED104A72EEE42A62EE222AB0
:10101000DDED0B4A73EEA43A63EE233A72EEA32A97
:10102000DDED083A72EEE32A21EE221A31EE211AA2
:1010300022EE000A35EE205A22EE052A9DED0F5AC7
:1010400034EE455A35EE475A23EE053A32EE032A7E
:101050009DED073A32EE432A20EE020A30EE010AF5
:101060008DED2B0A9DED160ADDED0D2A32EEA21A4A
:101070009DED152A31EE421A9DED062A31EE421AF7
:1010800020EE010A9DED191ADDED126A36EEA62A50
:101090009DED143A32EE032A9DED053A32EE432AD5
:1010A00021EE021A30EE011A3098D0ED005AD0ED40
:1010B000014AD0ED023A90ED032AB1EE000A24EE87
:1010C000803A9DED0F7A37EE075A75EE461ADDED40
:1010D0000C0A30EEA05A75EE211A9DED045A35EE39
:1010E000215A23EE053A31EE031A9DED1C5A65EEA6
:1010F000027A9DED1D3A74EE601A9DED0A8A71EE3A
:10110000C81A23EE218ADDED111A32EEE19A25EE9E
:10111000099A38EE098A9DED099A38EE498A67EEF8
:10112000887A31EE271A63EE233A65EE255A73EE7C
:10113000A53ADDED0E5ADDED107A75EEE75A63EE55
:10114000255ADDED0B7A76EEA76A65EE266A75EE16
:10115000A65ADDED086A75EEE65A63EEA53A31EE61
:10116000231A23EE022ADDED1A3A63EEA43A32EE98
:10117000632A71EEA21A23EE213A34EE477A37EE53
:10118000607A25EE075A33EE053A9DED075A33EEA5
:10119000453A22EE032A31EE021A8DED2A1A9DED10
:1011A000191ADDED0D0A30EEA03A9DED152A32EE4A
:1011B000433A9DED062A32EE032A21EE021A9DEDF6
:1011C000162ADDED124A34EEA43A9DED145A33EEA0
:1011D000053A9DED055A33EE453A22EE032A31EEEB
:1011E000022A309890ED001AD0ED011AD0ED022AB3
:1011F000D0ED033A22EE800A9DED0F5A35EE053A06
:1012000033EE467A9DED0C6A36EE063A33EE077AF7
:101210009DED043A33EE073A20EE030A70EE025ACF
:101220009DED1B0A20EE620A9DED1C3A23EE012A79
:1012300030EE420A9DED1D2A34EE467ADDED0A6A53
:1012400037EE667A62EE076A9DED117A70EEC77A24
:1012500063EE277A76EEA76ADDED097A76EEE76A25
:1012600020EE260A30EE250A62EE211A63EE233ABA
:1012700071EEA31ADDED0E3ADDED105A73EEE53A8C
:1012800062EE233ADDED0B5A74EEA54A63EE244A72
:1012900073EEA43ADDED084A73EEE43A61EEA31A68
:1012A00030EE210A22EE011ADDED1A1A61EEA21AC1
:1012B00031EE611A37EE207A22EE072A34EE455AD3
:1012C00035EE465A23EE053A32EE032A9DED073AF3
:1012D00032EE432A21EE021A30EE010A8DED290A80
:1012E0009DED180A9DED0D7A37EE071A9DED152A32
:1012F00031EE421A9DED062A31EE421A20EE010A25
:101300009DED171ADDED122A32EEA22A9DED143A58
:1013100032EE032A9DED053A32EE432A21EE021AFF
:1013200070EE013A9DED1B1A3098D0ED001A90ED49
:10133000010AD0ED020A90ED032A21EE022A9DED6A
:101340001C3A23EE001A31EE421A9DED1D2A9DED46
:101350000C5A34EE456ADDED0A4A36EE646A62EEF6
:10136000064A9DED116A77EE465A63EE255A74EEF1
:10137000A54ADDED095A74EEE54A21EE241A31EE54
:10138000231A62EE211A63EE200A70EEE10ADDED07
:101390000E1ADDED103A71EEE31A62EE211ADDED60
:1013A0000B3A72EEA32A63EE222A71EEA21ADDED49
:1013B000082A71EEE21A60EEA10A31EE201A22EE3E
:1013C000000A36EE076A22EE062A9DED0F6A34EE19
:1013D000464A34EE454A23EE043A32EE032A9DEDA6
:1013E000073A32EE432A20EE020A30EE010A8DED72
:1013F000280A9DED2B0A20EE000A9DED2A1A21EE07
:10140000011A30EE010A9DED291A21EE011A30EE83
:10141000010A9DED281A21EE011A30EE010A09F0A9
:10142000C3FA8DED2C0A9DED2C1A9DED2B0A20EEB2
:10143000010A8DED2B0A9DED2C1A9DED2A0A20EE56
:10144000010A8DED2A0A9DED2C1A9DED290A20EE48
:10145000010A8DED290A9DED2C1A9DED280A20EE3A
:10146000010A8DED280A40F20400C2F2000090ED5E
:10147000000A9DED2B1A20EE011A9DED270A30EE91
:10148000410A8DED270A90ED000A9DED2A1A20EE03
:10149000011A9DED260A30EE410A8DED260A90EDE7
:1014A000000A9DED291A20EE011A9DED250A30EE65
:1014B000410A8DED250A90ED000A9DED281A20EED7
:1014C000011A9DED240A30EE410A8DED240AFFE752
:1014D0009DED271A309890ED000A90ED042A21EE38
:1014E000021A30EE010A80ED000A9DED261A3098AE
:1014F00090ED010A90ED042A21EE021A30EE010A65
:1015000080ED010A9DED251A309890ED020A90EDCC
:10151000042A21EE021A30EE010A80ED020A9DED46
:10152000241A309890ED030A90ED042A21EE021A55
:1015300030EE010A80ED030A309890ED000A90ED3C
:10154000013A90ED022A90ED031A20EE000A23EEF4
:10155000033A30EE030A22EE022A30EE020A21EEAE
:10156000011A30EE010A09F01FFA8DED2C0A9DEDEB
:101570002C1A309890ED000A20EE010A80ED000A46
:101580009DED2C1A309890ED010A20EE010A80EDB5
:10159000010A9DED2C1A309890ED020A20EE010A06
:1015A00080ED020A9DED2C1A309890ED030A20EE92
:1015B000010A80ED030A00208DF8C700FFE79DF9BE
:1015C000C70032B0BDEC048B80BD000080B5A0B078
:1015D0001E901D911C921E9820B9FFE7FF208DF8E8
:1015E0007F00D3E21D9820B9FFE7FF208DF87F0030
:1015F000CCE21C9820B9FFE7FF208DF87F00C5E200
:1016000040F20401C2F2000142F60230C3F6075074
:1016100008601D9800681B901D9840681A901D98DE
:10162000806819901C98006818901C984068179062
:101630001C98806816901E989DED183A90ED010A4E
:1016400090ED022A90ED031A20EE430A9DED173A21
:1016500022EE032A30EE420A9DED162A21EE021AEE
:1016600030EE410AB6EE001A20EE010A8DED100AA6
:101670001E989DED184A90ED000A90ED023A90ED0B
:10168000032A20EE040A9DED164A23EE043A30EEBA
:10169000030A9DED173A22EE032A30EE420A20EEAD
:1016A000010A8DED0F0A1E989DED174A90ED000A74
:1016B00090ED013A90ED032A20EE040A9DED164AC2
:1016C00023EE043A30EE430A9DED183A22EE032A47
:1016D00030EE020A20EE010A8DED0E0A1E989DEDF5
:1016E000164A90ED000A90ED013A90ED022A20EEA4
:1016F000040A9DED174A23EE043A30EE030A9DEDED
:10170000183A22EE032A30EE420A20EE010A8DED4D
:101710000D0A9DED1B0AB5EE400AF1EE10FA11D14B
:10172000FFE79DED1A0AB5EE400AF1EE10FA09D175
:10173000FFE79DED190AB5EE400AF1EE10FA00F050
:10174000AE81FFE79DED1B0A20EE000A9DED1A1AFF
:1017500021EE011A30EE010A9DED191A21EE011A4F
:1017600030EE010A09F020F98DED150A9DED151AEC
:101770009DED1B0A20EE010A8DED1B0A9DED151A49
:101780009DED1A0A20EE010A8DED1A0A9DED151A3B
:101790009DED190A20EE010A8DED190A1E9890EDB3
:1017A000000A30EE000A8DED0C0A1E9890ED010A39
:1017B00030EE000A8DED0B0A1E9890ED020A30EE15
:1017C000000A8DED0A0A1E9890ED030A30EE000A19
:1017D0008DED090A1E9890ED000AB1EE003A20EE58
:1017E000030A8DED080A1E9890ED010A20EE030A07
:1017F0008DED070A1E9890ED020A20EE030A8DED8A
:10180000060A1E9890ED010AB2EE001A20EE010AB7
:101810008DED050A1E9890ED020A20EE010A8DED6D
:10182000040A1E9890ED000A20EE000A8DED030ACE
:101830001E9890ED010A20EE000A8DED020A1E9816
:1018400090ED020A20EE000A8DED010A1E9890ED3F
:10185000030A20EE000A8DED000A9DED081A9DEDA9
:10186000010A21EE000A9DED0A2A9DED1B4A22EE97
:10187000042A30EE020A9DED022A21EE021A30EE11
:10188000010A9DED0B1A9DED1A2A21EE021A30EE87
:10189000410A8DED140A9DED071A9DED000A21EE17
:1018A000000A9DED092A9DED1B4A22EE042A30EE26
:1018B000420A9DED032A22EE032A1E9890ED014A6A
:1018C00022EE042A30EE020A9DED0C2A9DED1A4A02
:1018D00022EE042A30EE420A30EE410A9DED052A3E
:1018E0009DED024A22EE044A30EE040A9DED014AC3
:1018F00022EE042A30EE020A9DED192A21EE021A88
:1019000030EE010A8DED130A9DED030A20EE030A65
:101910001E9890ED021A20EE010A9DED0C1A9DED25
:101920001B2A21EE021A30EE010A9DED061A9DEDEA
:10193000002A21EE022A30EE020A9DED092A9DEDD1
:101940001A4A22EE042A30EE420A30EE410A9DED98
:10195000042A9DED024A22EE044A30EE040A9DED6F
:10196000014A22EE042A30EE020A9DED192A21EEE8
:10197000021A30EE010A8DED120A9DED020A20EEE8
:10198000030A1E9890ED032A20EE020A9DED0B1A21
:101990009DED1B4A21EE041A30EE410A9DED011A1D
:1019A00021EE031A21EE021A30EE010A9DED0A1A09
:1019B0009DED1A2A21EE021A30EE410A8DED110A30
:1019C0009DED140A20EE000A9DED131A21EE011A76
:1019D00030EE010A9DED121A21EE011A30EE010AD5
:1019E0009DED111A21EE011A30EE010A08F0DCFF1C
:1019F0008DED150A9DED151A9DED140A20EE010AD4
:101A00008DED140A9DED151A9DED130A20EE010AC5
:101A10008DED130A9DED151A9DED120A20EE010AB7
:101A20008DED120A9DED151A9DED110A20EE010AA9
:101A30008DED110A40F20400C2F2000090ED000AA0
:101A40009DED141A20EE011A9DED100A30EE410AA8
:101A50008DED100A90ED000A9DED131A20EE011A8B
:101A60009DED0F0A30EE410A8DED0F0A90ED000A50
:101A70009DED121A20EE011A9DED0E0A30EE410A7C
:101A80008DED0E0A90ED000A9DED111A20EE011A5F
:101A90009DED0D0A30EE410A8DED0D0AFFE79DED3B
:101AA000101A1E9890ED000A90ED042A21EE021AF9
:101AB00030EE010A80ED000A9DED0F1A1E9890EDA0
:101AC000010A90ED042A21EE021A30EE010A80ED9F
:101AD000010A9DED0E1A1E9890ED020A90ED042A5F
:101AE00021EE021A30EE010A80ED020A9DED0D1A78
:101AF0001E9890ED030A90ED042A21EE021A30EEB2
:101B0000010A80ED030A1E9890ED000A90ED013A5B
:101B100090ED022A90ED031A20EE000A23EE033A1C
:101B200030EE030A22EE022A30EE020A21EE011AFA
:101B300030EE010A08F038FF8DED150A9DED151AFB
:101B40001E9890ED000A20EE010A80ED000A9DED3E
:101B5000151A1E9890ED010A20EE010A80ED010A87
:101B60009DED151A1E9890ED020A20EE010A80EDF7
:101B7000020A9DED151A1E9890ED030A20EE010A47
:101B800080ED030A00208DF87F00FFE79DF97F00BC
:101B900020B080BD84B08DED030ACDED020A9DED2D
:101BA000030A9DED021AB1EE411AB4EE410AF1EEBC
:101BB00010FA07DAFFE79DED020AB1EE400A8DED5B
:101BC000010A18E09DED030A9DED021AB4EE410AE8
:101BD000F1EE10FA05DDFFE79DED020A8DED000A3A
:101BE00004E09DED030A8DED000AFFE79DED000A7C
:101BF0008DED010AFFE79DED010A04B0704700007A
:101C000080B541F61C70C2F20000006808210EF099
:101C100069FE80BD80B582B040F23862C2F2000237
:101C2000002001901221132300F02CFA019802B039
:101C300080BD000080B5022001214FF0FF320EF080
:101C4000A3FE80BD81B000909FED010A01B07047F6
:101C50000000C84380B541F61C70C2F20000006865
:101C600010210EF03FFE80BD80B540F23860C2F218
:101C70000000C21D01200221062300F003FA00200B
:101C800080BD000080B5042001214FF0FF320EF02E
:101C90007BFE80BD80B58AB008900791089820B976
:101CA000FFE7FE208DF82700B4E0079820B9FFE792
:101CB000FE208DF82700ADE041F22150C2F2000075
:101CC0000078C00720B1FFE7FD208DF82700A1E0D4
:101CD0000EF0E8FE41F61C71C2F20001086020B966
:101CE000FFE7FE208DF8270094E007980899C86266
:101CF000002006907E21B622049200F059FA049A40
:101D00000120142100F054FA1E20059001F0A8FAD9
:101D10000599069800F0F2F90699084600F0EEF9E8
:101D20001E2804D0FFE7FC208DF8270072E0012078
:101D3000002100F0E3F90F2804D0FFE7FC208DF824
:101D4000270067E00320019001F014F804200290BE
:101D500001F010F842F22902C0F6000200200390C0
:101D60000121009101F01AFA019841F60141C0F6F3
:101D7000000101F085F8029841F65541C0F60001D6
:101D800001F07EF803984021AA2200F011FA009A8F
:101D90000398412100F00CFA03985321082200F027
:101DA00007FA029A0398582100F002FA029A03985F
:101DB0007D2100F0FDF9322001F052FA009A0F2146
:101DC000104600F0F5F90098019A102100F0F0F9A2
:101DD0000098039A162100F0EBF9009A182110469A
:101DE00000F0E6F900981521802200F0E1F90A20C0
:101DF00001F036FA0099019841F22152C2F2000234
:101E0000117000F0E7FF029800F0E4FF03988DF8EE
:101E10002700FFE79DF927000AB080BD84B002903B
:101E2000029820B9FFE7FE208DF80F006AE040F22B
:101E30003861C2F20001B1F80100ADF80600B1F856
:101E40000300ADF80400B1F80500ADF80200BDF9DB
:101E5000060000EE100AB8EEC00A029880ED040AEF
:101E6000BDF9040000EE100AB8EEC00A029880ED39
:101E7000050ABDF9020000EE100AB8EEC00A029889
:101E800080ED060A029890ED040A9FED201A80EE7C
:101E9000010A80ED040A029890ED050A80EE010A1D
:101EA00080ED050A029890ED060A80EE010A80EDA9
:101EB000060A487C897CC00040EA5110ADF8000059
:101EC000BDF90000B0F5806F07DBFFE7BDF800004B
:101ED000A0F50060ADF80000FFE7BDF9000000EEDE
:101EE000100AB8EEC00AB4EE001A20EE010AB3EEF2
:101EF000071A30EE010A029880ED0A0A00208DF8D8
:101F00000F00FFE79DF90F0004B0704700A0AA453D
:101F100084B00290029820B9FFE7FE208DF80F00F0
:101F20007AE040F23860C2F20000B0F80710ADF875
:101F30000610B0F80910ADF80410B0F80B00ADF8B9
:101F40000200BDF9060000EE100AB8EEC00A0298C1
:101F500080ED070ABDF9040000EE100AB8EEC00AD1
:101F6000029880ED080ABDF9020000EE100AB8EEF2
:101F7000C00A029880ED090A029890ED070A9FEDC9
:101F8000281A80EE010A80ED070A029890ED080AEF
:101F900080EE010A80ED080A029890ED090A80EEB1
:101FA000010A80ED090A029890ED070A9FED1D1ABB
:101FB00020EE010A80ED070A029890ED080A20EE53
:101FC000010A80ED080A029890ED090A20EE010A44
:101FD00080ED090A0298C16A91ED001A90ED070A96
:101FE00030EE410A80ED070A0298C16A91ED011AAC
:101FF00090ED080A30EE410A80ED080A0298C16AA5
:1020000091ED021A90ED090A30EE410A80ED090ABD
:10201000FE208DF80F00FFE79DF90F0004B0704718
:102020006F12034235FA8E3C80B5012000F002FFAA
:1020300068B9FFE70121084600F06AFF41F61C700D
:10204000C2F20000006802210EF04CFCFFE7022003
:1020500000F0F0FE68B9FFE70220012100F058FF10
:1020600041F61C70C2F20000006804210EF03AFC38
:10207000FFE780BD80B5182001214FF0FF320EF040
:1020800083FC80BD80B586B08DF817008DF81610E2
:1020900004928DF80F30049808B9FFE72BE09DF803
:1020A00017000146029120B1FFE70298012805D0F0
:1020B00009E00120002100F02BFF04E002200021B4
:1020C00000F026FFFFE79DF8160040F0800040F288
:1020D0004B61C2F2000108700122009200230193BB
:1020E000184601F07DF8009B019804999DF80F2097
:1020F00001F014F8FFE706B080BD000080B586B09F
:102100008DF816008DF81510012001F0A9F89DF842
:1021100016000146049120B1FFE70498012805D07C
:1021200009E00120002100F0F3FE04E0022000217C
:1021300000F0EEFEFFE79DF8150040F0800040F251
:102140004B61C2F200010191087001220023029349
:10215000184601F045F80199029B0222184600F04A
:10216000DDFF9DF816000146039120B1FFE70398BB
:1021700001280CD017E00121084600F0C9FE40F20A
:102180004B60C2F2000040788DF817000BE002208F
:10219000012100F0BDFE40F24B60C2F20000007869
:1021A0008DF81700FFE79DF8170006B080BD00000E
:1021B00080B584B08DF80F008DF80E108DF80D20CD
:1021C0009DF80E0000F07F0040F24B61C2F200016A
:1021D00008709DF80D004870012001F041F89DF84D
:1021E0000F000146029120B1FFE70298012805D0B7
:1021F00009E00120002100F08BFE04E00220002114
:1022000000F086FEFFE740F24B61C2F200010222BD
:102210000023184600F0E4FF9DF80F0001460191ED
:1022200020B1FFE70198012805D009E00121084607
:1022300000F06EFE04E00220012100F069FEFFE7DD
:1022400004B080BD80B586B08DF8160004918DF87D
:102250000F209DF80F0020B9FFE70A208DF80F002E
:10226000FFE741F6B420C2F20000006864210EF0DE
:1022700015FA20B1FFE7FB208DF8170070E041F65A
:10228000B020C2F2000000680290FFE70298E0B1BF
:10229000FFE7029800789DF81610884211D1FFE7F9
:1022A00002984068049988420BD1FFE741F6B420B8
:1022B000C2F2000000680EF0D5FAFF208DF817007A
:1022C0004EE0029800690290E0E7142000F048FE1A
:1022D0000190019858B9FFE741F6B420C2F200001E
:1022E00000680EF0BFFAFE208DF8170038E09DF868
:1022F0000F001C2100220EF0CFF801998860019890
:10230000806870B9FFE7019800F02CFD41F6B42019
:10231000C2F2000000680EF0A5FAFF208DF8170049
:102320001EE09DF816000199087004980199486014
:102330009DF80F000199087341F6B021C2F2000127
:102340000868019A10610198086041F6B420C2F251
:10235000000000680EF086FA00208DF81700FFE7F5
:102360009DF9170006B080BD82B001908DF8031072
:10237000019802B07047000084B08DF80B00019105
:1023800041F6B020C2F2000000680090FFE700981C
:10239000A8B1FFE7009800789DF80B1088420AD199
:1023A000FFE7009840680199884204D1FFE7009850
:1023B0008068039006E0009800690090E7E700203D
:1023C0000390FFE7039804B07047000082B00090CC
:1023D0000098C068022809D1FFE7009881680220B0
:1023E000042908BF03208DF8070008E000988068E2
:1023F0000438B0FA80F040098DF80700FFE79DF837
:10240000070002B07047000083B08DF807009DF808
:102410000700022803DBFFE70020029018E09DF888
:1024200007000146009120B1FFE70098012806D07F
:102430000BE041F2CC00C2F20000029008E041F251
:10244000F400C2F20000029002E000200290FFE7D8
:10245000029803B07047000080B586B08DF8160072
:1024600004910392029341F22050C2F200000078DE
:10247000C00720B9FFE7FD208DF8170037E003986B
:1024800020B9FFE7FE208DF8170030E041F6B420B8
:10249000C2F20000006864210EF000F920B1FFE7ED
:1024A000FB208DF8170022E09DF816000499FFF735
:1024B00063FF019041F6B420C2F2000000680EF004
:1024C000D1F9019820B9FFE7FC208DF817000EE044
:1024D00001980399029B00220DF07EFF0090009866
:1024E000002818BF4FF0FF308DF81700FFE79DF967
:1024F000170006B080BD000080B596B041F22050B4
:10250000C2F200000078C00720B1FFE7FD208DF87F
:102510005700A7E040F29440C2F200006821FDF7A6
:10252000DAFF00201490FFE71498012809DCFFE788
:102530009DF8500000F01CFBFFE714980130149048
:10254000F2E741F2D441C2F2000142F26930C0F632
:102550000000086000200EF0F1F8014641F6B420BA
:10256000C2F200000160006820B9FFE7FF208DF88B
:10257000570077E041F22051C2F20001079101209B
:10258000089008700AA803902821FDF7A4FF03997A
:10259000089A002009900F900A900B9010901192C9
:1025A0000C900D9012920E22029213920E9041F214
:1025B000CC00C2F20000019003F016FD019804F077
:1025C000FFFB099842F27972C0F60002062100F082
:1025D0006FF8099942F6F922C0F600020592084602
:1025E00000F066F8059A0899099800F061F8059AD4
:1025F00009980221049100F05BF80198032103F08F
:102600001DFC029A039908980F920E9041F2F40073
:10261000C2F20000069003F0E7FC069804F0D0FB3D
:10262000089842F65D02C0F60002082100F040F86A
:10263000059A0999089800F03BF8059A0899084608
:1026400000F036F80499059A089800F031F80698D9
:10265000112103F0F3FB079A0899099811708DF87E
:102660005700FFE79DF9570016B080BD80B584B0D4
:1026700002908DF8071041F2D440C2F200000068C9
:1026800058B1FFE741F2D440C2F20000026802985C
:102690009DF807109047039006E002989DF80710F8
:1026A000FFF762FE0390FFE7039804B080BD0000CF
:1026B00082B08DF806008DF80510009241F220508E
:1026C000C2F200000078C00720B9FFE7FD208DF8B6
:1026D00007002AE0009820B9FFE7FE208DF80700E8
:1026E00023E09DF80600022804DBFFE7FF208DF8B9
:1026F00007001AE09DF805000D2804DBFFE7FF2026
:102700008DF8070011E000989DF8061040F2944300
:10271000C2F20003342211FB02319DF8052041F87A
:10272000220000208DF80700FFE79DF9070002B0A6
:102730007047000080B584B08DF80E0002918DF8CE
:10274000072041F22050C2F200000078C00720B9F3
:10275000FFE7FD208DF80F0009E09DF80E000299BB
:102760009DF80720FFF76EFD8DF80F00FFE79DF93C
:102770000F0004B080BD000080B598B000200E901E
:10278000FFE70E98012867DCFFE79DF83800FFF7A8
:102790003BFE0D900D9808B9FFE759E0FFE70D9853
:1027A000002103F019FD002851D0FFE70D9800210A
:1027B00011AA0FAB03F03AFD002847D1FFE71398A9
:1027C00018B9FFE71198019002E012980190FFE715
:1027D00001980C9011A8FFF7F9FD8DF82F000C98C7
:1027E0009DF82F10FFF742FF0A909DF838000A99D4
:1027F000FFF7C2FD0990099838B3FFE70020089061
:102800000790069005900490039002909DF82F0089
:102810008DF808000C9803900A98049015988DF88C
:102820001400149838B9FFE702A80D30159A0FA9C3
:10283000FDF7D2FDFFE705F0DFF90890099802A93E
:1028400000231A460DF0A8FEFFE7FFE7A7E7FFE722
:102850000E9801300E9094E718B080BD80B598B006
:1028600000200E90FFE70E98012867DCFFE79DF837
:102870003800FFF7C9FD0D900D9808B9FFE759E042
:10288000FFE70D98012103F0A7FC002851D0FFE7D6
:102890000D98012111AA0FAB03F0C8FC002847D105
:1028A000FFE7139818B9FFE71198019002E012981A
:1028B0000190FFE701980C9011A8FFF787FD8DF8B4
:1028C0002F000C989DF82F10FFF7D0FE0A909DF86E
:1028D00038000A99FFF750FD0990099838B3FFE7CF
:1028E00000200890079006900590049003900290B5
:1028F0009DF82F008DF808000C9803900A9804901A
:1029000015988DF81400149838B9FFE702A80D3017
:10291000159A0FA9FDF760FDFFE705F06DF9089026
:10292000099802A900231A460DF036FEFFE7FFE7DB
:10293000A7E7FFE70E9801300E9094E718B080BD2E
:1029400080B592B0844614988DF846C08DF8451035
:1029500010920F938DF83B0041F22050C2F200001C
:102960000078C00720B9FFE7FD208DF847009EE002
:102970009DF84600022804DBFFE7FF208DF84700A2
:1029800095E00F9870B9FFE79DF84500022809D03F
:10299000FFE79DF84500032804D0FFE7FE208DF8EF
:1029A000470084E09DF83B00092804DBFFE7FF2097
:1029B0008DF847007BE09DF84600FFF725FD0D9060
:1029C0000D9820B9FFE7FE208DF847006FE000204A
:1029D00001900C900B900A90099008900790069037
:1029E00005909DF845000146029103281FD80299E1
:1029F000DFE801F002080F161098059000200790FC
:102A0000089018E010980690042007900020089085
:102A100011E01098059000200790022008900AE02D
:102A200010980690042007900220089003E0FF20F1
:102A30008DF847003BE09DF83B00099000208DF8A1
:102A400028000F9868B1FFE79DF83B00012808DBDC
:102A5000FFE705A818300F999DF83B20FDF7BCFC57
:102A6000FFE70D9803F0ECFC90B1FFE70D9805A986
:102A700001F1180204AB03F00BFA8DF80F009DF87A
:102A80000F0020B9FFE700208DF847000FE0FFE7B7
:102A90009DF8460005A900F00FF920B1FFE70020DE
:102AA0008DF8470003E0FF208DF84700FFE79DF910
:102AB000470012B080BD000080B584B08DF80E00D4
:102AC0000291029820B9FFE7FE208DF80F000EE07A
:102AD0009DF80E0002990A684B1D0979EC46CCF866
:102AE00000100021FFF72CFF8DF80F00FFE79DF984
:102AF0000F0004B080BD000080B58CB000200B90AA
:102B0000FFE70B98012831DCFFE70B988DF82B00CD
:102B10009DF82B00FFF778FC0990099808B9FFE7AA
:102B200020E0FFE79DF82B0000F044F8C8B9FFE76C
:102B3000099803F085FC08B9FFE712E09DF82B0027
:102B400001A900F063F808B9FFE70AE0099801A9B4
:102B500001F118026B4603F09BF908B1FFE700E0B2
:102B6000E0E7FFE70B9801300B90CAE70CB080BD9F
:102B700081B08DF803009DF80300022801DBFFE718
:102B800015E09DF8030000EBC01041F62471C2F27D
:102B9000000101EBC0020020C2F800049DF80320F0
:102BA00002EBC21201EBC201C1F80404FFE701B05D
:102BB0007047000081B08DF802009DF802000228E5
:102BC00004DBFFE701208DF803001AE09DF8020006
:102BD00000EBC01041F62471C2F2000101EBC0000D
:102BE000D0F800049DF8022002EBC21201EBC201F2
:102BF000D1F80414401AB0FA80F040098DF80300AF
:102C0000FFE79DF8030001B070470000B0B584B045
:102C10008DF80E0002919DF80E00012803DCFFE7FD
:102C2000029820B9FFE700208DF80F0040E09DF8E2
:102C30000E0000EBC01141F62470C2F2000000EB60
:102C4000C10001900198D0F800040199D1F8041452
:102C5000884204D1FFE700208DF80F0028E0029998
:102C600000910198D0F8043400EB43125B01C05886
:102C70005368D2F808C0D2F80CE0146955694D6168
:102C80000C61C1F80CE0C1F808C04B6008609069A5
:102C9000D269CA6188610198D0F80404013000F05B
:102CA0001F000199C1F8040401208DF80F00FFE70F
:102CB0009DF80F0004B0B0BDF0B585B08DF81200DE
:102CC00003919DF81200012803DCFFE7039820B967
:102CD000FFE700208DF8130040E09DF8120000EBA4
:102CE000C01141F62470C2F2000000EBC100029056
:102CF0000298D0F80004013000F01F000190019804
:102D00000299D1F80414884204D1FFE700208DF81D
:102D1000130023E0029ED6F8000406EB40114701A1
:102D2000039A0092D2F810E05469156850689368CD
:102D3000D2F80CC0F5514C61C1F810E0C1F80CC0DC
:102D40008B6048609069D269CA6188610198029974
:102D5000C1F8000401208DF81300FFE79DF813006F
:102D600005B0F0BD80B582B0019001980FF010FA67
:102D700002B080BD80B582B08DF806009DF80600D7
:102D80000146009140B1FFE7009803280BD0FFE710
:102D9000009804280ED014E0062004F0C1FF0020A3
:102DA0008DF8070011E00A2004F0BAFF00208DF82A
:102DB00007000AE0172004F0B3FF00208DF8070099
:102DC00003E0FF208DF80700FFE79DF9070002B040
:102DD00080BD000080B582B08DF806009DF8060029
:102DE0000146009140B1FFE7009803280BD0FFE7B0
:102DF000009804280ED014E0062004F09BFF002069
:102E00008DF8070011E00A2004F094FF00208DF8EF
:102E100007000AE0172004F08DFF00208DF807005E
:102E200003E0FF208DF80700FFE79DF9070002B0DF
:102E300080BD000080B582B08DF806009DF80600C8
:102E4000082804DBFFE700208DF8070013E09DF859
:102E5000062048F24811C0F6010101EBC2004068AB
:102E600031F8321004F098FE0138B0FA80F04009D1
:102E70008DF80700FFE79DF8070002B080BD000055
:102E800083B08DF80A000191019820B9FFE7FE2078
:102E90008DF80B0038E09DF80A00082804DBFFE7F6
:102EA000FF208DF80B002FE09DF80A1048F2481023
:102EB000C0F6010030F83100ADF8020000208DF8B6
:102EC0000100FFE79DF801000F2819DCFFE7BDF8BE
:102ED00002009DF80110C840C00750B1FFE70198FB
:102EE0009DF8012040F2FC41C2F2000141F82200AD
:102EF00006E0FFE79DF8010001308DF80100E1E7F1
:102F000000208DF80B00FFE79DF90B0003B0704720
:102F100080B582B08DF806008DF805109DF806008A
:102F2000082804DBFFE7FF208DF8070014E09DF878
:102F3000062048F24811C0F6010101EBC2004068CA
:102F400031F832109DF8052002F0010204F03CFE39
:102F500000208DF80700FFE79DF9070002B080BD53
:102F600080B582B0019001980EF06AFE02B080BD7B
:102F700086B08DF816008DED040A9DF81600012824
:102F800004DBFFE7FF208DF817008CE09DED040ABD
:102F9000B7EE001AB4EE410AF1EE10FA04DDFFE7D5
:102FA0004FF07E500490FFE79DED040AB5EE400A15
:102FB000F1EE10FA03DAFFE700200490FFE79DF836
:102FC000161048F28810C0F6010050F83110096858
:102FD000C96A03919DED040A0399013101EE101AAB
:102FE000B8EE411A20EE010ABCEEC00A8DED020ACD
:102FF0009DF8161000EBC100808860B9FFE70298C9
:103000009DF8162048F28811C0F6010151F83210DF
:103010000968486343E09DF8161048F28810C0F62E
:10302000010000EBC100808804280DD1FFE7029861
:103030009DF8162048F28811C0F6010151F83210AF
:1030400009688863019028E09DF8161048F28810FE
:10305000C0F6010000EBC100808808280DD1FFE711
:1030600002989DF8162048F28811C0F6010151F827
:1030700032100968C86300900CE002989DF8162091
:1030800048F28811C0F6010151F83210096808644D
:103090000090FFE700980190FFE70198FFE700200C
:1030A0008DF81700FFE79DF9170006B07047000084
:1030B00080B582B08DF806009DF80600012804DB7B
:1030C000FFE7FF208DF8070010E09DF8062048F28A
:1030D0008810C0F6010000EBC20150F83200898868
:1030E00006F066FE00208DF80700FFE79DF9070057
:1030F00002B080BD82B08DF803009DF8030030B9A6
:10310000FFE741F25C30C2F20000019002E00020D3
:103110000190FFE7019802B07047000080B584B0CD
:103120008DF80E000291ADF806208DF805309DF85F
:103130000E00012804DBFFE7FF208DF80F0029E0D7
:103140009DF80E00FFF7D6FF0090009820B9FFE72A
:10315000FF208DF80F001DE09DF80500C00760B14D
:10316000FFE700980299BDF8062005F0DBFD002876
:1031700018BF01208DF80F000CE000980299BDF8EF
:103180000620142305F0A6FC002818BF01208DF8A6
:103190000F00FFE79DF90F0004B080BD82B08DF8ED
:1031A00006008DF805100092009820B9FFE7FE2078
:1031B0008DF8070010E000989DF8062040F2445179
:1031C000C2F2000101EB42119DF8052041F82200F6
:1031D00000208DF80700FFE79DF9070002B0704757
:1031E00080B584B08DF80E000291ADF806208DF800
:1031F00005309DF80E00012804DBFFE7FF208DF865
:103200000F0029E09DF80E00FFF774FF0090009872
:1032100020B9FFE7FF208DF80F001DE09DF80500A5
:10322000C00760B1FFE700980299BDF8062006F0DC
:10323000C7FA002818BF01208DF80F000CE0009895
:103240000299BDF80620142305F08CFE002818BF53
:1032500001208DF80F00FFE79DF90F0004B080BD3D
:1032600080B586B004900DF001F801464FF47A70F5
:10327000B0FBF1F0039004980399B0FBF1F00290D9
:103280000CF0B6FF0146481C019198B1FFE7019888
:10329000022820D3FFE7019802280FD0FFE701980A
:1032A0000338022806D3FFE701986FF000418842F7
:1032B00015D1FFE7FF208DF8170014E0029818B130
:1032C000FFE70298009002E001200090FFE70098DD
:1032D0000CF048FF03E0049804F010FAFFE7002028
:1032E0008DF81700FFE79DF9170006B080BD0000BC
:1032F00080B58AB00CF0BAFF079010F043FD079A32
:103300004FF47A710191B1FBF2F1484306904EF20D
:103310001800CEF2000002900068059010F032FD17
:10332000019A01460298079BB2FBF3F251430491C4
:103330000068039006980499884215D1FFE7049825
:103340004FF47A725043059951434EF21402CEF273
:10335000000212680132B1FBF2F1401A00F57A70F6
:1033600000210991089014E004984FF47A725043B8
:10337000039951434EF21402CEF200021268013258
:10338000B1FBF2F1401A00F57A7000210991089022
:10339000FFE7089809990AB080BD000083B08DF856
:1033A00007009DF807000146009140B1FFE7009833
:1033B00001280AD0FFE7009802280CD011E041F262
:1033C0004440C2F2000002900EE041F28C40C2F292
:1033D0000000029008E041F2FC30C2F200000290CE
:1033E00002E000200290FFE7029803B0704700005F
:1033F00080B582B00190019800680068C00600287E
:103400002AD5FFE7FFE700200090019800680068D8
:10341000009001980068406800900098FFE70198CC
:103420000CF0D6F800EBC00140F26850C2F2000088
:1034300000EB8100006A70B1FFE701980CF0C8F85A
:1034400000EBC00140F26850C2F2000000EB8100C6
:10345000006A8047FFE7FFE702B080BD82B08DF8C9
:1034600006008DF805100092009820B9FFE7FE20B5
:103470008DF8070020E09DF80600022805DCFFE734
:103480009DF80500092804DBFFE7FF208DF8070001
:1034900012E000989DF8061001EBC10240F268515D
:1034A000C2F2000101EB82019DF8052041F82200E3
:1034B00000208DF80700FFE79DF9070002B0704774
:1034C000FFE7FEE780B541F2CC00C2F2000002F057
:1034D000EFFF80BD80B541F2CC00C2F2000002F0E7
:1034E000E7FF80BD80B541F2F400C2F2000002F0B7
:1034F000DFFF80BD80B541F2F400C2F2000002F0AF
:10350000D7FF80BD82B00090009820B9FFE703206C
:103510008DF807001DE00098006846F20041C4F2F3
:103520000001884204D1FFE700208DF8070010E079
:103530000098006846F60001C4F20001884204D1F8
:10354000FFE701208DF8070003E003208DF8070056
:10355000FFE79DF8070002B0704700008AB00990AD
:1035600008910792069308980078E0B9FFE7089859
:10357000807C01460591032814D80599DFE801F005
:103580000E02060A0999012008710BE00999022030
:10359000087107E009990220087103E009990220E7
:1035A0000871FFE7A4E008980078022840F09F80A7
:1035B000FFE7089890F8240001460491032814D8E6
:1035C0000499DFE801F00E020A0609990220087149
:1035D0000BE009990420087107E00999052008719A
:1035E00003E0099902200871FFE7089890F8250088
:1035F0000146039103281CD80399DFE801F0140267
:103600000E080799002008740699487011E0079980
:1036100001200874069948700BE00799012008748E
:103620000699487005E007990020087406994870CB
:10363000FFE7089890F8280001460291032814D863
:103640000299DFE801F00E020A06079900200870CF
:103650000BE007990120087007E007990220087025
:1036600003E0079900200870FFE7089890F826000B
:1036700001460191032814D80199DFE801F00E02F8
:103680000A060699002008700BE0069901200870D0
:1036900007E006990320087003E0069900200870EF
:1036A000FFE7089890F827000146009103281DD8ED
:1036B0000099DFE801F015020F0806990020C87094
:1036C0000699887012E006990020C87006990120BA
:1036D00088700BE006990120C8700699887005E093
:1036E00006990020C87006998870FFE7FFE7FFE79A
:1036F00000200AB07047000082B00190009101994B
:1037000000200860019A022111710099087002B02E
:103710007047000080B584B0039002910192029836
:1037200000780146009148B1FFE70098013802286F
:103730001BD3FFE70098032828D02CE00298807C58
:1037400020B1FFE70298407C40B9FFE70398019958
:1037500000F024F803990020086005E0029803991E
:10376000019A00F025F8FFE715E0029890F827008D
:1037700028B9FFE70398019900F010F805E00298D6
:103780000399019A00F014F8FFE704E00398019907
:1037900000F004F8FFE704B080BD000082B00190A3
:1037A00000910199002008710099087002B07047DB
:1037B00083B002900191009202980078D0B9FFE79F
:1037C0000298D0F80900019988600298D0F80D009D
:1037D0000199C8600298D0F8010001990861029827
:1037E000D0F809000099C8600298D0F80D0000993F
:1037F0008860FFE702980078022821D1FFE702984D
:10380000C069019988600298006A0199C8600298AD
:10381000406901990861029840690199886102989C
:1038200080690199C8610298C06980F000400099E0
:10383000C8600298006A80F0004000998860FFE745
:1038400003B070470000000080B588B08DED070A16
:10385000CDED060A05909DED050AB8EE400A10EE82
:10386000100A14F0D1F941EC100B9FED2B1B53EC17
:10387000112B51EC100B13F025FE41EC100B51EC09
:10388000100B13F09BFA00EE100A12F059FB9FED9B
:10389000261A20EE010A10EE100A14F0B5F941ECD8
:1038A000100B51EC100B9FED1E0B52EC103BD20F86
:1038B00062F3DF7141EC100B8DED020B079814F0F1
:1038C000A3F99DED021B41EC100B51EC110B53ECD5
:1038D000102B13F0A5FA41EC100B51EC100B13F068
:1038E0006DFA04909DED040A9FED101AB4EE410AA2
:1038F000F1EE10FA05DDFFE79DED060A8DED010AF8
:1039000004E09DED040A8DED010AFFE79DED010A3B
:1039100008B080BD00BF00BFFCA9F1D24D62503F8E
:103920000000000000000000CDCC4C3ECDCC4C3F50
:1039300080B58EB00C900B910A920C9818B1FFE7ED
:103940000B9820B9FFE7FE208DF837009DE10A991A
:103950000C980268891A00EE101AB8EE400A9FED22
:10396000CD1A80EE010A80ED010A0A980C990860D0
:103970000C980B9909790A9A00F09AF920B1FFE79F
:10398000FD208DF8370080E10C98007A0146049103
:10399000052800F2BD800499DFE801F0030B030362
:1039A000992E0C990020C8600C9908610C99486107
:1039B000B2E00B9890ED020A90ED051A20EE010A94
:1039C0000C9880ED030A0B9890ED030A90ED051A10
:1039D00020EE010A0C9880ED040A0B9890ED040A81
:1039E00090ED051A20EE010A0C9880ED050A0B985F
:1039F00040690C9988618FE00C9890ED3F0A9FED2B
:103A0000A81A80EE010A9FEDA71A20EE010A00F520
:103A1000C66090ED001A30EE410A40F20460C2F236
:103A20000000019080ED000A90ED000A11F0C8FA44
:103A3000019840F64851C2F20001029181ED000A5E
:103A400090ED000A12F07CFA029841F64061C2F251
:103A5000000181ED000A90ED000A0B9A92ED061A22
:103A600092ED072A20EE010A91ED001A21EE021ACA
:103A700030EE410A0C9A82ED030A91ED000A0B998F
:103A800091ED061A91ED072A20EE010A90ED001A39
:103A900021EE021A30EE010A0C9880ED040A0C980F
:103AA00000F2246090ED000A8DED030A0A989FED64
:103AB0007E0ADFED7E0AFFF7C7FEB0EE401A9DEDED
:103AC000030A20EE010A0C9880ED050A24E00B9809
:103AD00090ED070AB1EE400A0C9880ED030A0B98AE
:103AE00090ED060AB1EE400A0C9880ED040A0C999C
:103AF00001F57770D1ED011AD1ED3F0A9FED660A0D
:103B00009FED661A08F046FC0C9880ED050A03E06C
:103B1000FD208DF83700B8E00C9901F2944091ED4A
:103B2000030A06F0A5FF0C9880ED030A0C9901F238
:103B3000B44091ED040A06F09BFF0C9880ED040A56
:103B40000C9901F2D44091ED050A06F091FF0C9812
:103B500080ED050A0C980B9900F04AF900200990B5
:103B6000FFE70998032800F38C80FFE70C98099978
:103B700000EB8101C86CC8650C99099AC2EB021070
:103B800001EB800000F5867001EB820292ED170ACE
:103B9000D2ED330AD1ED011A9FED401A8DED001AD6
:103BA00008F0F8FB9DED001A099805AB03EB8000C7
:103BB00080ED000A0C99099AC2EB021001EB80001B
:103BC00000F5FE7003EB820393ED000A01EB820225
:103BD000D2ED2F0AD1ED011A08F0DCFB0C980999FF
:103BE00000EB810080ED1F0A0C99099A01EB42104D
:103BF00000F2745001EB820191ED1F0A06F038FFCC
:103C00009DED001A0C98099900EB810000F21460F8
:103C100080ED000A0C98099900EB8101C86AC8661A
:103C20000C99099AC2EB021001EB800000F53B7081
:103C300001EB820292ED1B0AD2ED270AD1ED011AA7
:103C400008F0A8FB0C98099900EB810080ED230A8D
:103C50000C99099A01EB421000F2F44001EB820149
:103C600091ED230A06F004FF0C98099900EB8100FE
:103C700000F2046080ED000AFFE709980130099026
:103C80006FE700208DF83700FFE79DF937000EB091
:103C900080BD00BF00007A44DC68803D0000000069
:103CA00000003443DB0F49409A99193FCDCC4C3F7B
:103CB00080B586B004908DF80F100292049820B958
:103CC000FFE7FE208DF817004FE09DF80F000499E4
:103CD000097A884204D1FFE700208DF8170044E0FC
:103CE0009DF80F0005280ED1FFE70498007A0528FB
:103CF00009D0FFE70298FCF751FB04994FF07E5082
:103D0000C1F82406FFE700200190FFE7019803288F
:103D100023DCFFE704980199C1EB011100EB81005E
:103D200000F53B7008F07AFD04980199C1EB011190
:103D300000EB810000F5FE7008F070FD0498019919
:103D4000C1EB011100EB810000F5867008F066FD03
:103D5000FFE7019801300190D8E79DF80F00049922
:103D6000087200208DF81700FFE79DF9170006B0D4
:103D700080BD000080B582B0019000200090FFE778
:103D80000098032823DCFFE70199D1F87004009A1A
:103D900000EBC200803001EB820101F2046191ED81
:103DA000000A07F0C7FD0199D1F87004009A00EBF2
:103DB000C200A03001EB820101F2146191ED000A12
:103DC00007F0B8FDFFE7009801300090D8E70198B0
:103DD000D0F87004803007F073FB0198D0F87004BD
:103DE000A03007F06DFB02B080BD000000000000B5
:103DF00080B5ADF53E7DBD90BC91BD98007A01289F
:103E00007ED1FFE7BD98C06813F0FEFE41EC100BB9
:103E10009FED551B50EC111BC20F51EC100B62F3C0
:103E2000DF7141EC100B51EC100B9FED510B53EC7B
:103E3000102B13F029FF002862D1FFE7BD9800691D
:103E400013F0E2FE41EC100B9FED471B50EC111BF1
:103E5000C20F51EC100B62F3DF7141EC100B51EC0F
:103E6000100B9FED430B53EC102B13F00DFF0028AC
:103E700046D1FFE7BD98406913F0C6FE41EC100B38
:103E80009FED391B50EC111BC20F51EC100B62F36C
:103E9000DF7141EC100B51EC100B9FED350B53EC27
:103EA000102B13F0F1FE58BBFFE7BD9890F81804F3
:103EB00028B9FFE7BD99012081F81804FFE7002029
:103EC0008DF8EF02FFE79DF8EF02032816DCFFE70D
:103ED000BD989DF8EF1200EB8101D1F8F405C8639D
:103EE000BD989DF8EF1200EB81010020C861FFE74B
:103EF0009DF8EF0201308DF8EF02E4E700F0CCBD51
:103F0000BD99002081F818048DF8EE02FFE79DF8B6
:103F1000EE0203280FDCFFE7BD989DF8EE1200EBE0
:103F20008101C86BC1F8F405FFE79DF8EE0201308E
:103F30008DF8EE02EBE7BD98007A0146B4910028B7
:103F400000F08D85FFE7B498012819D0FFE7B498F9
:103F500002380228C0F08385FFE7B49804380128AE
:103F600000F299850CE000BF000000000000000096
:103F70009A9999999999B93F000000000000F03F83
:103F8000BD980090C06813F03FFE02460098019271
:103F90000A46019942EC101B8DED040B406913F0A9
:103FA00033FE41EC100B8DED020B1FED0D0B8DED73
:103FB000AA0B10F0DDFB11F05FFF9DED021B51EC31
:103FC000110B53EC102B13F07DFA9DED040B41EC1B
:103FD000110B53EC112B51EC100B12F021FF41ECA3
:103FE000100B8DED0C0BBD99C8684969069113F053
:103FF0000BFE0246069807920A46079942EC101BF0
:104000008DED0A0B13F000FE9DEDAA0B41EC110B98
:104010008DED081B10F0ACFB11F02EFF9DED081B81
:1040200051EC110B53EC102B13F04CFA9DED0A0BD5
:1040300041EC110B53EC112B51EC100B12F0F0FE74
:104040009DED0C1B41EC100B51EC110B53EC102BA4
:1040500013F038FA41EC100B8DED1C0BBD9908697B
:1040600049690E9113F0D0FD02460E980F920A4650
:104070000F9942EC101B8DED120B13F0C5FD9DED59
:10408000AA0B41EC110B8DED101B10F071FB10F021
:1040900033FF9DED101B51EC110B53EC102B13F063
:1040A00011FA9DED120B41EC110B53EC112B51EC5D
:1040B000100B12F0B5FE41EC100B8DED1A0BBD99F3
:1040C00008694969149113F09FFD024614981592EE
:1040D0000A46159942EC101B8DED180B13F094FD58
:1040E0009DEDAA0B41EC110B8DED161B10F040FB62
:1040F00010F002FF9DED161B51EC110B53EC102B31
:1041000013F0E0F99DED180B41EC110B53EC112B62
:1041100051EC100B12F084FE9DED1A1B41EC100BBC
:1041200051EC110B53EC102B13F0CCF99DED1C1B33
:1041300041EC100B51EC110B53EC102B12F070FEF4
:1041400041EC100B11F0C4FF51EC100B12F036FED5
:10415000BD99C861BD99C86849691E9113F054FDA5
:1041600002461E981F920A461F9942EC101B8DEDC5
:10417000220B13F049FD9DEDAA0B41EC110B8DEDC7
:10418000201B10F0F5FA11F077FE9DED201B51EC8D
:10419000110B53EC102B13F095F99DED220B41EC14
:1041A000110B53EC112B51EC100B12F039FE41ECBA
:1041B000100B8DED2A0BBD99C8684969249113F045
:1041C00023FD0246249825920A46259942EC101BAD
:1041D0008DED280B13F018FD9DEDAA0B41EC110B92
:1041E0008DED261B10F0C4FA11F046FE9DED261B46
:1041F00051EC110B53EC102B13F064F99DED280BCF
:1042000041EC110B53EC112B51EC100B12F008FE8A
:104210009DED2A1B41EC100B51EC110B53EC102BB4
:1042200013F050F941EC100B8DED3A0BBD99086974
:1042300049692C9113F0E8FC02462C982D920A460D
:104240002D9942EC101B8DED300B13F0DDFC9DED34
:10425000AA0B41EC110B8DED2E1B10F089FA10F01A
:104260004BFE9DED2E1B51EC110B53EC102B13F05C
:1042700029F99DED300B41EC110B53EC112B51EC56
:10428000100B13F0D3FB41EC100B8DED380BBD99E7
:1042900008694969329113F0B7FC024632983392AB
:1042A0000A46339942EC101B8DED360B13F0ACFC33
:1042B0009DEDAA0B41EC110B8DED341B10F058FA5B
:1042C00010F01AFE9DED341B51EC110B53EC102B2A
:1042D00013F0F8F89DED360B41EC110B53EC112B5C
:1042E00051EC100B13F0A2FB9DED381B41EC100BB1
:1042F00051EC110B53EC102B13F0E4F89DED3A1B2D
:1043000041EC100B51EC110B53EC102B12F088FD0B
:1043100041EC100B11F0DCFE51EC100B12F04EFDD5
:10432000BD990862BD99C86849693C9113F06CFC5D
:1043300002463C983D920A463D9942EC101B8DED99
:10434000400B13F061FC9DEDAA0B41EC110B8DEDC0
:104350003E1B10F00DFA11F08FFD9DED3E1B51EC50
:10436000110B53EC102B13F0ADF89DED400B41EC0D
:10437000110B53EC112B51EC100B13F057FB41ECCC
:10438000100B8DED480BBD99C8684969429113F037
:104390003BFC0246429843920A46439942EC101B6A
:1043A0008DED460B13F030FC9DEDAA0B41EC110B8B
:1043B0008DED441B10F0DCF911F05EFD9DED441B0A
:1043C00051EC110B53EC102B13F07CF89DED460BC8
:1043D00041EC110B53EC112B51EC100B13F026FB9D
:1043E0009DED481B41EC100B51EC110B53EC102BC5
:1043F00013F068F841EC100B8DED580BBD9908696E
:1044000049694A9113F000FC02464A984B920A46C9
:104410004B9942EC101B8DED4E0B13F0F5FB9DED0F
:10442000AA0B41EC110B8DED4C1B10F0A1F910F013
:1044300063FD9DED4C1B51EC110B53EC102B13F055
:1044400041F89DED4E0B41EC110B53EC112B51EC4F
:10445000100B13F0EBFA41EC100B8DED560BBD99E0
:1044600008694969509113F0CFFB02465098519268
:104470000A46519942EC101B8DED540B13F0C4FB0E
:104480009DEDAA0B41EC110B8DED521B10F070F954
:1044900010F032FD9DED521B51EC110B53EC102B23
:1044A00013F010F89DED540B41EC110B53EC112B54
:1044B00051EC100B13F0BAFA9DED561B41EC100BAA
:1044C00051EC110B53EC102B12F0FCFF9DED581B1F
:1044D00041EC100B51EC110B53EC102B12F0A0FC23
:1044E00041EC100B11F0F4FD51EC100B12F066FCD6
:1044F000BD994862BD99C86849695A9113F084FB17
:1045000002465A985B920A465B9942EC101B8DED6D
:104510005E0B13F079FB9DEDAA0B41EC110B8DEDB9
:104520005C1B10F025F911F0A7FC9DED5C1B51EC14
:10453000110B53EC102B12F0C5FF9DED5E0B41ECFF
:10454000110B53EC112B51EC100B13F06FFA41ECE3
:10455000100B8DED660BBD99C8684969609113F029
:1045600053FB0246609861920A46619942EC101B27
:104570008DED640B13F048FB9DEDAA0B41EC110B84
:104580008DED621B10F0F4F811F076FC9DED621BCE
:1045900051EC110B53EC102B12F094FF9DED640BBA
:1045A00041EC110B53EC112B51EC100B13F03EFAB4
:1045B0009DED661B41EC100B51EC110B53EC102BD5
:1045C00012F080FF41EC100B8DED760BBD99086960
:1045D0004969689113F018FB0246689869920A4687
:1045E000699942EC101B8DED6C0B13F00DFB9DEDEA
:1045F000AA0B41EC110B8DED6A1B10F0B9F810F00D
:104600007BFC9DED6A1B51EC110B53EC102B12F04F
:1046100059FF9DED6C0B41EC110B53EC112B51EC40
:10462000100B12F0FDFB41EC100B8DED740BBD99DE
:10463000086949696E9113F0E7FA02466E986F9225
:104640000A466F9942EC101B8DED720B13F0DCFAE9
:104650009DEDAA0B41EC110B8DED701B10F088F84D
:1046600010F04AFC9DED701B51EC110B53EC102B1C
:1046700012F028FF9DED720B41EC110B53EC112B46
:1046800051EC100B12F0CCFB9DED741B41EC100BA8
:1046900051EC110B53EC102B12F014FF9DED761B17
:1046A00041EC100B51EC110B53EC102B12F0B8FB3A
:1046B00041EC100B11F00CFD51EC100B12F07EFBD5
:1046C000BD998862BD9908694969789113F09CFA8F
:1046D0000246789879920A46799942EC101B8DED42
:1046E0007C0B13F091FA9DEDAA0B41EC110B8DEDB3
:1046F0007A1B10F03DF810F0FFFB9DED7A1B51EC9A
:10470000110B53EC102B12F0DDFE9DED7C0B41ECF8
:10471000110B53EC112B51EC100B12F081FB41ECFF
:10472000100B8DED840BBD99C86849697E9113F01B
:104730006BFA02467E987F920A467F9942EC101BE4
:104740008DED820B13F060FA9DEDAA0B41EC110B7D
:104750008DED801B10F00CF811F08EFB9DED801B91
:1047600051EC110B53EC102B12F0ACFE9DED820BB3
:1047700041EC110B53EC112B51EC100B12F050FBD0
:104780009DED840B41EC110B10F05EF951EC100B18
:104790009FEDED0B53EC102BB393B29212F092FEFF
:1047A00041EC100B51EC100B12F008FBBD99C863E3
:1047B000BD9908694969869113F026FA02468698E0
:1047C00087920A46879942EC101B8DED8A0B13F0F5
:1047D0001BFA9DEDAA0B41EC110B8DED881B0FF020
:1047E000C7FF10F089FB9DED881B51EC110B53ECBA
:1047F000102B12F067FE9DED8A0B41EC110B53EC70
:10480000112B51EC100B13F011F941EC100B8DED45
:10481000920BBD99C86849698C9113F0F5F902466D
:104820008C988D920A468D9942EC101B8DED900B61
:1048300013F0EAF99DEDAA0B41EC110B8DED8E1BE7
:104840000FF096FF11F018FB9DED8E1B51EC110B34
:1048500053EC102B12F036FE9DED900B41EC110B3A
:1048600053EC112B51EC100B12F0DAFA9DED920B78
:1048700041EC110B10F0E8F8B29AB39B51EC100B1D
:1048800012F020FE41EC100B51EC100B12F096FAD6
:10489000BD990864BD9908694969949113F0B4F908
:1048A0000246949895920A46959942EC101B8DED1C
:1048B000980B13F0A9F99DEDAA0B41EC110B8DEDAE
:1048C000961B0FF055FF10F017FB9DED961B51EC5A
:1048D000110B53EC102B12F0F5FD9DED980B41ECF4
:1048E000110B53EC112B51EC100B13F09FF841EC12
:1048F000100B8DEDA00BBD99C86849699A9113F012
:1049000083F902469A989B920A469B9942EC101BA7
:104910008DED9E0B13F078F99DEDAA0B41EC110B78
:104920008DED9C1B0FF024FF11F0A6FA9DED9C1B52
:1049300051EC110B53EC102B12F0C4FD9DED9E0BAE
:1049400041EC110B53EC112B51EC100B13F06EF8E2
:104950009DEDA00B41EC110B10F076F8B29AB39BD1
:1049600051EC100B12F0AEFD41EC100B51EC100BA2
:1049700012F024FABD994864BD9908694969A29169
:1049800013F042F90246A298A3920A46A39942EC78
:10499000101B8DEDA60B13F037F99DEDAA0B41EC22
:1049A000110B8DEDA41B0FF0E3FE10F0A5FA9DEDA9
:1049B000A41B51EC110B53EC102B12F083FD9DED59
:1049C000A60B41EC110B53EC112B51EC100B12F018
:1049D00027FA41EC100B8DEDB00BBD99C868496901
:1049E000A89113F011F90246A898A9920A46A9992C
:1049F00042EC101B8DEDAE0B13F006F99DEDAA0BEA
:104A000041EC110B8DEDAC1B0FF0B2FE11F034FA3E
:104A10009DEDAC1B51EC110B53EC102B12F052FD21
:104A20009DEDAE0B41EC110B53EC112B51EC100B27
:104A300012F0FCFF9DEDB00B41EC110B10F004F8EF
:104A4000B29AB39B51EC100B12F03CFD41EC100BF1
:104A500051EC100B12F0B2F9BD9988641BE00020F4
:104A6000BA90FFE7BA9803280BDCFFE7BD98BA9924
:104A700000EB81010020C861FFE7BA980130BA90CD
:104A8000F0E7BD990020C863BD990864BD994864EA
:104A9000BD998864FFE7FFE700208DF8E702FFE794
:104AA0009DF8E702032822DCFFE7BD989DF8E71296
:104AB00000EB810090ED0F0AB5EE400AF1EE10FA1E
:104AC0000EDAFFE7BD989DF8E71200EB810090ED4C
:104AD0000F0A9FED871A30EE010A80ED0F0AFFE7FB
:104AE000FFE79DF8E70201308DF8E702D8E70020E4
:104AF0008DF8E602FFE79DF8E602032800F3EC805C
:104B0000FFE7BD989DF8E61200EB810090ED0F0ADB
:104B100090ED331A30EE410AB5A800EB810080ED2C
:104B2000000AFFE79DF8E612B5A800EB810090EDC2
:104B3000000A9FED6B1AB4EE410AF1EE10FA15DD92
:104B400006E000BF00BF00BF00000000DCA54C4035
:104B50009DF8E612B5A800EB810090ED000A9FEDEC
:104B6000651A30EE010A80ED000ADBE7FFE79DF8E9
:104B7000E612B5A800EB810090ED000A9FED591AEE
:104B8000B4EE410AF1EE10FA0EDAFFE79DF8E612F4
:104B9000B5A800EB810090ED000A9FED551A30EEAC
:104BA000010A80ED000AE2E79DF8E612B5A800EBE5
:104BB000810090ED000A9FED4C1AB4EE410AF1EE2F
:104BC00010FA2BDDFFE79DF8E612B5A800EB810097
:104BD00090ED000A9FED421AB4EE410AF1EE10FA90
:104BE0001CDCFFE7BD989DF8E61200EB8101C86967
:104BF000C862BD989DF8E62200EB820090ED330A72
:104C0000B5A901EB820191ED001A30EE010A9FED8A
:104C1000351A30EE010A80ED130A56E09DF8E612CF
:104C2000B5A800EB810090ED000A9FED301AB4EEBC
:104C3000410AF1EE10FA2BDAFFE79DF8E612B5A86B
:104C400000EB810090ED000A9FED261AB4EE410AB8
:104C5000F1EE10FA1CDBFFE7BD989DF8E61200EBC1
:104C60008101C869C862BD989DF8E62200EB820008
:104C700090ED330AB5A901EB820191ED001A30EEF7
:104C8000010A9FED171A30EE010A80ED130A1BE0AE
:104C9000BD989DF8E61200EB810090ED070AB1EE99
:104CA000400A80ED0B0ABD989DF8E62200EB8200D9
:104CB00090ED330AB5A901EB820191ED001A30EEB7
:104CC000010A80ED130AFFE7FFE7FFE79DF8E60220
:104CD00001308DF8E6020EE70DF53E7D80BD00BF88
:104CE00000003443000034C30000B4420000B4C2EA
:104CF0000000B4430000B4C380B584B002900298B1
:104D000020B9FFE7FE208DF80F0091E006F022FFAA
:104D100000200190FFE70198032800F38580FFE75A
:104D20000298D0F87004019900EBC100A03006F0A1
:104D300001FD183006F054FB9FED411A80EE010A88
:104D40009FED401A20EE010A0298019900EB8100C4
:104D500080ED330A0298D0F87004019900EBC1008D
:104D6000A03006F0E7FC183006F04CFB9FED361A39
:104D700080EE010A0298019900EB810080ED2F0A74
:104D80000298D0F87004019900EBC100803006F061
:104D9000D1FC183006F036FB9FED2C1A80EE010A8C
:104DA0000298019900EB810080ED270A0298019991
:104DB00000EB810090ED330A00F58C6090ED001A55
:104DC00030EE410A10EE100A12F01EFF41EC100BFB
:104DD0009FED191B10F09CF951EC100B11F0EEFF38
:104DE0000299019A01EB8201C1F8CC000298019965
:104DF00000EB810090ED330AB5EE400AF1EE10FAB7
:104E00000DDAFFE70298019900EB810090ED330A7B
:104E10009FED0F1A30EE010A80ED330AFFE7FFE73E
:104E200001980130019076E700208DF80F00FFE730
:104E30009DF90F0004B080BD0000000000807640A6
:104E4000DB0F4940000034430000A04300401C46F3
:104E50000000B44384B003908DED020ACDED010A49
:104E6000039890ED000A9DED021A30EE010A8DEDD7
:104E7000000A9DED010AB5EE400AF1EE10FA26DDBA
:104E8000FFE79DED000A9DED011AB4EE410AF1EE37
:104E900010FA09DBFFE79DED011A9DED000A30EEE7
:104EA000410A8DED000A11E09DED000AB5EE400AC1
:104EB000F1EE10FA09DAFFE79DED011A9DED000A07
:104EC00030EE010A8DED000AFFE7FFE7FFE70098EB
:104ED0000399086004B0704785B08DED040ACDEDEC
:104EE000030A8DED021A9DED040A9DED031A30EEC2
:104EF000410A8DED010A9DED020AB5EE400AF1EE80
:104F000010FA32DDFFE79DED020AB0EE001A80EEE6
:104F1000010A8DED000A9DED010A9DED001AB4EE27
:104F2000410AF1EE10FA09DDFFE79DED021A9DED51
:104F3000010A30EE410A8DED010A15E09DED010AEE
:104F40009DED001AB1EE411AB4EE410AF1EE10FAED
:104F500009DAFFE79DED021A9DED010A30EE010A24
:104F60008DED010AFFE7FFE7FFE79DED010A05B0C0
:104F70007047000040F21400C2F2000070470000C9
:104F800080B541F23C20C2F2000002F00DF980BD74
:104F900080B541F29C20C2F2000002F005F980BD0C
:104FA00080B541F21C10C2F2000002F0FDF880BD95
:104FB00080B541F27C10C2F2000002F0F5F880BD2D
:104FC00080B541F2DC10C2F2000002F0EDF880BDC5
:104FD00080B541F2FC20C2F2000002F0E5F880BD8D
:104FE00082B001900198007810384AF6AB21CAF6D9
:104FF000AA21A0FB011000090090009948F240107E
:10500000C0F60100405C0199C8650098042807D3E8
:10501000FFE701990868042262F30900886506E049
:105020000199086840F2FF3290438865FFE70198D4
:10503000806D02B07047000086B0059000208DF8AA
:1050400013000598806A03900598806910BBFFE7FC
:105050000398029003281BD80299DFE801F0020DA3
:105060000218059890F82F00C00720B1FFE7012033
:105070008DF81300FFE70CE00598C06AB0F1C07F1F
:1050800004D1FFE701208DF81300FFE701E000E005
:10509000FFE745E005988069B0F5005F25D1FFE79F
:1050A0000398019003281ED80199DFE801F0020659
:1050B000021101208DF8130016E0059890F82F00DA
:1050C000C00720B1FFE701208DF81300FFE70BE0D8
:1050D0000598C06AB0F1C07F04D1FFE701208DF8C8
:1050E0001300FFE700E0FFE719E0039800900328B2
:1050F00004D3FFE70098032804D00EE001208DF8C8
:1051000013000BE0059890F82F00C00720B1FFE7CF
:1051100001208DF81300FFE700E0FFE7FFE7FFE75E
:105120009DF8130006B0704784B00390029101927D
:10513000009303980168086820F4802008600098B4
:1051400003990968486003988068402809D1FFE7FF
:105150000198039909688860029803990968C860F2
:1051600008E0029803990968886001980399096822
:10517000C860FFE704B0704783B0019000910198C8
:1051800020B9FFE7FE208DF80B0018E0009820B949
:10519000FFE7FE208DF80B0011E000990320087056
:1051A00000990020A1F81100C1F80D00C1F8090014
:1051B000C1F80500C1F801008DF80B00FFE79DF96B
:1051C0000B0003B0704700007047000085B00390EB
:1051D0000291039820B9FFE7FE208DF8130020E02C
:1051E000029820B9FFE7FE208DF8130019E002991C
:1051F000032008700299009100200190C1F82F004F
:10520000C1F82B00C1F82700C1F82300C1F81F0026
:10521000C1F81B00C1F81700C1F813008DF8130086
:10522000FFE79DF9130005B0704700000000000083
:1052300080B586B0059040F26461C2F20001009131
:1052400048788A7840EA02206FF3DF2000EE100AE7
:10525000B8EEC00A059880ED000A8878CA78C008C0
:1052600040EA42106FF3DF2000EE100AB8EEC00AE9
:10527000059880ED030AC8780B794A79800940EADD
:10528000830040EA82206FF3DF2000EE100AB8EEC0
:10529000C00A059880ED010A48798A79400840EAF9
:1052A000C2106FF3DF2000EE100AB8EEC00A0598B6
:1052B00080ED020A8879CA79000940EA02106FF38A
:1052C000DF20059A9083C8790B7A4A7AC00940EAB0
:1052D000430040EA42206FF3DF20059A1082487AAB
:1052E0008A7A800840EA82106FF3DF20059A5083A3
:1052F000887ACA7A400940EAC200059A1083087B7E
:105300004A7B40EA02206FF3DF20059AD082487B77
:105310008A7BC00840EA42106FF3DF20059A908232
:10532000887BCB7B0A7C800940EA830040EA8220AC
:105330006FF3DF20059A5082087C497C400840EAE0
:10534000C1106FF3DF200599C883059890ED010A1D
:10535000DFED6F0ACDED010A9FED6E1A8DED021A99
:10536000FFEE001ACDED031AB7EE002A8DED042AE8
:105370000AF0D4FEDDED010A9DED021ADDED031AFF
:105380009DED042A059880ED010A059890ED000A2C
:105390000AF0C4FEDDED010A9DED021ADDED031AEF
:1053A0009DED042A059880ED000A059890ED020A0B
:1053B0000AF0B4FEDDED010A9DED021ADDED031ADF
:1053C0009DED042A059880ED020A059890ED030AE8
:1053D0000AF0A4FE059880ED030A0598006812F013
:1053E00013FC41EC100B9FED461B53EC112B51ECC1
:1053F000100B12F050FCA0B9FFE70598006812F0FE
:1054000003FC41EC100B9FED401B53EC112B51ECB6
:10541000100B12F032FC20B9FFE70599002008605C
:10542000FFE70598406812F0EFFB41EC100B9FED91
:10543000341B53EC112B51EC100B12F02CFCA0B9C7
:10544000FFE70598406812F0DFFB41EC100B9FED81
:105450002E1B53EC112B51EC100B12F00EFC20B94B
:10546000FFE7059900204860FFE70598806812F083
:10547000CBFB41EC100B9FED221B53EC112B51EC9D
:10548000100B12F008FCA0B9FFE70598806812F035
:10549000BBFB41EC100B9FED1C1B53EC112B51EC93
:1054A000100B12F0EAFB20B9FFE705990020886095
:1054B000FFE70598C06812F0A7FB41EC100B9FEDC9
:1054C000101B53EC112B51EC100B12F0E4FBA0B9A4
:1054D000FFE70598C06812F097FB41EC100B9FEDB9
:1054E0000A1B53EC112B51EC100B12F0C6FB20B928
:1054F000FFE705990020C860FFE7012006B080BDE6
:105500007B14AE47E17A84BF7B14AE47E17A843FD7
:105510000080B04300E0D34480B5012002F044F99C
:1055200080BD000080B5102002F03EF980BD000073
:1055300080B5202002F038F980BD000072B6FFE788
:10554000FEE7000080B594B012901191129818B146
:10555000FFE7119820B9FFE7FF208DF84F0045E2E3
:10556000FDF7C6FE129A089213685268C01A91415C
:1055700012F09FFB0146089800EE101A9FEDC01A2A
:1055800080EE010A80ED020AFDF7B2FE0A4612998A
:105590004A60086012981199097800F033FB11985D
:1055A00090ED030AB2EE041A20EE010A129890ED73
:1055B000021A20EE010A8DED100A1298C06890EDD3
:1055C0003B0AB5EE400AF1EE10FA40F38980FFE79E
:1055D000129890EDA11A90EDB00A30EE410A41F216
:1055E0003C50C2F2000080ED000A90ED000A9FEDF1
:1055F000A51AB4EE410AF1EE10FA0DDDFFE741F213
:105600003C50C2F2000090ED000A9FED9F1A30EE70
:10561000010A80ED000AFFE741F23C50C2F20000AF
:1056200090ED000A9FED991AB4EE410AF1EE10FADE
:105630000DDAFFE741F23C50C2F2000090ED000AA3
:105640009FED931A30EE010A80ED000AFFE71298F1
:1056500090ED051A90ED650A41F23C50C2F200004F
:10566000069090ED002A31EE021A9DED102A71EE9F
:10567000020A9FEDE31A8DED071AFFF72DFC06983D
:105680009DED071A8DED0F0A129991ED052A91ED06
:10569000660A90ED003A32EE032A9DED103A72EE62
:1056A000030AFFF719FC8DED0E0A9DED100A9DED22
:1056B0000F1AB4EE410AF1EE10FA03DDFFE70F987E
:1056C0001090FFE79DED100A9DED0E1AB4EE410A11
:1056D000F1EE10FA03DAFFE70E981090FFE7FFE70C
:1056E000129814309DED100ADFEDC50AFFF7B2FBEA
:1056F0001298C06890ED380A90ED3B1AB6EE002A79
:1057000021EE021A30EE010A8DED0D0A0D98129964
:105710000862119890ED020AB2EE001A20EE010A1A
:10572000129890ED021A20EE010A8DED0C0A1298E3
:10573000C06890ED3D0AB5EE400AF1EE10FA72DD58
:10574000FFE7129890EDA31A90EDAC0A30EE410AF3
:105750008DED0B0A9DED0B0A9FEDA61AB4EE410AE2
:10576000F1EE10FA09DDFFE79DED0B0A9FEDA21A9D
:1057700030EE010A8DED0B0AFFE79DED0B0A9FED60
:105780009F1AB4EE410AF1EE10FA09DAFFE79DED37
:105790000B0A9FED9B1A30EE010A8DED0B0AFFE715
:1057A000129890ED061A90ED690A9DED0B2A31EEE4
:1057B000021A9DED0C2A71EE020A9FED911A8DEDF1
:1057C000051AFFF789FB9DED051A8DED0A0A12985F
:1057D00090ED062A90ED6A0A9DED0B3A32EE032A0F
:1057E0009DED0C3A72EE030AFFF776FB8DED090A88
:1057F0009DED0C0A9DED0A1AB4EE410AF1EE10FA85
:1058000003DDFFE70A980C90FFE79DED0C0A9DED84
:10581000091AB4EE410AF1EE10FA03DAFFE709982B
:105820000C90FFE7FFE7129818309DED0C0ADFEDB2
:10583000740AFFF70FFB1298007C0146049148B1EF
:10584000FFE70498012810D0FFE70498022800F031
:10585000BE80C7E012990020C1F870021299C1F809
:1058600074021299C1F86C02BCE01198007C08B96E
:10587000FFE719E01198007C012814D10AE000BF6D
:1058800000247449DB0F4940DB0FC9C0DB0F49C05E
:10589000DB0FC940119840691299486111988069DD
:1058A00012998861FFE7FFE7129901F12C00D1ED11
:1058B000021A91ED050AD1EDA10A9FED521A8DED64
:1058C000011A06F067FD9DED011A42F61872C2F248
:1058D000010282ED000A129901F1680092ED000ABE
:1058E000D1ED021AD1EDA00A06F054FD129880ED18
:1058F0009B0A129901F1A400D1ED021A91ED080A58
:10590000D1EDB00A91EDB11A06F044FD9DED011AFA
:1059100042F61C72C2F2010282ED000A129901F1F4
:10592000E00092ED000AD1ED021AD1EDA90A06F0CD
:1059300031FD129880ED9C0A129901F58E70D1ED1F
:10594000021A91ED060A91ED9F1AD1EDA30AB1EE6C
:10595000411A06F01FFD9DED011A41F24052C2F2BC
:10596000000282ED000A129901F5AC7092ED000A76
:10597000B2EE002A20EE020AD1ED021A91ED9F2A22
:10598000F1EE420A06F006FD10EE100A12F03CF9A4
:1059900041EC100B8DED020B1298D0F8B00212F012
:1059A00033F941EC100B0BF063F99DED021B51EC48
:1059B000110B53EC102B11F033FA41EC100B51EC9E
:1059C000100B11F0FBF91299C1F874020AE0129958
:1059D0000020C1F870021299C1F874021299C1F83E
:1059E0006C02FFE700208DF84F00FFE79DF94F00A4
:1059F00014B080BDDB0F4940DB0FC9C0DB0F49C0CD
:105A0000DB0FC9400000000080B586B00490039110
:105A10008DED020A049818B1FFE7039820B9FFE75B
:105A2000FF208DF81700AAE003980499C860049835
:105A3000002101910174049A02F12C009DED020AEB
:105A4000D268383206F01EFE049901F168009DED1F
:105A5000020AC96801F118020121009106F012FE44
:105A6000049901F1A4009DED020AC96801F17802D0
:105A7000022106F007FE0099049A02F1E0009DED74
:105A8000020AD268583206F0FDFD0199049A02F527
:105A90008E709DED020AD268B83206F0F3FD0099CF
:105AA000049A02F5AC709DED020AD268983206F0B5
:105AB000E9FD049901F5D6709DED020AC968D1EDA2
:105AC000360A05F031F8049901F503709DED020ADC
:105AD000C968D1ED370A05F027F8049901F50B7074
:105AE0009DED020AC968D1ED370A05F01DF8049949
:105AF00001F513709DED020AC968D1ED370A05F072
:105B000013F80498C16891ED380A91ED3B1A30EE14
:105B1000010A80ED650A0499C868D0F8E000C1F870
:105B200098010498C16891ED3A0A91ED3D1A30EE62
:105B3000010A80ED690A0499C868D0F8E800C1F844
:105B4000A801FCF7D9FC0498C068083005F08AFA6F
:105B50000498C068103005F085FA0498C06805F014
:105B60004DFE0498C068083005F012F90498C0682A
:105B7000103005F00DF901988DF81700FFE79DF939
:105B8000170006B080BD000080B58CB00B900B995B
:105B9000C86891ED9B0A05F0CDFE00200A9009909F
:105BA0000890079006900B9991ED9C0AB0EE041AAC
:105BB00020EE010A8DED060A4CF6CD41C3F6CC511C
:105BC0000A91059004900390029001900B98D0F8F0
:105BD000740201904CF6CD40C3F64C6005900B98D2
:105BE000C06805F06DFC0B98C068083006A905F088
:105BF00069F90B98C068103001A905F063F90CB081
:105C000080BD000080B584B002908DF80710029826
:105C100020B9FFE7FF208DF80F005AE09DF807003C
:105C20000299097C884204D1FFE700208DF80F001B
:105C30004FE00298A43006F0F1FD0298E03006F043
:105C4000EDFD029800F58E7006F0E8FD029800F573
:105C5000AC7006F0E3FD02982C3006F0DFFD0298F0
:105C6000683006F0DBFD029800F5E6709FED1B0A38
:105C70008DED000A04F0F6FF9DED000A029800F594
:105C8000F67004F0EFFF9DED000A029800F5D67063
:105C900004F0E8FF0298C068083005F079F802982F
:105CA000C068103005F074F8029800F52170FAF71A
:105CB00075FE0299D1F88C0288610299D1F88402AC
:105CC00048619DF807000299087400208DF80F00C4
:105CD000FFE79DF90F0004B080BD00BF0000000089
:105CE00080B584B00290029820B9FFE7FE208DF8BD
:105CF0000F005BE005F02EFF0298C06805F0A8FEDB
:105D00000298C06805F016FD183005F069FB02988E
:105D100080EDB00A0298C06805F00CFD183005F05F
:105D200071FBB2EE041A80EE010A029880EDB10A0E
:105D30000298C068083005F0CDFA0298C0680830B3
:105D400005F07CF80190019878B1FFE701980830E0
:105D500005F046FB029880EDA80A0198083005F08E
:105D600051FB029880EDA90AFFE70298C068103045
:105D700005F0B0FA0298C068103005F05FF80090A6
:105D8000009878B1FFE70098083005F029FB0298E9
:105D900080EDAC0A0098083005F034FB029880EDE5
:105DA000AD0AFFE700208DF80F00FFE79DF90F0017
:105DB00004B080BD83B001900091019820B9FFE745
:105DC000FF208DF80B0034E00199009B18685A6899
:105DD0009B68C1F88032C1F87C22C1F87802019931
:105DE000009BD8681A695B69C1F88C32C1F88822B7
:105DF000C1F88402009890ED050AB1EE400A0198BE
:105E000080EDA20A0199DDF800C0DCF81800DCF88A
:105E10001C20DCF82030DCF824C0C1F89CC2C1F89A
:105E20009832C1F89422C1F8900200208DF80B003E
:105E3000FFE79DF90B0003B07047000084B00290AB
:105E40000191029890F820008DF803009DF803005E
:105E5000012805D0FFE79DF8030002280AD1FFE7DB
:105E6000019A0298016848691043486100208DF842
:105E70000F0008E00299486A40F48020486201203F
:105E80008DF80F00FFE79DF80F0004B07047000089
:105E900088B00690059104920393069890F820002C
:105EA0008DF8070006980068806800900598806863
:105EB00008B9FFE700E0FFE79DF80700012806D0DA
:105EC000FFE79DF80700022840F08080FFE79DF87B
:105ED0000300400700280CD4FFE79DF803000007EB
:105EE000002806D4FFE79DF80300C006002864D50B
:105EF000FFE70098C0F301600290029901208840FA
:105F0000039908600598806868B9FFE705980168FB
:105F1000C06840EA415006990968029A01EB0211F3
:105F2000C1F880010EE005994A688868C96840EAAE
:105F3000C200084306990968029A01EB0211C1F8F0
:105F40008001FFE70598006906990968029A01EB4C
:105F50000211C1F884010598007D01280CD1FFE7EA
:105F600006980068029900EB0111D1F8840140F411
:105F70008070C1F88401FFE70498406806990968B9
:105F8000029A01EB0211C1F88C010498006806998D
:105F90000968029A01EB0211C1F8880106980068AD
:105FA000029900EB0111D1F8800140F00100C1F825
:105FB000800100208DF81F0011E00699486A40F426
:105FC0000010486201208DF81F0008E00699486A19
:105FD00040F48020486201208DF81F00FFE79DF803
:105FE0001F0008B07047000086B004900391049829
:105FF00090F820008DF803009DF80300012806D0DA
:10600000FFE79DF80300022840F0B080FFE746F26A
:106010000040C4F2000001900199D1F8000240F064
:106020000100C1F800020199D1F8000220F47C506F
:10603000C1F800020398426A0199D1F8000240EACF
:106040000220C1F800020398406900F01F010120FE
:1060500088400290029A0199D1F81C029043C1F83D
:106060001C020398C069F0B9FFE7029A0199D1F8C0
:106070000C029043C1F80C02039A9088D1685269CF
:1060800040EA0140019901EBC201C1F84002039AC4
:1060900010889168526940EA0140019901EBC20100
:1060A000C1F84402FFE70398C06901281ED1FFE749
:1060B000029A0199D1F80C021043C1F80C02039A1C
:1060C00090881168526940EA0140019901EBC201D0
:1060D000C1F84002039A90899168526940EA0140F0
:1060E000019901EBC201C1F84402FFE703988069FE
:1060F00040B9FFE7029A0199D1F804029043C1F830
:10610000040207E0029A0199D1F804021043C1F891
:106110000402FFE70398006940B9FFE7029A01997A
:10612000D1F814029043C1F8140207E0029A0199D1
:10613000D1F814021043C1F81402FFE70398006A73
:10614000012808D1FFE7029A0199D1F81C021043F7
:10615000C1F81C02FFE70199D1F8000220F001000C
:10616000C1F8000200208DF8170008E00499486A81
:1061700040F48020486201208DF81700FFE79DF869
:10618000170006B07047000080B582B001900198FA
:10619000FDF7B8F98DF803009DF80300032819D026
:1061A000FFE79DF8030040F29442C2F2000234215E
:1061B00010FB0120006B60B1FFE79DF8030040F287
:1061C0009442C2F20002342110FB0120006B804790
:1061D000FFE7FFE702B080BD84B00390029100208A
:1061E0000190039890F820008DF803009DF80300BB
:1061F000012805D0FFE79DF80300022812D1FFE730
:10620000029838B9FFE703980068C06800F00300FF
:10621000019006E003980068006900F00300019017
:10622000FFE7FFE7019804B07047000086B00490D4
:10623000039102920193049890F820008DF80300D6
:106240009DF80300012806D0FFE79DF8030002280F
:1062500040F0E880FFE7039880B9FFE70498006802
:10626000C068800748B9FFE70499486A40F4001005
:10627000486201208DF81700DDE00FE00498006807
:106280000069800748B9FFE70499486A40F40010A4
:10629000486201208DF81700CDE0FFE70498006800
:1062A000039900EB0110D0F8B00100F0040002994E
:1062B00088600298806858B9FFE7049800680399DD
:1062C00000EB0110D0F8B001400D029908600AE01F
:1062D00004980068039900EB0110D0F8B001C008E1
:1062E00002994860FFE704980068039900EB0110E9
:1062F000D0F8B00100F002000299C860049800686C
:10630000039900EB0110D0F8B40100F00F00082849
:1063100004D3FFE70299082008610BE004980068A5
:10632000039900EB0110D0F8B40100F00F000299BE
:106330000861FFE704980068039900EB0110D0F8AA
:10634000B40180B2000A0299886104980068039938
:1063500000EB0110D0F8B401000C029948610498D8
:106360000068039900EB0110D0F8B801019908709A
:1063700004980068039900EB0110D0F8B801000AF6
:106380000199487004980068039900EB0110D0F857
:10639000B801000C0199887004980068039900EB1B
:1063A0000110D0F8B801000E0199C8700498006877
:1063B000039900EB0110D0F8BC0101990871049811
:1063C0000068039900EB0110D0F8BC01000A0199A4
:1063D000487104980068039900EB0110D0F8BC01E3
:1063E000000C0199887104980068039900EB011072
:1063F000D0F8BC01000E0199C871039838B9FFE7C5
:1064000004980168C86840F02000C86006E004985D
:106410000168086940F020000861FFE700208DF85E
:10642000170008E00499486A40F48020486201207F
:106430008DF81700FFE79DF8170006B070470000C1
:1064400083B0029000200190029890F820008DF80F
:1064500003009DF80300012805D0FFE79DF8030025
:10646000022822D1FFE702980068806840010028D6
:1064700004D5FFE7019801300190FFE7029800681A
:1064800080680001002804D5FFE7019801300190E1
:10649000FFE7029800688068C000002804D5FFE785
:1064A000019801300190FFE7FFE7019803B07047C2
:1064B00080B58AB00990002008900998006840696A
:1064C00007900998006840680690099800688068FD
:1064D000059009980068C0680490099800680069F0
:1064E000039009980068806902909DF81C00C0071D
:1064F000002800F09480FFE79DF81400C00758B30F
:10650000FFE709980168012088609DF81400800762
:10651000002804D5FFE7099800F0C0FC1BE09DF8B7
:1065200014004007002805D5FFE7089840F40060F4
:1065300008900FE09DF814000007002805D5FFE73C
:10654000089840F48050089003E0099800F07EFC21
:10655000FFE7FFE7FFE7FFE79DF81500C00760B31F
:10656000FFE7099801684FF4807088609DF8150076
:106570008007002804D5FFE7099800F0DDFC1BE048
:106580009DF815004007002805D5FFE7089840F45E
:10659000005008900FE09DF815000007002805D571
:1065A000FFE7089840F48040089003E0099800F065
:1065B0009BFCFFE7FFE7FFE7FFE79DF81600C0073A
:1065C00060B3FFE7099801684FF4803088609DF858
:1065D00016008007002804D5FFE7099800F0FCFCAE
:1065E0001BE09DF816004007002805D5FFE7089836
:1065F00040F4004008900FE09DF8160000070028C6
:1066000005D5FFE7089840F48030089003E009982A
:1066100000F0BAFCFFE7FFE7FFE7FFE7FFE79DF8C1
:106620001C000007002810D5FFE79DF81000C006E9
:10663000002809D5FFE7089840F4007008900998F1
:1066400001681020C860FFE7FFE79DF81C004007C5
:1066500000280FD5FFE79DF810000007002808D597
:10666000FFE7099801680820C860099800F0E0FA7F
:10667000FFE7FFE79DF81C00800700280BD5FFE728
:1066800009980068C068800720B1FFE7099800F00A
:10669000F7FAFFE7FFE79DF81C004006002810D539
:1066A000FFE79DF80C00C006002809D5FFE7089811
:1066B00040F4806008900998016810200861FFE7A5
:1066C000FFE79DF81C00800600280FD5FFE79DF826
:1066D0000C000007002808D5FFE70998016808208A
:1066E0000861099800F0F4FAFFE7FFE79DF81C0045
:1066F000C00600280BD5FFE70998006800698007ED
:1067000020B1FFE7099800F00BFBFFE7FFE79DF8DA
:106710001E00800700280FD5FFE79DF81800C0066F
:10672000002808D5FFE709980168102048600998FB
:1067300000F01EFBFFE7FFE79DF81E00C00778B1E1
:10674000FFE79DF818000007002808D5FFE7099823
:10675000016808204860099800F066FCFFE7FFE741
:106760009DF81D000006002840F18D80FFE79DF890
:1067700018004007002840F18180FFE79DF81D00C8
:10678000C00750B1FFE79DF80800C00728B1FFE738
:10679000089840F001000890FFE79DF81D00800771
:1067A00000280BD5FFE79DF808008007002805D5D5
:1067B000FFE7089840F002000890FFE79DF81D00F1
:1067C000400700280BD5FFE79DF808004007002888
:1067D00005D5FFE7089840F004000890FFE79DF812
:1067E0001D000007002848D5FFE79DF8080010F0BD
:1067F000700F42D0FFE7029800F07000014601914F
:10680000102814D0FFE70198202815D0FFE7019841
:10681000302816D0FFE70198402817D0FFE70198ED
:10682000502818D0FFE70198602819D01DE008987B
:1068300040F00800089019E0089840F01000089017
:1068400014E0089840F0200008900FE0089840F00D
:10685000400008900AE0089840F08000089005E0A9
:10686000089840F48070089000E0FFE709980168FC
:10687000886920F070008861FFE7FFE709980168E8
:1068800004204860FFE7089848B1FFE7089A099993
:10689000486A104348620998FFF776FCFFE70AB0A0
:1068A00080BD000080B584B00290029820B9FFE757
:1068B00001208DF80F00E0E0029890F8200020B948
:1068C000FFE7029800F0DEF8FFE702980168086829
:1068D00040F00100086001F08FF90190FFE7029895
:1068E00000684068C007A8B9FFE701F085F9019981
:1068F000401A0B280DD3FFE70299486A40F4003094
:1069000048620299052081F8200001208DF80F00CF
:10691000B3E0E4E702980168086820F0020008602C
:1069200001F06AF90190FFE702980068406880076B
:10693000002815D5FFE701F05FF90199401A0B28EF
:106940000DD3FFE70299486A40F40030486202998B
:10695000052081F8200001208DF80F008DE0E3E78D
:106960000298007E012807D1FFE7029801680868B5
:1069700040F08000086006E002980168086820F096
:1069800080000860FFE70298407E012807D1FFE7FA
:1069900002980168086840F04000086006E002982C
:1069A0000168086820F040000860FFE70298807ED8
:1069B000012807D1FFE702980168086840F020002D
:1069C000086006E002980168086820F0200008606E
:1069D000FFE70298C07E012807D1FFE7029801680F
:1069E000086820F01000086006E002980168086856
:1069F00040F010000860FFE70298007F012807D1EF
:106A0000FFE702980168086840F00800086006E0A7
:106A100002980168086820F008000860FFE7029803
:106A2000407F012807D1FFE702980168086840F01D
:106A30000400086006E002980168086820F004007D
:106A40000860FFE7029B19685A689868D3F80CC081
:106A500040EA0C00D3F810C040EA0C005B69184310
:106A6000013A1043C861029900204862029A01214C
:106A700082F820108DF80F00FFE79DF80F0004B09A
:106A800080BD000080B594B013900020129011904A
:106A900010900F900E901398006846F20041C4F2D7
:106AA0000001884253D1FFE740F23C50C2F200009F
:106AB0000168013101600068012812D1FFE7FFE79A
:106AC00000200D9043F64000C4F20200016841F03E
:106AD00000710160006800F000700D900D98FFE7F4
:106AE000FFE7FFE700200C9043F63000C4F20200FD
:106AF000016841F008010160006800F008000C9096
:106B00000C98FFE703200E9002210F9100210791BE
:106B1000109111900920129040F60040C4F202003A
:106B20000EA900F05DFE079A14200590052106913C
:106B300001F00AF9059801F0FDF80699079A152069
:106B4000089001F001F9089801F0F4F86EE013984C
:106B5000006846F60001C4F20001884265D1FFE7F3
:106B6000FFE700200B9043F64000C4F202000168EA
:106B700041F080610160006800F080600B900B982C
:106B8000FFE740F23C50C2F20000016801310160B1
:106B90000068012812D1FFE7FFE700200A9043F6C2
:106BA0004000C4F20200016841F000710160006819
:106BB00000F000700A900A98FFE7FFE7FFE7002067
:106BC000099043F63000C4F20200016841F002016E
:106BD0000160006800F0020009900998FFE760205A
:106BE0000E9002200F90002003901090032011902F
:106BF0000920129040F20040C4F202000EA900F0F9
:106C0000EFFD039A402001900521029101F09CF8CC
:106C1000019801F08FF80299039A4120049001F045
:106C200093F8049801F086F8FFE7FFE714B080BD01
:106C300080B582B001900198FCF764FC8DF80300E8
:106C40009DF80300032819D0FFE79DF8030040F2E8
:106C50009442C2F20002342110FB0120C06960B1ED
:106C6000FFE79DF8030040F29442C2F20002342193
:106C700010FB0120C0698047FFE7FFE702B080BD3D
:106C800080B582B001900198FCF73CFC8DF80300C0
:106C90009DF80300032819D0FFE79DF8030040F298
:106CA0009442C2F20002342110FB0120806960B1DD
:106CB000FFE79DF8030040F29442C2F20002342143
:106CC00010FB012080698047FFE7FFE702B080BD2D
:106CD00080B582B001900198FCF714FC8DF8030098
:106CE0009DF80300032819D0FFE79DF8030040F248
:106CF0009442C2F20002342110FB0120406A60B1CC
:106D0000FFE79DF8030040F29442C2F200023421F2
:106D100010FB0120406A8047FFE7FFE702B080BD1B
:106D200080B582B001900198FCF7ECFB8DF8030070
:106D30009DF80300032819D0FFE79DF8030040F2F7
:106D40009442C2F20002342110FB0120006A60B1BB
:106D5000FFE79DF8030040F29442C2F200023421A2
:106D600010FB0120006A8047FFE7FFE702B080BD0B
:106D700080B582B001900198FCF7C4FB8DF8030048
:106D80009DF80300032819D0FFE79DF8030040F2A7
:106D90009442C2F20002342110FB0120806A60B1EB
:106DA000FFE79DF8030040F29442C2F20002342152
:106DB00010FB0120806A8047FFE7FFE702B080BD3B
:106DC00080B584B00290029890F8200001282FD15D
:106DD000FFE70299022081F8200002980168086804
:106DE00020F00100086000F007FF0190FFE7029823
:106DF00000684068C007A8B1FFE700F0FDFE0199F8
:106E0000401A0B280DD3FFE70299486A40F400307E
:106E100048620299052081F8200001208DF80F00BA
:106E20000FE0E4E70299002048628DF80F0008E0C7
:106E30000299486A40F40020486201208DF80F0052
:106E4000FFE79DF80F0004B080BD000080B582B060
:106E500001900198FCF756FB8DF803009DF80300A4
:106E6000032819D0FFE79DF8030040F29442C2F2D4
:106E70000002342110FB0120C06860B1FFE79DF8DB
:106E8000030040F29442C2F20002342110FB0120C0
:106E9000C0688047FFE7FFE702B080BD80B582B0E1
:106EA00001900198FCF72EFB8DF803009DF803007C
:106EB000032817D0FFE79DF803003421414340F237
:106EC0009440C2F20000405858B1FFE79DF803001B
:106ED0003421414340F29440C2F2000040588047C0
:106EE000FFE7FFE702B080BD80B582B00190019856
:106EF000FCF708FB8DF803009DF80300032819D068
:106F0000FFE79DF8030040F29442C2F200023421F0
:106F100010FB0120006960B1FFE79DF8030040F21B
:106F20009442C2F20002342110FB01200069804724
:106F3000FFE7FFE702B080BD80B582B00190019805
:106F4000FCF7E0FA8DF803009DF80300032819D040
:106F5000FFE79DF8030040F29442C2F200023421A0
:106F600010FB0120406860B1FFE79DF8030040F28C
:106F70009442C2F20002342110FB01204068804795
:106F8000FFE7FFE702B080BD80B582B001900198B5
:106F9000FCF7B8FA8DF803009DF80300032819D018
:106FA000FFE79DF8030040F29442C2F20002342150
:106FB00010FB0120406960B1FFE79DF8030040F23B
:106FC0009442C2F20002342110FB01204069804744
:106FD000FFE7FFE702B080BD80B582B00190019865
:106FE000FCF790FA8DF803009DF80300032819D0F0
:106FF000FFE79DF8030040F29442C2F20002342100
:1070000010FB0120806860B1FFE79DF8030040F2AB
:107010009442C2F20002342110FB012080688047B4
:10702000FFE7FFE702B080BD80B582B00190019814
:10703000FCF768FA8DF803009DF80300032819D0C7
:10704000FFE79DF8030040F29442C2F200023421AF
:1070500010FB0120C06A60B1FFE79DF8030040F219
:107060009442C2F20002342110FB0120C06A804722
:10707000FFE7FFE702B080BD80B584B002900298C0
:10708000806D019000F0B8FD0090029890F83500F6
:1070900002280DD0FFE7029980204865FFE702999A
:1070A000002081F83400FFE701208DF80F0055E043
:1070B00002980168086820F01600086002980168CC
:1070C000486920F0800048610298006C20B9FFE711
:1070D0000298806C38B1FFE702980168086820F0D8
:1070E00008000860FFE702980168086820F00100C6
:1070F0000860FFE7029800680068C007C8B1FFE7B2
:1071000000F07AFD0099401A062811D3FFE7029992
:10711000202048650299032081F83500FFE7029995
:10712000002081F83400FFE703208DF80F0015E000
:10713000E0E70298C16D3F2088400199886002997C
:10714000012081F83500FFE70299002081F8340022
:10715000FFE7FFE700208DF80F00FFE79DF80F0025
:1071600004B080BD82B00090009890F835000228ED
:1071700007D0FFE700998020486501208DF80700BF
:107180000EE00099052081F8350000980168086834
:1071900020F001000860FFE700208DF80700FFE7FE
:1071A0009DF8070002B0704780B586B005900020BA
:1071B000039040F20000C2F20000006848F2B511EE
:1071C000C1F64E31A0FB0110800A02900598806D37
:1071D000019001980068049004980599C96DC84011
:1071E000000700281AD5FFE70598006800684007E7
:1071F000002812D5FFE705980168086820F0040010
:1072000008600598C16D082088400199886005993B
:10721000486D40F001004865FFE7FFE704980599D5
:10722000C96DC840C007A0B1FFE705980068406974
:10723000000600280CD5FFE70598C16D01208840A5
:10724000019988600599486D40F002004865FFE7A4
:10725000FFE704980599C96DC8404007002814D578
:10726000FFE7059800680068800700280CD5FFE755
:107270000598C16D04208840019988600599486D82
:1072800040F004004865FFE7FFE704980599C96DE1
:10729000C840C006002847D5FFE705980068006889
:1072A000000700283FD5FFE70598C16D10208840F2
:1072B00001998860059800680068400300281AD585
:1072C000FFE70598006800680003002809D4FFE77D
:1072D0000598006C20B1FFE70598016C8847FFE72F
:1072E00008E00598806C20B1FFE70598816C88471D
:1072F000FFE7FFE716E0059800680068C005002872
:1073000007D4FFE705980168086820F008000860C6
:10731000FFE70598006C20B1FFE70598016C8847EE
:10732000FFE7FFE7FFE7FFE704980599C96DC8404D
:107330008006002840F18D80FFE70598006800680E
:10734000C006002840F18480FFE70598C16D202029
:10735000884001998860059890F83500052834D157
:10736000FFE705980168086820F016000860059896
:107370000168486920F0800048610598006C20B9D8
:10738000FFE70598806C38B1FFE705980168086849
:1073900020F008000860FFE70598C16D3F20884095
:1073A000019988600599012081F83500FFE705996A
:1073B000002081F83400FFE70598006D20B1FFE759
:1073C0000598016D8847FFE77BE005980068006835
:1073D000400300281AD5FFE70598006800680003FD
:1073E000002809D4FFE70598406C20B1FFE7059815
:1073F000416C8847FFE708E00598C06B20B1FFE7C4
:107400000598C16B8847FFE7FFE720E00598006813
:107410000068C005002811D4FFE7059801680868D6
:1074200020F0100008600599012081F83500FFE781
:107430000599002081F83400FFE7FFE70598C06B4D
:1074400020B1FFE70598C16B8847FFE7FFE7FFE73B
:10745000FFE70598406DA0B3FFE70598406DC007B2
:1074600030B3FFE70599052081F8350005980168DC
:10747000086820F001000860FFE7039801300390DE
:107480000299884201D9FFE707E0FFE70598006805
:107490000068C0070028F0D1FFE70599012081F8B6
:1074A0003500FFE70599002081F83400FFE7FFE78A
:1074B0000598C06C20B1FFE70598C16C8847FFE7CD
:1074C000FFE706B080BD000080B586B004900020C4
:1074D000039000F091FB0290049820B9FFE701208F
:1074E0008DF81700A3E00498406A08B1FFE7FFE7B2
:1074F0000499022081F83500FFE70499002081F803
:107500003400FFE704980168086820F00100086073
:10751000FFE7049800680068C00790B1FFE700F03B
:107520006BFB0299401A06280AD3FFE70499202032
:1075300048650499032081F835008DF8170076E03E
:10754000E7E70498006800680390039848F23F0159
:10755000CFF2100108400390049900914868D1F8D7
:1075600008C0CB680A6940EA0C00184310434A6916
:1075700010438A691043CA691043096A014303989A
:10758000084303900498406A042808D1FFE704994F
:10759000C86A096B0143039808430390FFE7039807
:1075A000049909680860049800684069039003988A
:1075B00020F0070003900498416A03980843039061
:1075C0000498406A04281AD1FFE70498816A039856
:1075D000084303900498C06A80B1FFE70498FDF760
:1075E0002BFD50B1FFE70499402048650499012024
:1075F00081F835008DF8170019E0FFE7FFE70398E1
:107600000499096848610498FDF7EAFC0190049820
:10761000C16D3F2088400199886004990020486529
:10762000049A012182F835108DF81700FFE79DF8C4
:10763000170006B080BD000080B588B006900591A7
:107640000492039300208DF80B000698806D019042
:10765000FFE7069890F83400012804D1FFE70220E4
:107660008DF81F0045E00699012081F83400FFE7FE
:10767000FFE7069890F8350001282BD1FFE706991F
:10768000022081F835000699002048650698059982
:10769000049A039BFDF748FD0698C16D3F20884082
:1076A0000199886006980168086840F01600086033
:1076B0000698006C38B1FFE706980168086840F04A
:1076C00008000860FFE706980168086840F00100BC
:1076D000086009E0FFE70699002081F83400FFE721
:1076E00002208DF80B00FFE79DF80B008DF81F00BE
:1076F000FFE79DF81F0008B080BD000080B584B092
:10770000039000F079FA02900398019001980130FB
:1077100048B1FFE740F24430C2F20000017801981E
:1077200008440190FFE7FFE700F066FA0299401A6B
:107730000199884201D2FFE7F6E704B080BD00005E
:1077400080B582B0ADF8060000208DF80500FFE797
:107750009DF805000F2824DCFFE7BDF806009DF822
:107760000510C840C007A8B1FFE79DF8051040F21A
:10777000FC40C2F2000050F8210050B1FFE79DF834
:10778000051040F2FC40C2F2000050F82100804792
:10779000FFE7FFE7FFE79DF8050001308DF80500E2
:1077A000D6E702B080BD000080B582B0ADF806001B
:1077B00043F61440C4F201000068BDF80610084208
:1077C0000CD0FFE7BDF8060043F61441C4F20101F6
:1077D0000860BDF80600FFF7B3FFFFE702B080BD09
:1077E0008EB00D900C9100200A90099008900B909B
:1077F000FFE70B980F2800F2CC81FFE70B990120DF
:1078000088400A900C9800680A99084009900998E5
:107810000A99884240F0B881FFE70C98406800F070
:107820000300012807D0FFE70C98406800F0030030
:1078300002282FD1FFE70D98806808900B9841002F
:10784000032000FA01F10898884308900C98C0685A
:107850000B99490000FA01F108980843089008982C
:107860000D9988600D98406808900B99012000FAE6
:1078700001F10898884308900C984068C0F3001004
:107880000B9900FA01F108980843089008980D999F
:107890004860FFE70C98406800F00300032818D008
:1078A000FFE70D98C06808900B984100032000FA8C
:1078B00001F10898884308900C9880680B9949005A
:1078C00000FA01F108980843089008980D99C860DB
:1078D000FFE70C98406800F00300022826D1FFE77C
:1078E0000D980B996FF0030202EA51010844006AF7
:1078F00008900B9800F0070081000F2000FA01F1BA
:107900000898884308900C9800690B9901F00701CA
:10791000890000FA01F108980843089008980D9929
:107920000B9B02EA530211440862FFE70D980068BE
:1079300008900B984100032000FA01F10898884351
:1079400008900C98406800F003000B99490000FA79
:1079500001F108980843089008980D9908600C9860
:1079600080798007002800F00E81FFE7FFE7002004
:10797000079043F64400C4F20200016841F48041DC
:107980000160006800F4804007900798FFE70B98BB
:1079900020F0030043F60801C4F2010140580890AA
:1079A0000B9800F0030081000F2000FA01F1089805
:1079B000884308900D980021C4F20201884203D147
:1079C000FFE7002006905EE00D9840F20041C4F20F
:1079D0000201884203D1FFE70120059050E00D9895
:1079E00040F60001C4F20201884203D1FFE7022001
:1079F000049042E00D9840F60041C4F20201884232
:107A000003D1FFE70320039034E00D9841F2000119
:107A1000C4F20201884203D1FFE70420029026E06D
:107A20000D9841F20041C4F20201884203D1FFE700
:107A30000520019018E00D9841F60001C4F2020102
:107A4000884203D1FFE7062000900AE00D9941F635
:107A50000042C4F202020820914208BF07200090B1
:107A6000FFE700980190FFE701980290FFE7029876
:107A70000390FFE703980490FFE704980590FFE761
:107A800005980690FFE70698C0B20B9901F0030134
:107A9000890000FA01F108980843089008980B99AA
:107AA00021F0030143F60802C4F20102885043F6B4
:107AB0000840C4F2010000680890099908988843BA
:107AC00008900C988079C006002805D5FFE7099931
:107AD000089808430890FFE7089843F60841C4F265
:107AE0000101086043F60C40C4F2010000680890F0
:107AF00009990898884308900C9880798006002896
:107B000005D5FFE70999089808430890FFE708980A
:107B100043F60C41C4F20101086043F60440C4F28C
:107B200001000068089009990898884308900C980B
:107B300080798007002805D5FFE709990898084350
:107B40000890FFE7089843F60441C4F20101086079
:107B500043F60040C4F201000068089009990898B3
:107B6000884308900C988079C00728B1FFE70999ED
:107B7000089808430890FFE7089843F60041C4F2CC
:107B800001010860FFE7FFE7FFE70B9801300B906A
:107B90002FE60EB07047000082B00190ADF80210E1
:107BA00001980069BDF80210084204D0FFE70120E7
:107BB0008DF8010003E000208DF80100FFE79DF83B
:107BC000010002B07047000082B00190ADF80210D1
:107BD0008DF801209DF8010028B1FFE7BDF80200F3
:107BE0000199886105E0BDF80200000401998861EF
:107BF000FFE702B07047000042F23C70C2F20100A1
:107C00000068704740F24430C2F20000027842F24D
:107C10003C71C2F20101086810440860704700001E
:107C200080B543F60041C4F20201086840F40070D8
:107C30000860086840F480600860086840F480705C
:107C40000860032000F09AF80F2000F005F800F01B
:107C50003BF8002080BD000080B582B0009040F26B
:107C60000000C2F20000006840F24431C2F200019C
:107C70000A784FF47A71B1FBF2F1B0FBF1F001F048
:107C8000F7FE20B1FFE701208DF8070018E000980B
:107C90000F280DD8FFE700994FF0FF30002200F0C9
:107CA00053F8009840F24831C2F20001086003E046
:107CB00001208DF8070003E000208DF80700FFE7A2
:107CC0009DF8070002B080BD80B582B0FFE70020BC
:107CD000019043F64400C4F20200016841F480417F
:107CE0000160006800F4804001900198FFE7FFE721
:107CF0000020009043F64000C4F20200016841F009
:107D000080510160006800F0805000900098FFE70B
:107D10006FF001000F21002200F016F802B080BDC4
:107D200080B582B08DF807009DF9070007F042FF8B
:107D300002B080BD80B582B08DF807009DF90700C4
:107D400007F054FF02B080BD80B586B08DF81700F3
:107D5000049103920020029007F060FF02909DF9C9
:107D60001700019002980499039A04F0DDFA014685
:107D7000019807F05BFF06B080BD000080B582B0BF
:107D80000190019807F096FF02B080BD80B584B0E5
:107D900002900191029820B9FFE701208DF80F00B1
:107DA00021E1019843F60041C4F20201096801F0A3
:107DB0000701884212D9FFE7019943F60040C4F257
:107DC00002000170006800F007000199884204D0A9
:107DD000FFE701208DF80F0005E1FFE7029800782A
:107DE000800700282AD5FFE702980078400700287E
:107DF00009D5FFE743F60801C4F20201086840F420
:107E0000E0500860FFE7029800780007002809D5D5
:107E1000FFE743F60801C4F20201086840F460403D
:107E20000860FFE743F60801C4F20201086820F089
:107E3000F000029A926810430860FFE70298007809
:107E4000C00700286ED0FFE702984068012811D1D2
:107E5000FFE743F60000C4F20200006800F40031BE
:107E60000020B0EB514F04D1FFE701208DF80F0047
:107E7000B9E02CE002984068022805D0FFE702989C
:107E80004068032811D1FFE743F60000C4F2020066
:107E9000006800F000710020B0EB516F04D1FFE7E3
:107EA00001208DF80F009EE010E043F60000C4F2C0
:107EB0000200006800F002010020B0EB510F04D175
:107EC000FFE701208DF80F008DE0FFE7FFE743F6A5
:107ED0000801C4F20201086820F00300029A526807
:107EE00010430860FFF788FE0090FFE743F60800A4
:107EF000C4F20200006800F00C0002994968B0EB7F
:107F0000810F0ED0FFE7FFF777FE0099401A41F28C
:107F10008931884204D3FFE703208DF80F0062E027
:107F2000E4E7FFE7019843F60041C4F20201096863
:107F300001F00701884212D2FFE7019943F60040A1
:107F4000C4F202000170006800F007000199884245
:107F500004D0FFE701208DF80F0044E0FFE702980E
:107F60000078400700280CD5FFE743F60801C4F26B
:107F70000201086820F4E050029AD26810430860B9
:107F8000FFE702980078000700280DD5FFE743F6C9
:107F90000801C4F20201086820F46040029A1269E4
:107FA00040EAC2000860FFE700F04CF843F6080121
:107FB000C4F202010968C9B20A0948F22811C0F6E0
:107FC0000101895CC84040F20001C2F20001086072
:107FD00040F24830C2F200000068FFF73DFE00208A
:107FE0008DF80F00FFE79DF80F0004B080BD000082
:107FF00040F20000C2F200000068704780B5FFF751
:10800000F7FF43F60801C4F202010968C1F38222B6
:1080100048F23811C0F60101895CC84080BD0000FB
:1080200080B5FFF7E5FF43F60801C4F202010968D5
:1080300089B24A0B48F23811C0F60101895CC84088
:1080400080BD000080B586B00020059004900390AC
:10805000029043F60800C4F20200006800F00C0031
:108060000146019140B1FFE7019804280AD0FFE7DB
:10807000019808280CD04FE042F20040C0F2F40012
:1080800002904FE041F60030C0F2B700029049E0A4
:1080900043F60400C4F20200016801F03F010591BB
:1080A00000684002002813D5FFE743F60400C4F23D
:1080B00002000068C0F3881041F60031C0F2B70139
:1080C000A0FB0101059A0023F8F7F0F8049012E0F4
:1080D00043F60400C4F202000068C0F3881042F2C4
:1080E0000041C0F2F401A0FB0101059A0023F8F75A
:1080F000DDF80490FFE743F60400C4F202000068D4
:1081000000F44031022000EBD13003900498039931
:10811000B0FBF1F0029005E042F20040C0F2F40042
:108120000290FFE7029806B080BD000080B586B0DF
:108130000490049820B9FFE701208DF8170050E360
:1081400004980078C007002800F0A580FFE743F6F8
:108150000800C4F20200006800F00C00042813D0EC
:10816000FFE743F60800C4F20200006800F00C00CC
:1081700008281ED1FFE743F60400C4F2020000689D
:108180004002002815D5FFE743F60000C4F20200C4
:10819000006800F400310020B0EB514F08D0FFE739
:1081A0000498406820B9FFE701208DF8170018E314
:1081B00070E0FFE704984068B0F5803F09D1FFE721
:1081C00043F60001C4F20201086840F48030086000
:1081D00020E004984068B0F5A02F0DD1FFE743F6EA
:1081E0000001C4F20201086840F4802008600868B9
:1081F00040F4803008600CE043F60001C4F2020154
:10820000086820F480300860086820F48020086046
:10821000FFE7FFE7FFE704984068E8B1FFE7FFF7F3
:10822000EBFC0390FFE743F60000C4F20200006895
:1082300000F400310020B0EB514F0CD1FFE7FFF705
:10824000DBFC0399401A652804D3FFE703208DF86F
:108250001700C6E2E7E71CE0FFF7CEFC0390FFE75C
:1082600043F60000C4F20200006800F40031002070
:10827000B0EB514F0CD0FFE7FFF7BEFC0399401A5B
:10828000652804D3FFE703208DF81700A9E2E7E78C
:10829000FFE7FFE7FFE7049800788007002840F138
:1082A0009680FFE743F60800C4F20200006810F071
:1082B0000C0F13D0FFE743F60800C4F20200006879
:1082C00000F00C0008282CD1FFE743F60400C4F2AC
:1082D000020000684002002823D4FFE743F60000B4
:1082E000C4F20200006800F002010020B0EB510F60
:1082F00009D0FFE70498C068012804D0FFE70120F7
:108300008DF817006DE243F60001C4F2020108681F
:1083100020F0F800049A126940EAC2000860FFE702
:1083200054E00498C06870B3FFE70021C4F247210D
:1083300001200860FFF760FC0390FFE743F60000B0
:10834000C4F20200006800F002010020B0EB510FFF
:108350000CD1FFE7FFF750FC0399401A032804D320
:10836000FFE703208DF817003BE2E7E743F6000143
:10837000C4F20201086820F0F800049A126940EA89
:10838000C200086021E00021C4F2472100200860FB
:10839000FFF732FC0390FFE743F60000C4F202004F
:1083A000006800F002010020B0EB510F0CD0FFE795
:1083B000FFF722FC0399401A032804D3FFE70320A8
:1083C0008DF817000DE2E7E7FFE7FFE7FFE7049806
:1083D0000078000700284BD5FFE70498406918B3E0
:1083E000FFE740F68061C4F2472101200860FFF7F3
:1083F00003FC0390FFE743F67400C4F20200006838
:1084000000F002010020B0EB510F0CD1FFE7FFF7A5
:10841000F3FB0399401A032804D3FFE703208DF8E8
:108420001700DEE1E7E722E040F68061C4F2472171
:1084300000200860FFF7E0FB0390FFE743F67400BD
:10844000C4F20200006800F002010020B0EB510FFE
:108450000CD0FFE7FFF7D0FB0399401A032804D3A1
:10846000FFE703208DF81700BBE1E7E7FFE7FFE731
:10847000049800784007002840F1CE80FFE70020F4
:108480008DF8070043F64000C4F202000068C00007
:10849000002815D4FFE7FFE70020009043F64000D6
:1084A000C4F20200016841F080510160006800F0F0
:1084B000805000900098FFE701208DF80700FFE74B
:1084C00047F20000C4F200000068C005002822D472
:1084D000FFE747F20001C4F20001086840F4807031
:1084E0000860FFF789FB0390FFE747F20000C4F242
:1084F00000000068C00500280CD4FFE7FFF77CFBF4
:108500000399401A032804D3FFE703208DF81700CE
:1085100067E1EAE7FFE7FFE704988068012809D1EF
:10852000FFE743F67001C4F20201086840F0010061
:1085300008601FE00498806805280DD1FFE743F626
:108540007001C4F20201086840F004000860086885
:1085500040F0010008600CE043F67001C4F2020133
:10856000086820F001000860086820F00400086036
:10857000FFE7FFE7FFE704988068F8B1FFE7FFF740
:108580003BFB0390FFE743F67000C4F20200006873
:1085900000F002010020B0EB510F0ED1FFE7FFF712
:1085A0002BFB0399401A41F28931884204D3FFE73B
:1085B00003208DF8170014E1E5E71EE0FFF71CFB30
:1085C0000390FFE743F67000C4F20200006800F079
:1085D00002010020B0EB510F0ED0FFE7FFF70CFBBC
:1085E0000399401A41F28931884204D3FFE70320FE
:1085F0008DF81700F5E0E5E7FFE79DF80700012893
:1086000009D1FFE743F64001C4F20201086820F0F7
:1086100080500860FFE7FFE704988069002800F0B9
:10862000DC80FFE743F60800C4F20200006800F0B7
:108630000C00082800F08580FFE704988069022874
:108640005CD1FFE76021C4F2472100200860FFF7FA
:10865000D3FA0390FFE743F60000C4F2020000687B
:1086600000F000710020B0EB516F0CD0FFE7FFF776
:10867000C3FA0399401A032804D3FFE703208DF8B7
:108680001700AEE0E7E70499C869D1F820C04B6A4B
:108690008A6A40EA0C0040EA8310D2034FF6FF7367
:1086A0009A43A2F580321043C96A40EA016043F65A
:1086B0000401C4F2020108606021C4F247210120D4
:1086C0000860FFF799FA0390FFE743F60000C4F251
:1086D0000200006800F000710020B0EB516F0CD177
:1086E000FFE7FFF789FA0399401A032804D3FFE74D
:1086F00003208DF8170074E0E7E721E06021C4F261
:10870000472100200860FFF777FA0390FFE743F660
:108710000000C4F20200006800F000710020B0EB1D
:10872000516F0CD0FFE7FFF767FA0399401A03284F
:1087300004D3FFE703208DF8170052E0E7E7FFE7D7
:108740004AE004988069012804D1FFE701208DF8F0
:10875000170046E043F60400C4F2020000680290ED
:1087600004988069012831D0FFE7029800F4800066
:108770000499C969884229D1FFE7029800F03F00B7
:108780000499096A884221D1FFE7029847F6C0712F
:1087900008400499496AB0EB811F17D1FFE702989E
:1087A00000F440300499896AC9034FF6FF7291437F
:1087B000A1F58031884209D1FFE7029800F070608E
:1087C0000499C96AB0EB016F04D0FFE701208DF86E
:1087D000170006E0FFE7FFE7FFE700208DF817002E
:1087E000FFE79DF8170006B080BD000080B582B09D
:1087F0000190019804F05AFB8DF803009DF80300E6
:1088000002281BD0FFE7019804F050FB014640F21C
:108810004450C2F2000000EB4110806968B1FFE7EC
:10882000019804F043FB014640F24450C2F20000BC
:1088300000EB411080698047FFE7FFE702B080BD91
:1088400080B584B00290029820B9FFE701208DF82E
:108850000F0071E00298406A60B9FFE70298406833
:10886000B0F5827F01D1FFE703E002990020C861E3
:10887000FFE705E002990020086102994861FFE7DF
:10888000029900208862029890F8510040B9FFE7F1
:108890000299002081F85000029800F051F8FFE79B
:1088A0000299022081F8510002980168086820F0BE
:1088B00040000860029A019211685068D2F808C01E
:1088C000D36800F482700CF4044C604403F4006339
:1088D0001844136903F002031844536903F00103B9
:1088E0001844936903F400731844D36903F0380300
:1088F0001844136A03F080031843926A02F400528A
:1089000010430860029A508B00F004001168526A0C
:1089100002F010021044486002980168C86920F40F
:108920000060C861029900204865029A012182F81E
:1089300051108DF80F00FFE79DF80F0004B080BDC7
:1089400080B590B00F9000200E900D900C900B9081
:108950000A900F98006843F20001C4F201018842B6
:1089600040F0B680FFE7FFE70020099043F644009F
:10897000C4F20200016841F480510160006800F413
:10898000805009900998FFE7FFE70020089043F620
:108990003000C4F20200016841F002010160006889
:1089A00000F0020008900898FFE7FFE7002007901A
:1089B00043F63000C4F20200016841F00101016099
:1089C000006800F0010007900798FFE718200A9060
:1089D000022001900B90002005900C900320029043
:1089E0000D90052003900E9040F20040C4F202006A
:1089F0000AA90491FEF7F4FEDDF804C0029A039878
:108A00000499059B4FF0800ECDF828E0CDF82CC0DE
:108A10000C930D920E900020C4F20200FEF7E0FECF
:108A2000059941F21C10C2F20000069046F2404245
:108A3000C4F2020202604FF0C06242608160C16015
:108A40004FF48062026141618161C1614FF4403243
:108A500002624162FEF738FD18B1FFE7FCF76EFDD8
:108A6000FFE7FFE70F9841F21C11C2F20001C16459
:108A70000F988863FFE741F27C10C2F2000000907B
:108A800046F25841C4F2020101604FF0C0614160FA
:108A9000402181600021C1604FF480620261416128
:108AA0008161C1614FF4003202624162FEF70CFD48
:108AB00018B1FFE7FCF742FDFFE7FFE70F9841F22F
:108AC0007C11C2F2000181640F988863FFE7FFE721
:108AD00010B080BD80B588B006900591ADF8122029
:108AE0000393069890F85100012804D0FFE7022074
:108AF0008DF81F0011E1059820B1FFE7BDF81200C5
:108B000020B9FFE701208DF81F0006E106984068B4
:108B1000B0F5827F16D1FFE70698806890B9FFE72D
:108B20000699042081F851000698059ABDF8123084
:108B30000399EC46CCF80010114600F065FB8DF867
:108B40001F00EAE0FFF758F80290FFE7069890F858
:108B50005000012804D1FFE702208DF81F00DCE05F
:108B60000699012081F85000FFE7FFE706990420ED
:108B700081F851000699002048650599069A91638D
:108B8000BDF81210069A9187BDF81210069AD18787
:108B900006990863069988860699C8860699086426
:108BA0000699486406988068B0F5004F0DD1FFE73C
:108BB00006980168086820F040000860069801687F
:108BC000086820F480400860FFE7069800680068A5
:108BD00000F04000402807D0FFE7069801680868C9
:108BE00040F040000860FFE70698C068D0BBFFE790
:108BF000FFE70698C08FA0B3FFE70698006880687B
:108C0000C00778B1FFE706980068007B0699896B7A
:108C100008700699886B013088630699C88F0138FF
:108C2000C8871DE0FEF7E8FF0299401A03998842C1
:108C300004D3FFE70398013018B9FFE7039870B930
:108C4000FFE70699012081F85100FFE7069900200F
:108C500081F85000FFE703208DF81F005DE0FFE77B
:108C6000C7E739E0FFE70698C08FA0B3FFE7069893
:108C700000688068C00778B1FFE706980068C068A0
:108C80000699896B08800699886B0230886306997B
:108C9000C88F0138C8871DE0FEF7AEFF0299401A61
:108CA0000399884204D3FFE70398013018B9FFE71E
:108CB000039870B9FFE70699012081F85100FFE79A
:108CC0000699002081F85000FFE703208DF81F006F
:108CD00023E0FFE7C7E7FFE706980399029A04F04D
:108CE0000DF820B1FFE7069920204865FFE70699B7
:108CF000012081F85100FFE70699002081F850001B
:108D0000FFE70698406D20B1FFE701208DF81F00B6
:108D100003E000208DF81F00FFE79DF81F0008B05A
:108D200080BD000080B584B002900191ADF80220B2
:108D3000029890F85100012804D0FFE702208DF836
:108D40000F00B7E0019820B1FFE7BDF8020020B99D
:108D5000FFE701208DF80F00ACE002988068A0B911
:108D6000FFE702984068B0F5827F0ED1FFE70299D5
:108D7000042081F851000298019ABDF80230114692
:108D800000F014FC8DF80F0094E0FFE7029890F8D3
:108D90005000012804D1FFE702208DF80F0089E080
:108DA0000299012081F85000FFE7FFE702990420B3
:108DB00081F851000299002048650199029A916357
:108DC000BDF80210029A9187BDF80210029AD1876D
:108DD0000299086402994864029988860299C886B3
:108DE00002988068B0F5004F0DD1FFE70298016846
:108DF000086820F04000086002980168086820F4C4
:108E000080400860FFE70298C16C4CF6E120C0F694
:108E1000000008640298C16C4CF62930C0F60000CE
:108E2000C8630298C16C4CF6AD20C0F60000C8645F
:108E30000298C16C00200865029B19689A6BD86C77
:108E40000C31DB8FFEF7F8FB78B1FFE70299486D34
:108E500040F010004865FFE70299002081F85000BB
:108E6000FFE701208DF80F0024E0029800680068F9
:108E700000F04000402807D0FFE70298016808682A
:108E800040F040000860FFE7FFE70299002081F80A
:108E90005000FFE702980168486840F020004860F1
:108EA00002980168486840F00100486000208DF891
:108EB0000F00FFE79DF80F0004B080BD80B582B0C1
:108EC0000190019803F0F2FF8DF803009DF8030074
:108ED00002281BD0FFE7019803F0E8FF014640F2AB
:108EE0004450C2F2000000EB4110406868B1FFE757
:108EF000019803F0DBFF014640F24450C2F200004B
:108F000000EB411040688047FFE7FFE702B080BDFB
:108F100080B582B00190019803F0C8FF8DF803007E
:108F20009DF8030002281BD0FFE7019803F0BEFF65
:108F3000014640F24450C2F2000000EB41100069CB
:108F400068B1FFE7019803F0B1FF014640F24450D9
:108F5000C2F2000000EB411000698047FFE7FFE725
:108F600002B080BD80B588B006900591ADF81220A2
:108F70000393FEF741FE0290BDF81200ADF8060023
:108F8000069890F85100012804D0FFE702208DF8E0
:108F90001F0034E1059820B1FFE7BDF8120020B9A9
:108FA000FFE701208DF81F0029E1FFE7069890F800
:108FB0005000012804D1FFE702208DF81F001EE1B8
:108FC0000699012081F85000FFE7FFE7069903208A
:108FD00081F851000699002048650599069A1163A9
:108FE000BDF81210069A9186BDF81210069AD18625
:108FF00006998863069988870699C8870699486400
:109000000699086406988068B0F5004F0DD1FFE717
:1090100006980168086820F040000860069801681A
:10902000086840F480400860FFE706980068006820
:1090300000F04000402807D0FFE706980168086864
:1090400040F040000860FFE70698C068B0F5006F88
:1090500051D1FFE70698406828B1FFE7BDF8060048
:1090600001280ED1FFE706980168006B0088C860F0
:109070000699086B023008630699C88E0138C886C5
:10908000FFE7FFE70698C08EA0B3FFE706980068E9
:109090008068800700280ED5FFE706980168006BFE
:1090A0000088C8600699086B023008630699C88E6C
:1090B0000138C8861DE0FEF79FFD0299401A03990A
:1090C000884204D3FFE70398013018B9FFE70398FB
:1090D00070B9FFE70699012081F85100FFE7069972
:1090E000002081F85000FFE703208DF81F0086E084
:1090F000FFE7C7E750E00698406828B1FFE7BDF8F2
:10910000060001280ED1FFE706980168006B007881
:1091100008730699086B013008630699C88E0138F8
:10912000C886FFE7FFE70698C08EA0B3FFE7069862
:1091300000688068800700280ED5FFE70698016860
:10914000006B007808730699086B01300863069974
:10915000C88E0138C8861DE0FEF74EFD0299401A00
:109160000399884204D3FFE70398013018B9FFE759
:10917000039870B9FFE70699012081F85100FFE7D5
:109180000699002081F85000FFE703208DF81F00AA
:1091900035E0FFE7C7E7FFE706980399029A03F077
:1091A0001FFE20B1FFE7069920204865FFE70698DB
:1091B000806870B9FFE7FFE700200090069800681C
:1091C000C068009006980068806800900098FFE7EB
:1091D000FFE70699012081F85100FFE7069900207A
:1091E00081F85000FFE70698406D20B1FFE70120AD
:1091F0008DF81F0003E000208DF81F00FFE79DF8A9
:109200001F0008B080BD000080B58CB0DDF838C00C
:109210000A9009910892ADF81E3001200390FEF7E4
:10922000EBFC04900A9890F851008DF817000A980A
:1092300040680690BDF81E00ADF81C009DF81700B0
:10924000012812D0FFE70698B0F5827F09D1FFE729
:109250000A98806828B9FFE79DF81700042804D011
:10926000FFE702208DF82F009BE1099838B1FFE756
:10927000089820B1FFE7BDF81E0020B9FFE70120E4
:109280008DF82F008DE1FFE70A9890F85000012833
:1092900004D1FFE702208DF82F0082E10A99012016
:1092A00081F85000FFE7FFE70A9890F85100042882
:1092B00005D0FFE70A99052081F85100FFE70A99D8
:1092C0000020486508990A9A9163BDF81E100A9A11
:1092D000D187BDF81E100A9A918709990A9A1163DD
:1092E000BDF81E100A9AD186BDF81E100A9A918602
:1092F0000A9908640A9948640A980068006800F0AE
:109300004000402807D0FFE70A980168086840F04D
:1093100040000860FFE70A98C068B0F5006F40F0B1
:109320008180FFE70A98406828B1FFE7BDF81C007C
:1093300001280ED1FFE70A980168006B0088C86019
:109340000A99086B023008630A99C88E0138C886EA
:10935000FFE7FFE70A98C18E0120019039B9FFE7C6
:109360000A98C08F002818BF01200190FFE70198DC
:10937000C007002855D0FFE70A980068806880077A
:10938000002818D5FFE70A98C08EA0B1FFE7039820
:10939000012810D1FFE70A980168006B0088C860B7
:1093A0000A99086B023008630A99C88E0138C8868A
:1093B00000200390FFE70A9800688068C007A8B102
:1093C000FFE70A98C08F88B1FFE70A980068C06875
:1093D0000A99896B08800A99886B023088630A9918
:1093E000C88F0138C88701200390FFE7FEF704FC0F
:1093F0000499401A0E99884212D3FFE70E98013063
:1094000070B1FFE70A99012081F85100FFE70A993E
:10941000002081F85000FFE703208DF82F00C0E006
:1094200098E782E00A98406828B1FFE7BDF81C0081
:1094300001280ED1FFE70A980168006B00780873D5
:109440000A99086B013008630A99C88E0138C886EA
:10945000FFE7FFE70A98C18E0120009039B9FFE7C6
:109460000A98C08F002818BF01200090FFE70098DD
:10947000C007002858D0FFE70A9800688068800776
:10948000002818D5FFE70A98C08EA0B1FFE703981F
:10949000012810D1FFE70A980168006B0078087373
:1094A0000A99086B013008630A99C88E0138C8868A
:1094B00000200390FFE70A9800688068C007A8B101
:1094C000FFE70A98C08F88B1FFE70A980068C06874
:1094D0000A99896B08700A99886B013088630A9928
:1094E000C88F0138C88701200390FFE7FEF784FB8F
:1094F0000499401A0E99884204D3FFE70E98013070
:1095000018B9FFE70E9870B9FFE70A99012081F8B2
:109510005100FFE70A99002081F85000FFE703207F
:109520008DF82F003DE095E7FFE70A980E99049A21
:1095300003F056FC68B1FFE70A9920204865FFE771
:109540000A99002081F85000FFE701208DF82F00D4
:1095500027E00A98806870B9FFE7FFE700200290D3
:109560000A980068C06802900A98006880680290B3
:109570000298FFE7FFE70A99012081F85100FFE711
:109580000A99002081F85000FFE70A98406D20B149
:10959000FFE701208DF82F0003E000208DF82F0059
:1095A000FFE79DF82F000CB080BD000080B588B0AB
:1095B000069005910492ADF80E30069890F851008F
:1095C0008DF807000698406802909DF80700012872
:1095D00012D0FFE70298B0F5827F09D1FFE7069825
:1095E000806828B9FFE79DF80700042804D0FFE74A
:1095F00002208DF81F00DFE0059838B1FFE70498DE
:1096000020B1FFE7BDF80E0020B9FFE701208DF87B
:109610001F00D1E0FFE7069890F85000012804D120
:10962000FFE702208DF81F00C6E00699012081F8AF
:109630005000FFE7FFE7069890F85100042805D096
:10964000FFE70699052081F85100FFE70699002001
:1096500048650599069A1163BDF80E10069A918621
:10966000BDF80E10069AD1860499069A9163BDF84A
:109670000E10069A9187BDF80E10069AD1870699AA
:10968000086406994864069890F8510004280FD1A0
:10969000FFE70698C16C4CF6E120C0F600000864B4
:1096A0000698C16C4CF62930C0F60000C8630EE085
:1096B0000698C16C4CF61130C0F60000086406989C
:1096C000C16C4CF67540C0F60000C863FFE7069811
:1096D000C16C4CF6AD20C0F60000C8640698C16CA1
:1096E00000200865069B19689A6BD86C0C31DB8FDB
:1096F000FDF7A2FF78B1FFE70699486D40F0100032
:109700004865FFE70699002081F85000FFE7012037
:109710008DF81F0050E006980168486840F001008D
:1097200048600698816C002008640699896CC863BB
:109730000699896CC8640699896C0865069B1A6845
:10974000196B986C0C32DB8EFDF776FF78B1FFE772
:109750000699486D40F010004865FFE70699002023
:1097600081F85000FFE701208DF81F0024E00698E3
:109770000068006800F04000402807D0FFE7069826
:109780000168086840F040000860FFE7FFE70699BD
:10979000002081F85000FFE706980168486840F013
:1097A0002000486006980168486840F00200486060
:1097B00000208DF81F00FFE79DF81F0008B080BD56
:1097C00080B584B002900191ADF80220029890F823
:1097D0005100012804D0FFE702208DF80F00A1E01E
:1097E000019820B1FFE7BDF8020020B9FFE7012092
:1097F0008DF80F0096E0FFE7029890F850000128DE
:1098000004D1FFE702208DF80F008BE002990120C0
:1098100081F85000FFE7FFE70299032081F851002B
:109820000299002048650199029A1163BDF802105F
:10983000029A9186BDF80210029AD1860299886335
:109840000299486402990864029988870299C88736
:1098500002988068B0F5004F0DD1FFE702980168CB
:10986000086820F04000086002980168086840F429
:1098700080400860FFE70298816C4CF6F920C0F642
:10988000000008640298816C4CF6CD30C0F60000F0
:10989000C8630298816C4CF6AD20C0F60000C86425
:1098A0000298816C00200865029B1A68196B986CFD
:1098B0000C32DB8EFDF7C0FE78B1FFE70299486DF0
:1098C00040F010004865FFE70299002081F8500041
:1098D000FFE701208DF80F0024E00298006800687F
:1098E00000F04000402807D0FFE7029801680868B0
:1098F00040F040000860FFE7FFE70299002081F890
:109900005000FFE702980168486840F02000486076
:1099100002980168486840F00200486000208DF815
:109920000F00FFE79DF80F0004B080BD80B582B046
:109930000190019803F0BAFA8DF803009DF8030036
:10994000022815D0FFE79DF80300410140F2445082
:10995000C2F20000405850B1FFE79DF803004101FA
:1099600040F24450C2F2000040588047FFE7FFE752
:1099700002B080BD80B582B00190019803F096FAE4
:109980008DF803009DF8030002281BD0FFE7019823
:1099900003F08CFA014640F24450C2F2000000EBA2
:1099A0004110C06868B1FFE7019803F07FFA0146F3
:1099B00040F24450C2F2000000EB4110C068804702
:1099C000FFE7FFE702B080BD80B582B0019001984B
:1099D00003F06CFA8DF803009DF8030002281BD0F9
:1099E000FFE7019803F062FA014640F24450C2F2E8
:1099F000000000EB4110806868B1FFE7019803F0B8
:109A000055FA014640F24450C2F2000000EB41100A
:109A100080688047FFE7FFE702B080BD80B582B075
:109A20000190019803F042FA8DF803009DF80300BD
:109A300002281BD0FFE7019803F038FA014640F2F4
:109A40004450C2F2000000EB4110406968B1FFE7EA
:109A5000019803F02BFA014640F24450C2F2000094
:109A600000EB411040698047FFE7FFE702B080BD8F
:109A700080B582B00190019804F016FC02B080BD60
:109A800080B582B00090009820B9FFE701208DF8E2
:109A900007003FE0009890F83D0040B9FFE70099CB
:109AA000002081F83C00009800F038F8FFE70099AA
:109AB000022081F83D00009951F8040B04F092FC5B
:109AC0000099012081F84600FFE70099012081F804
:109AD0003E00009981F83F00009981F8400000990C
:109AE00081F84100FFE7FFE70099012081F842007B
:109AF000009981F84300009981F84400009981F8A9
:109B00004500FFE70099012081F83D0000208DF815
:109B10000700FFE79DF8070002B080BD82B001900A
:109B20000198006844F20041C4F20101884212D158
:109B3000FFE7FFE70020009043F64400C4F2020074
:109B4000016841F400310160006800F400300090C9
:109B50000098FFE7FFE702B07047000080B588B0CB
:109B600007900020069005900490039002900798BB
:109B7000006844F20041C4F20101884222D1FFE7AB
:109B8000FFE70020019043F63000C4F202000168B4
:109B900041F020010160006800F020000190019870
:109BA000FFE74020029002200390002104910590DD
:109BB0000320069041F20040C4F2020002A9FDF722
:109BC0000FFEFFE708B080BD80B586B0049003911A
:109BD000029200208DF80700FFE7049890F83C00FF
:109BE000012804D1FFE702208DF8170089E00499CD
:109BF000012081F83C00FFE7FFE7029800900C2865
:109C000000F270800099DFE801F0076D6D6D206D46
:109C10006D6D3A6D6D6D530004980068039904F002
:109C2000CFFC04980168886940F0080088610498B6
:109C30000168886920F0040088610398026904982B
:109C4000016888691043886150E0049800680399AE
:109C500004F02CFD04980168886940F40060886174
:109C600004980168886920F480608861039802691B
:109C700004980168886940EA0220886136E0049807
:109C80000068039904F08CFD04980168C86940F0ED
:109C90000800C86104980168C86920F00400C86120
:109CA0000398026904980168C8691043C8611DE0FF
:109CB00004980068039904F0EDFD04980168C869F0
:109CC00040F40060C86104980168C86920F48060AD
:109CD000C8610398026904980168C86940EA0220D3
:109CE000C86103E001208DF80700FFE7FFE7049952
:109CF000002081F83C00FFE79DF807008DF8170071
:109D0000FFE79DF8170006B080BD000080B582B067
:109D10000090009820B9FFE701208DF807003FE090
:109D2000009890F83D0040B9FFE70099002081F8C5
:109D30003C00009800F038F8FFE70099022081F815
:109D40003D00009951F8040B04F04CFB00990120F0
:109D500081F84600FFE70099012081F83E00009954
:109D600081F83F00009981F84000009981F8410096
:109D7000FFE7FFE70099012081F84200009981F890
:109D80004300009981F84400009981F84500FFE7FD
:109D90000099012081F83D0000208DF80700FFE7C1
:109DA0009DF8070002B080BD81B0009001B07047FF
:109DB00080B58CB00A900991099828B9FFE70A98F4
:109DC00090F83E0007901CE00998042805D1FFE7B1
:109DD0000A9890F83F00069010E00998082805D1ED
:109DE000FFE70A9890F84000059004E00A9890F880
:109DF00041000590FFE705980690FFE70698079059
:109E0000FFE70798012804D0FFE701208DF82F0015
:109E1000AFE0099828B9FFE70A99022081F83E00CF
:109E20001EE00998042806D1FFE70A99022081F86C
:109E30003F00049012E00998082806D1FFE70A992C
:109E4000022081F84000039005E00A99022081F881
:109E500041000390FFE703980490FFE70498FFE7B1
:109E60000A98006809990122019204F08DFB01987B
:109E70000A9909680022C4F20102914202900CD0B2
:109E8000FFE70A9800684FF60041CBF6FE710844E0
:109E9000B0FA80F040090290FFE70298C00738B19D
:109EA000FFE70A980168486C40F400404864FFE707
:109EB0000A9800680021C4F2010188423CD0FFE703
:109EC0000A980068B0F1804F36D0FFE70A98006822
:109ED00040F20041C4F2000188422DD0FFE70A9809
:109EE000006840F60001C4F20001884224D0FFE778
:109EF0000A98006840F60041C4F2000188421BD075
:109F0000FFE70A98006840F20041C4F2010188426C
:109F100012D0FFE70A98006844F20001C4F2010180
:109F2000884209D0FFE70A98006841F60001C4F2B0
:109F30000001884212D1FFE70A980068806800F0AB
:109F4000070008900898062807D0FFE70A980168DC
:109F5000086840F001000860FFE706E00A98016821
:109F6000086840F001000860FFE700208DF82F002E
:109F7000FFE79DF82F000CB080BD000082B001907B
:109F8000ADF8021002B0704780B582B00190019820
:109F900005F01EFB8DF803009DF8030004281BD07C
:109FA000FFE79DF8030000EBC00140F26850C2F2E9
:109FB000000000EB8100006968B1FFE79DF8030035
:109FC00000EBC00140F26850C2F2000000EB8100DB
:109FD00000698047FFE7FFE702B080BD80B592B01F
:109FE0001190119800680068109011980068C0687E
:109FF0000F901198006840690E9000200D900C9011
:10A00000109800F00F000D900D9888B9FFE79DF8AB
:10A010004000800600280AD5FFE79DF83C00800636
:10A02000002804D5FFE7119805F004FB02E2FFE7E2
:10A030000D98002800F0C280FFE79DF83800C007A7
:10A0400038B9FFE7BDF83C0010F4907F00F0B6800F
:10A05000FFE79DF84000C00758B1FFE79DF83D00BD
:10A06000C00730B1FFE71199486C40F00100486427
:10A07000FFE79DF84000400700280BD5FFE79DF85B
:10A080003800C00730B1FFE71199486C40F002007A
:10A090004864FFE79DF84000800700280BD5FFE7E4
:10A0A0009DF83800C00730B1FFE71199486C40F0C7
:10A0B00004004864FFE79DF840000007002811D520
:10A0C000FFE79DF83C008006002805D4FFE79DF8D7
:10A0D0003800C00730B1FFE71199486C40F0080024
:10A0E0004864FFE71198406C002866D0FFE79DF8B0
:10A0F0004000800600280AD5FFE79DF83C00800656
:10A10000002804D5FFE7119805F094FAFFE71198AD
:10A1100000684069C0F380100C901198406C0007F3
:10A12000002804D4FFE70C9800283ED0FFE71198E0
:10A1300005F0D4F9119800684069400600282FD531
:10A14000FFE7FFE7FFE71198006850E8050F20F0F0
:10A1500040000B90FFE70B991198026842E8051048
:10A160000028F0D1FFE7FFE71198C06B98B1FFE737
:10A170001198C16B4FF21D30C0F6000008651198B0
:10A18000C06BFCF7EFFF28B1FFE71198C06B016DC2
:10A190008847FFE703E01198FFF7F6FEFFE703E0CB
:10A1A0001198FFF7F1FEFFE706E01198FFF7ECFECC
:10A1B000119900204864FFE7FFE73BE11198006B2D
:10A1C000012840F01781FFE79DF84000C0060028F5
:10A1D00040F11081FFE79DF83C00C006002840F1E7
:10A1E0000981FFE7FFE700200A90119800680068E6
:10A1F0000A901198006840680A900A98FFE7119841
:10A20000006840694006002840F19A80FFE71198F5
:10A21000C06B00684068ADF82600BDF82600002835
:10A2200075D0FFE7BDF826001199898D88426EDA56
:10A23000FFE7BDF826001199C8851198C06BC06969
:10A24000B0F5807F58D0FFE7FFE7FFE7119800687F
:10A2500050E8030F20F480700890FFE708991198E8
:10A26000026842E803100028F0D1FFE7FFE7FFE7AC
:10A27000FFE71198006850E8050F20F001000790F3
:10A28000FFE707991198026842E805100028F0D10D
:10A29000FFE7FFE7FFE7FFE71198006850E8050FC9
:10A2A00020F040000690FFE706991198026842E806
:10A2B00005100028F0D1FFE7FFE71199202081F871
:10A2C0004200119900200863FFE7FFE7119800683A
:10A2D00050E8030F20F010000590FFE70599119852
:10A2E000026842E803100028F0D1FFE7FFE7119869
:10A2F000C06BFCF7C1FEFFE711990220486311987B
:10A30000818DC28D891A89B2FFF738FE17E0BDF83A
:10A3100026001199898D884210D1FFE71198C06BF2
:10A32000C069B0F5807F08D1FFE71199022048632A
:10A330001198818DFFF722FEFFE7FFE7FFE779E045
:10A340001199888DC98D401AADF812001198C08DF1
:10A3500000284ED0FFE7BDF81200002849D0FFE7E3
:10A36000FFE7FFE71198006850E8030F20F49070B2
:10A370000390FFE703991198026842E80310002850
:10A38000F0D1FFE7FFE7FFE7FFE71198006850E82B
:10A39000050F20F001000290FFE702991198026872
:10A3A00042E805100028F0D1FFE7FFE711992020CF
:10A3B00081F84200119900200863FFE7FFE7119838
:10A3C000006850E8030F20F010000190FFE70199AA
:10A3D0001198026842E803100028F0D1FFE7FFE778
:10A3E0001199022048631198BDF81210FFF7C6FDBD
:10A3F000FFE71FE09DF84000000600280AD5FFE7B0
:10A400009DF83C000006002804D5FFE7119805F0F0
:10A41000FBFA0FE09DF84000400600280AD5FFE750
:10A420009DF83C004006002804D5FFE7119805F090
:10A430009FF8FFE712B080BD80B582B00090009811
:10A4400020B9FFE701208DF8070040E000988069FF
:10A4500008B1FFE700E0FFE7009890F8410040B93D
:10A46000FFE70099002081F84000009800F034F8E0
:10A47000FFE70099242081F8410000980168C8682E
:10A4800020F40050C860009805F088F90098016831
:10A49000086920F49040086100980168486920F03C
:10A4A0002A00486100980168C86840F40050C860FC
:10A4B000009900204864009A202182F84110009AF7
:10A4C00082F84210009948638DF80700FFE79DF875
:10A4D000070002B080BD000080B59CB01B9000203A
:10A4E0001A9019901890179016901B98006841F2D6
:10A4F0000001C4F20101884240F09380FFE7FFE7CA
:10A500000020159043F64400C4F20200016841F0B7
:10A5100010010160006800F0100015901598FFE729
:10A52000FFE70020149043F63000C4F202000168F7
:10A5300041F002010160006800F0020014901498DC
:10A54000FFE7FFE70020139043F63000C4F202005B
:10A55000016841F001010160006800F00100139002
:10A560001398FFE780201690022009901790002092
:10A570000D90189003200A90199007200B901A90C4
:10A5800040F20040C4F2020016A90C91FDF728F930
:10A59000DDF824C00A9A0B980C990D9B4FF4007EAD
:10A5A000CDF858E0CDF85CC0189319921A900020AD
:10A5B000C4F20200FDF714F90D9941F2DC10C2F269
:10A5C00000000E9046F28842C4F2020202604FF090
:10A5D000006242608160C1604FF48062026141614B
:10A5E0008161C1614FF4403202624162FCF76CFF4D
:10A5F00018B1FFE7FAF7A2FFFFE7FFE71B9841F268
:10A60000DC11C2F20001C1631B988863FFE72520BB
:10A61000089005210022FDF797FB0898FDF78AFBBB
:10A6200014E11B98006844F60001C4F2000188425E
:10A630006AD1FFE7FFE70020129043F64000C4F222
:10A640000200016841F480210160006800F480206C
:10A6500012901298FFE7FFE70020119043F63000B8
:10A66000C4F20200016841F004010160006800F0DA
:10A67000040011901198FFE74FF4406016900220FB
:10A6800017900020069018900320199007201A9028
:10A6900040F60000C4F2020016A9FDF7A1F80699E1
:10A6A00041F23C20C2F20000079046F22802C4F2B8
:10A6B000020202604FF0006242608160C1604FF4AC
:10A6C00080620261416181614FF48072C261016206
:10A6D0004162FCF7F9FE18B1FFE7FAF72FFFFFE739
:10A6E000FFE71B9841F23C21C2F20001C1631B98B5
:10A6F0008863FFE72720059005210022FDF724FB52
:10A700000598FDF717FBA0E01B98006841F2004197
:10A71000C4F20101884240F09780FFE7FFE7002084
:10A72000109043F64400C4F20200016841F0200199
:10A730000160006800F0200010901098FFE7FFE72C
:10A7400000200F9043F63000C4F20200016841F08F
:10A7500040010160006800F040000F900F98FFE793
:10A760004FF4844016900220179000200390189018
:10A770000320199008201A9041F60000C4F202004C
:10A7800016A9FDF72DF8039941F29C20C2F20000B2
:10A79000049046F22842C4F2020202604FF02062A6
:10A7A00042608160C1604FF48062026141618161F9
:10A7B000C1614FF4803202624162FCF785FE18B13C
:10A7C000FFE7FAF7BBFEFFE7FFE71B9841F29C218A
:10A7D000C2F20001C1631B988863FFE741F2FC20CD
:10A7E000C2F20000029046F2A041C4F202010160F0
:10A7F0004FF020614160402181600021C1604FF431
:10A800008062026141618161C1614FF48032026204
:10A810004162FCF759FE18B1FFE7FAF78FFEFFE738
:10A82000FFE71B9841F2FC21C2F2000181631B98F3
:10A830008863FFE74720019005210022FDF784FA95
:10A840000198FDF777FAFFE7FFE7FFE71CB080BD4F
:10A8500080B584B002900191ADF80220029890F882
:10A860004200202817D1FFE7019820B1FFE7BDF88B
:10A87000020020B9FFE701208DF80F000FE00299D8
:10A880000020086302980199BDF8022005F024F821
:10A890008DF80F0003E002208DF80F00FFE79DF810
:10A8A0000F0004B080BD000080B582B00190019817
:10A8B00004F08EFE8DF803009DF8030004281BD0E1
:10A8C000FFE79DF8030000EBC00140F26850C2F2C0
:10A8D000000000EB8100C06868B1FFE79DF803004D
:10A8E00000EBC00140F26850C2F2000000EB8100B2
:10A8F000C0688047FFE7FFE702B080BD80B582B047
:10A900000190019804F064FE8DF803009DF80300A7
:10A9100004281BD0FFE79DF8030000EBC00140F2C4
:10A920006850C2F2000000EB8100806868B1FFE768
:10A930009DF8030000EBC00140F26850C2F2000035
:10A9400000EB810080688047FFE7FFE702B080BD31
:10A9500080B582B00190019804F03AFE8DF80300B2
:10A960009DF8030004281BD0FFE79DF8030000EBCF
:10A97000C00140F26850C2F2000000EB8100406864
:10A9800068B1FFE79DF8030000EBC00140F268509A
:10A99000C2F2000000EB810040688047FFE7FFE75C
:10A9A00002B080BDFFE7FEE784B08DED030A9DEDA8
:10A9B000030AB6EE001A20EE010A8DED020A039892
:10A9C000019001980090009945F6DF10C5F63770A8
:10A9D000A0EB61000090009801909DED010A9DEDB3
:10A9E000021A21EE001A21EE002AB7EE081A31EE03
:10A9F000422A20EE020A8DED010A9DED010A9DED2D
:10AA0000022A22EE002A22EE002A31EE421A20EE1D
:10AA1000010A8DED010A9DED010A04B070470000A6
:10AA200083B0ADF80A00BDF90A0040F26111884216
:10AA300003D1FFE70120019015E0BDF90A00B0F550
:10AA4000806F03D1FFE70320009009E0BDF90A0001
:10AA5000A0F29F60B0FA80F0400940000090FFE74C
:10AA600000980190FFE70198C0B203B07047000062
:10AA700080B586B004908DED030A049818B9FFE7FD
:10AA8000002005904CE09DED030A049890ED014AEA
:10AA900090ED022A90ED063A90ED071A23EE043A63
:10AAA00030EE430A21EE021A30EE410A8DED020A21
:10AAB000002028B9FFE7029805F06EF858B90DE0BC
:10AAC00002980DF0A1F841EC100B51EC100B05F0C1
:10AAD00049F818B1FFE703980290FFE79DED020ADD
:10AAE000049890ED034A90ED043A90ED052A90ED1C
:10AAF000061A20EE040A21EE031A30EE010A90ED48
:10AB0000071A21EE021A30EE010A8DED010A0499AE
:10AB10008869C86102980499886101980590FFE7E7
:10AB20009DED050A06B080BD80B588B007908DED1B
:10AB3000060ACDED050A079808B9FFE78BE00598EE
:10AB4000079908600799002088610799C8610798EC
:10AB500090ED000AB5EE400AF1EE10FA0EDCFFE7C8
:10AB600007994FF07E50C860079900200861079947
:10AB7000486107994860079988606CE09DED060A76
:10AB8000079890ED001A80EE010A8DED040A9DED04
:10AB9000041A9FED320A80EE010A0BF0D7FA8DED10
:10ABA000030A9FED2F0A8DED000A0AF009FAB0EEB4
:10ABB000401A9DED000A31EE011A9DED033A21EE97
:10ABC000031AB7EE002A8DED012A31EE021A23EEA8
:10ABD000033A31EE031A8DED021A9DED031A21EEB0
:10ABE000011A9DED023A81EE031A079880ED031ACF
:10ABF000079890ED031A31EE011A80ED041A0799B7
:10AC0000C86848619DED031A21EE011A31EE421A1F
:10AC100031EE011A9DED022A81EE021A079880EDAD
:10AC2000011A0AF0CDF9B0EE401A9DED010A31EE9D
:10AC3000012A9DED031A22EE012A30EE420A21EE8E
:10AC4000011A30EE010A9DED021A80EE010A079802
:10AC500080ED020AFFE708B080BD00BFDB0F49406E
:10AC6000DB0F493F80B584B002908DED010A029858
:10AC700018B9FFE70020039039E09DED010A029822
:10AC800090ED031A90ED043A90ED052A31EE031A87
:10AC900031EE021A80EE010A8DED000A002028B97B
:10ACA000FFE7009804F046FF58B911E000980CF057
:10ACB000ABFF41EC100B51EC100B04F01BFF38B153
:10ACC000FFE700980299886100980299C86106E040
:10ACD00001980299886101980299C861FFE702987A
:10ACE0009DED010AFFF7C4FE8DED030AFFE79DED20
:10ACF000030A04B080BD000080B582B08DF8060064
:10AD00009DF80600022804DBFFE7FF208DF807000E
:10AD100039E09DF8061040F25460C2F2000050F88D
:10AD2000210020B1FFE700208DF807002BE08820EC
:10AD3000F8F716F901469DF8062040F25460C2F279
:10AD4000000040F822109DF8061050F8210020B9AC
:10AD5000FFE7FF208DF8070015E09DF8061040F290
:10AD60005460C2F20000009050F821008821F5F7ED
:10AD7000B2FB00999DF8060051F8201008700020E1
:10AD80008DF80700FFE79DF9070002B080BD0000C5
:10AD900080B588B00690069820B9FFE7FE208DF8B0
:10ADA0001F002EE0069800F049F80590059820B99C
:10ADB000FFE7FC208DF81F0023E0059880880190B4
:10ADC00008208DF80800FF208DF809008DF80A0092
:10ADD0008DF80B008DF80C008DF80D008DF80E002D
:10ADE0008DF80F00FC208DF810000598007801A95F
:10ADF000F7F762FE002818BF4FF0FF308DF81F00F4
:10AE0000FFE79DF91F0008B080BD000082B08DF8FB
:10AE100003009DF80300022803DBFFE700200190F8
:10AE200009E09DF8031040F25460C2F2000050F8AF
:10AE300021000190FFE7019802B0704780B586B00D
:10AE40000490049818B9FFE70020059036E00498B4
:10AE50000078FFF7DBFF0390039818B9FFE70020A5
:10AE600005902BE000200290FFE70298039991F8EB
:10AE7000841088421FDAFFE70398029900EB8100F3
:10AE800040680190019888B1FFE701980078049923
:10AE9000097888420AD1FFE70198408804994988D7
:10AEA000884203D1FFE70198059007E0FFE7029889
:10AEB00001300290D9E700200590FFE7059806B021
:10AEC00080BD000080B584B002900191029818B155
:10AED000FFE7019820B9FFE7FE208DF80F0011E091
:10AEE0000298FFF7ABFF0090009820B9FFE7FC2025
:10AEF0008DF80F0006E00098019900F049F98DF8EF
:10AF00000F00FFE79DF90F0004B080BD80B586B04B
:10AF100004900391049818B1FFE7039820B9FFE764
:10AF2000FE208DF8170090E003984178807840EA81
:10AF30000120ADF80A00BDF80A009FED460ADFEDDA
:10AF4000460A102106F0DAFF049880ED070A0399FB
:10AF5000C8780979000140EA1110ADF80800BDF881
:10AF60000800BBEE0E0AF3EE0E0A0C21009106F06B
:10AF7000C5FF0099049880ED080A0398027940798A
:10AF800002F00F0240EA0220ADF80600BDF806000C
:10AF9000BAEE080AF2EE080A06F0B0FF049880ED57
:10AFA000090A0398807900EE100AB8EE400A049866
:10AFB00080ED0A0AFFE7049890ED070AB5EE400A13
:10AFC000F1EE10FA0ADAFFE7049890ED070A9FED18
:10AFD000231A30EE010A80ED070AECE7FFE7049838
:10AFE00090ED070A9FED1D1AB4EE410AF1EE10FA3A
:10AFF0000ADBFFE7049890ED070A9FED191A30EE7F
:10B00000010A80ED070AEAE70498C079C007C0B1D9
:10B01000FFE7049890ED071A9FED100A30EE410A01
:10B0200080ED070A049890ED080AB1EE400A80ED21
:10B03000080A049890ED090AB1EE400A80ED090A69
:10B04000FFE700208DF81700FFE79DF9170006B015
:10B0500080BD00BFDA0F49C1DA0F4941DB0FC9409B
:10B06000DB0FC9C080B586B00490049820B9FFE713
:10B07000FE208DF8170087E004980078FFF73CFE6B
:10B0800020B1FFE7FF208DF817007DE004980078DD
:10B09000FFF7BCFE0390039820B9FFE7FF208DF86F
:10B0A000170071E000200290FFE70298039991F8E1
:10B0B000841088421BDAFFE70398029900EB8100B5
:10B0C000406878B1FFE70398029900EB810040687F
:10B0D000408804994988884204D1FFE7FD208DF813
:10B0E000170051E0FFE7029801300290DDE7039876
:10B0F00090F88400202804DBFFE7FF208DF817007C
:10B1000042E03020F7F72CFF0190019820B9FFE7CB
:10B11000FF208DF8170037E001983021F5F7DBF9B3
:10B120000199049A106852684A60086001990020E9
:10B1300008720498C079019900F00100087604981B
:10B140004088ADF8020004980078BDF80210032290
:10B15000F7F7F0FA38B1FFE70198F7F703FEFF20A1
:10B160008DF8170010E00198039991F8842001EB05
:10B1700082014860039991F88400013081F88400CD
:10B1800000208DF81700FFE79DF9170006B080BD7D
:10B1900080B58EB00C900B910C9818B1FFE70B980E
:10B1A00020B9FFE7FE208DF8370087E00C988088F3
:10B1B000ADF818000B9890ED020ADFED420A9FED02
:10B1C000421A102004F05CFFADF822000B9890EDBD
:10B1D000010AFBEE0E0AB3EE0E1A0C20019004F0E9
:10B1E0004FFF01460198ADF820100B9991ED030A2D
:10B1F000DFED360ACDED000A9FED351A04F040FF71
:10B20000DDED000A01460198ADF81E100B9991ED95
:10B21000040AB1EE041A04F033FF01460198ADF8B8
:10B220001C100B9991ED000AFAEE080AB2EE081A0A
:10B2300004F026FFADF81A009DF823008DF82400D5
:10B240009DF822008DF82500BDF8200000098DF83A
:10B250002600BDF820109DF81F0040EA01108DF86F
:10B2600027009DF81E008DF82800BDF81C0000097D
:10B270008DF82900BDF81C109DF81B0040EA011054
:10B280008DF82A009DF81A008DF82B000C98808804
:10B29000029008208DF80C0009980A99CDF8111039
:10B2A000CDF80D000C98007802A9F7F705FC0028EE
:10B2B00018BF4FF0FF308DF83700FFE79DF93700DA
:10B2C0000EB080BDDA0F49C1DA0F4941000000001D
:10B2D0000000FA4380B590B00E900E9820B9FFE7B9
:10B2E000FE208DF83F0077E00E980078FFF78EFD86
:10B2F0000D900D9820B9FFE7FC208DF83F006BE022
:10B3000000200C900B90FFE70B980D9991F884109A
:10B3100088421EDAFFE70D980B9900EB8100406828
:10B3200090B1FFE70D980B9900EB810040684088D1
:10B330000E994988884207D1FFE70D980B9900EBD9
:10B34000810040680C9004E0FFE70B9801300B90FF
:10B35000DAE70C9820B9FFE7FC208DF83F003BE0CE
:10B360000E984088ADF82A000E980078BDF82A1093
:10B3700003AA0023F7F770F8E0B1FFE7F7F7B8FF8B
:10B3800001910090009901980C9A13695269C91AA9
:10B39000904148F2A162C0F20102891A70F10000E6
:10B3A00004D3FFE70C9900200872FFE7FF208DF817
:10B3B0003F0011E00C9901200872F7F799FF0A4647
:10B3C0000C994A6108610C9803A90D31FFF79EFDA5
:10B3D00000208DF83F00FFE79DF93F0010B080BDD1
:10B3E00082B00090009820B9FFE74FF040400190F4
:10B3F00003E0009840690190FFE79DED010A02B06B
:10B400007047000082B00090009820B9FFE74FF02D
:10B410004040019003E0009880690190FFE79DEDB6
:10B42000010A02B07047000080B582B08DF80600B6
:10B430009DF80600022804DBFFE7FF208DF80700D7
:10B4400039E09DF8061040F25C60C2F2000050F84E
:10B45000210020B1FFE700208DF807002BE04820F5
:10B46000F7F77EFD01469DF8062040F25C60C2F2CF
:10B47000000040F822109DF8061050F8210020B975
:10B48000FFE7FF208DF8070015E09DF8061040F259
:10B490005C60C2F20000009050F821004821F5F7EE
:10B4A0001AF800999DF8060051F820100870002045
:10B4B0008DF80700FFE79DF9070002B080BD00008E
:10B4C00080B58EB00C900C9820B9FFE7FE208DF867
:10B4D0003700A9E00C98007800F0AAF80B900B98C0
:10B4E00020B9FFE7FC208DF837009DE00B98023073
:10B4F0000A900C984088ADF81600BDF81610A1F21D
:10B500000120019104280CD3FFE70198A0F2052047
:10B51000042829D3FFE70198A0F20920032849D382
:10B5200072E04FF40070069008208DF81C00002097
:10B530000490FFE70498032815DCFFE70A98049AB3
:10B5400000EB4200407806A9053101F812000A9884
:10B55000049A30F8120001EB42014870FFE70498AA
:10B5600001300490E6E753E040F2FF100690082017
:10B570008DF81C0004200390FFE70398072818DCCF
:10B58000FFE70A98039A00EB4200407806A90531CC
:10B5900001EB420202F8080C0A98039A30F81200F4
:10B5A00001EB420101F8070CFFE70398013003901B
:10B5B000E3E72DE040F2FF20069008208DF81C0004
:10B5C0000290FFE702980A2818DCFFE70A98029A1F
:10B5D00000EB4200407806A9053101EB420202F877
:10B5E000100C0A98029A30F8120001EB420101F89F
:10B5F0000F0CFFE7029801300290E3E700208DF87E
:10B6000023008DF8240003E0FF208DF837000BE0C5
:10B610000C98007806A9F7F74FFA002818BF4FF0EA
:10B62000FF308DF83700FFE79DF937000EB080BD81
:10B6300082B08DF803009DF80300022803DBFFE7CA
:10B640000020019009E09DF8031040F25C60C2F216
:10B65000000050F821000190FFE7019802B0704708
:10B6600082B08DF805009DF805000146009140B1BB
:10B67000FFE70098012809D0FFE7009802280AD0C8
:10B680000EE042F21070ADF806000EE04FF480407C
:10B69000ADF8060009E047F23050ADF8060004E0CE
:10B6A0004FF6FF70ADF80600FFE7BDF9060002B0E7
:10B6B0007047000083B0ADF808008DF807109DF8C2
:10B6C000070001460091022804D3FFE700980228F2
:10B6D00013D025E0BDF80800B0F5007F0CDDFFE7D2
:10B6E000BDF80800B0F5027F06DCFFE7BDF80800F2
:10B6F00001388DF80B0018E013E0BDF80800B0F534
:10B70000017F0CDDFFE7BDF80800B0F5037F06DA26
:10B71000FFE7BDF8080001388DF80B0005E000E0F8
:10B72000FFE7FF208DF80B00FFE79DF90B0003B04A
:10B730007047000080B586B00490049818B9FFE700
:10B74000002005902FE004980078FFF771FF039028
:10B75000039818B9FFE70020059024E0002002902C
:10B76000FFE70298039991F84410884218DAFFE73E
:10B770000398029900EB810080690190019850B113
:10B78000FFE70198408804994988884203D1FFE780
:10B790000198059007E0FFE7029801300290E0E78A
:10B7A00000200590FFE7059806B080BD83B08DF8B6
:10B7B00007009DF807000146009140B1FFE700989F
:10B7C000012809D0FFE7009802280BD00EE00020E6
:10B7D000C4F2102002900DE04AF22C00C4F299103D
:10B7E000029007E04FF07E50029003E04FF07E5051
:10B7F0000290FFE79DED020A03B0704780B586B066
:10B800000490049820B9FFE7FE208DF8170081E02E
:10B8100004980078FFF708FE20B1FFE7FF208DF8BD
:10B82000170077E004980078FFF702FF0390039871
:10B8300020B9FFE7FF208DF817006BE00020029091
:10B84000FFE70298039991F8441088421BDAFFE75A
:10B850000398029900EB8100806978B1FFE70398B3
:10B86000029900EB810080694088049949888842E8
:10B8700004D1FFE7FD208DF817004BE0FFE70298A9
:10B8800001300290DDE7039890F844000B2804DBB8
:10B89000FFE7FF208DF817003CE05020F7F760FB32
:10B8A0000190019820B9FFE7FF208DF8170031E0E3
:10B8B0000199049A106852684A600860019818302B
:10B8C0002821F4F708FE04984079019900F001005E
:10B8D00081F828000499087849880322F6F72AFF9E
:10B8E00038B1FFE70198F7F73DFAFF208DF8170010
:10B8F00010E00198039991F8442001EB82018861DE
:10B90000039991F84400013081F8440000208DF83B
:10B910001700FFE79DF9170006B080BD80B582B023
:10B92000019001989FED020A00F004F802B080BD7A
:10B930000000000080B58AB007A901910146019876
:10B94000089180ED000A089820B9FFE7FE208DF8E5
:10B95000270078E008980078FFF76AFE06900698BE
:10B9600020B9FFE7FC208DF827006CE0019890EDEE
:10B97000000AB7EE001AB4EE410AF1EE10FA04DD47
:10B98000FFE74FF07E500790FFE7019890ED000A27
:10B99000BFEE001AB4EE410AF1EE10FA05DAFFE745
:10B9A0000020CBF680700790FFE708984079C00729
:10B9B00040B1FFE7019890ED000AB1EE400A80ED3A
:10B9C000000AFFE70898FFF7B5FE0590059820B933
:10B9D000FFE7FC208DF8270035E0089948880979B1
:10B9E000FFF768FE8DF813009DF91300B0F1FF3FDB
:10B9F00004DCFFE7FF208DF8270024E0019806997A
:10BA00000231039190ED000A8DED000A089800794B
:10BA1000FFF726FE9DED000A01EE100AB8EEC11AEE
:10BA200020EE010ABDEEC00A10EE100AADF80A00C1
:10BA3000BDF80A0003999DF9132021F81200002097
:10BA40008DF82700FFE79DF927000AB080BD0000B0
:10BA500080B590B00E900E9820B9FFE7FE208DF8CB
:10BA60003F0072E00E980078FFF7E2FD0D900D9810
:10BA700020B9FFE7FC208DF83F0066E000200C9025
:10BA8000FFE70C980D9991F84410884259DAFFE7C6
:10BA90000D980C9900EB810080690B900B980028A1
:10BAA0004AD0FFE70B9840880E994988884243D1D5
:10BAB000FFE70E990878498804AA0023F6F7CCFC22
:10BAC000E8B1FFE7F7F714FC03910290029903989D
:10BAD0000B9A136A526AC91A904140F2E932891AE4
:10BAE00070F1000007D3FFE70B9900200876FC20D7
:10BAF0008DF83F0029E0FF208DF83F0025E00B99ED
:10BB000001200876F7F7F4FB0A460B994A620862AF
:10BB10000B9804A900F0F8FA0B9901918868CA689B
:10BB20000B69D1F814C0C1F838C04B630A63C8620E
:10BB300000208DF83F0008E0FFE70C9801300C90E2
:10BB40009FE7FC208DF83F00FFE79DF93F0010B014
:10BB500080BD000080B586B000208DF817000490ED
:10BB6000FFE70498012830DCFFE79DF81000FFF79D
:10BB70005FFD0390039808B9FFE722E000200290E0
:10BB8000FFE70298039991F84410884218DAFFE71A
:10BB90000398029900EB810080690190019850B1EF
:10BBA000FFE70198FFF754FF20B1FFE7FF208DF872
:10BBB0001700FFE7FFE7FFE7029801300290E0E798
:10BBC000FFE7049801300490CBE79DF9170006B019
:10BBD00080BD000080B582B041F2CC00C2F200000E
:10BBE000019046F20041C4F200010160032141606E
:10BBF00000218160C1604FF4A02202614FF4C002B5
:10BC000042610176417681760122C27601774177E1
:10BC1000FAF748FE18B1FFE7F9F790FCFFE702B02A
:10BC200080BD000080B582B041F2F400C2F2000095
:10BC3000019046F60001C4F2000101600321416059
:10BC400000218160C1604FF4A02202614FF4C00264
:10BC500042610176417681760122C2760177417791
:10BC6000FAF720FE18B1FFE7F9F768FCFFE702B02A
:10BC700080BD000080B58AB0FFE70020099043F640
:10BC80003000C4F20200016841F4800101600068E4
:10BC900000F4800009900998FFE7FFE70020089072
:10BCA00043F63000C4F20200016841F40011016063
:10BCB000006800F4001008900898FFE70C2000903E
:10BCC0000521059100220692FCF73EF80098FCF74A
:10BCD00031F80599069A39200190FCF735F801985A
:10BCE000FCF728F80599069A3A200290FCF72CF800
:10BCF0000298FCF71FF80599069A3B200390FCF781
:10BD000023F80398FCF716F80599069A4420049046
:10BD1000FCF71AF80498FCF70DF80599069A4520E7
:10BD20000790FCF711F80798FCF704F80AB080BDFB
:10BD300080B582B04EF29520C0F6000048F29C22F9
:10BD4000C0F601020021019104F0B4FE019940F611
:10BD50004C52C2F2000210604EF63910C0F60000DC
:10BD600048F22022C0F6010204F0A4FE02B080BD19
:10BD700080B59AB0002019901890179016901590E1
:10BD8000FFE70020149043F63000C4F2020001687F
:10BD900041F002010160006800F002001490149864
:10BDA000FFE7FFE70020139043F63000C4F20200E3
:10BDB000016841F040010160006800F0400013900C
:10BDC0001398FFE7FFE70020129043F63000C4F21B
:10BDD0000200016841F001010160006800F001000B
:10BDE00012901298FFE7FFE70020119043F6300011
:10BDF000C4F20200016841F008010160006800F02F
:10BE0000080011901198FFE7FFE70020109043F61B
:10BE10003000C4F20200016841F0040101600068D2
:10BE200000F0040010901098FFE7FFE700200F904B
:10BE300043F63000C4F20200016841F08001016065
:10BE4000006800F080000F900F98FFE7FFE70020E8
:10BE50000E9043F63000C4F20200016841F0200168
:10BE60000160006800F020000E900E98FFE741F698
:10BE70000040C4F2020002904FF4E0510191002210
:10BE80000C92FBF7A1FE0020C4F2020004901021E6
:10BE9000039101220692FBF797FE069A40F20040BA
:10BEA000C4F2020007901146FBF78EFE019B029838
:10BEB000069A0C991593169217910221189115A9BB
:10BEC0000891FBF78DFC0498069A089915924FF497
:10BED0008813059316931792FBF782FC039B049833
:10BEE000069A08991593169217921892FBF778FC08
:10BEF000059A06980899302315931692179040F6E4
:10BF00000000C4F20200FBF76BFC069A0798089940
:10BF10001592169217921892FBF762FC0C9A062063
:10BF2000099005210B91FBF70FFF0998FBF702FF22
:10BF30000B990C9A0A200A90FBF706FF0A98FBF768
:10BF4000F9FE0B990C9A17200D90FBF7FDFE0D984A
:10BF5000FBF7F0FE1AB080BD80B582B041F25C30D4
:10BF6000C2F20000019043F20001C4F2010101603D
:10BF70004FF48271416000218160C1600161012242
:10BF800042614FF4007282611822C2610162416213
:10BF900081620A21C162FCF753FC18B1FFE7F9F78F
:10BFA000CDFAFFE702B080BD80B588B000210091D6
:10BFB000079106910591049103910291019141F23B
:10BFC000B430C2F2000044F20042C4F20102026046
:10BFD0004160816041F28732C26001618161FDF799
:10BFE0004FFD18B1FFE7F9F7A9FAFFE741F2B430C6
:10BFF000C2F20000FDF78AFE18B1FFE7F9F79EFADA
:10C00000FFE760200190002202920392059241F224
:10C01000B430C2F2000001A9FDF7D6FD18B1FFE768
:10C02000F9F78CFAFFE741F2B430C2F20000FDF7F5
:10C0300095FD08B080BD000080B582B041F2FC30B3
:10C04000C2F20000019041F20001C4F2010101605E
:10C050004FF4E131416000218160C16001610C2237
:10C0600042618161C161FEF7E7F918B1FFE7F9F7B5
:10C0700065FAFFE702B080BD80B582B041F244406E
:10C08000C2F20000019044F60001C4F20001016018
:10C0900048F2A061C0F2010141604FF4805181601B
:10C0A0000021C1604FF4806202610C224261816113
:10C0B000C161FEF7C1F918B1FFE7F9F73FFAFFE7F1
:10C0C00002B080BD80B582B041F28C40C2F2000067
:10C0D000019041F20041C4F2010101604FF4E131ED
:10C0E000416000218160C16001610C224261816177
:10C0F000C161FEF7A1F918B1FFE7F9F71FFAFFE7F1
:10C1000002B080BDFFE7FEE780B58AB009900891D4
:10C110000898417B807B40EA0120ADF81E0008981A
:10C12000C17B007C40EA0120ADF81C000898417CEE
:10C13000807C40EA0120ADF81A0009980079FFF7E9
:10C140008FFAADF8180009980079FFF72FFB8DEDF5
:10C15000050ABDF81E0000EE100AB8EEC00A9FEDF9
:10C160006D1A80EE010A9FED6C1A20EE010A8DED2A
:10C17000040ABDF91C0000EE100AB8EEC00A8DEDED
:10C18000030ABDF91A00BDF91810484300EE100A61
:10C19000B8EEC00A9FED611A80EE010A8DED020A29
:10C1A00009988079C00700284CD0FFE7BDF81E0031
:10C1B0000999B1F84010401A01900198B0F5805FDC
:10C1C00005DDFFE70999486C013848640AE00198E9
:10C1D00010F5805F05DAFFE70999486C0130486483
:10C1E000FFE7FFE7BDF81E000999A1F84000049899
:10C1F0000090099890ED110AB8EEC00A9FED461A1A
:10C2000020EE010A9DED001A30EE010A9DED051A9F
:10C2100080EE010A80ED120A0999886C88609DED14
:10C22000030A9DED051A80EE010A099880ED030AC4
:10C230009DED020A9DED051A20EE010A099880ED98
:10C24000040A13E0099900204864BDF81E10099AF9
:10C25000A2F84010099988640498099988600398A5
:10C260000999C860029809990861FFE7FFE70998F2
:10C2700090ED020AB5EE400AF1EE10FA0ADAFFE795
:10C28000099890ED020A9FED241A30EE010A80ED24
:10C29000020AECE7FFE7099890ED020A9FED1E1AEB
:10C2A000B4EE410AF1EE10FA0ADBFFE7099890EDCF
:10C2B000020A9FED1B1A30EE010A80ED020AEAE73E
:10C2C000099890F82800C007C0B1FFE7099890EDE1
:10C2D000021A9FED110A30EE410A80ED020A099818
:10C2E00090ED030AB1EE400A80ED030A099890ED43
:10C2F000040AB1EE400A80ED040AFFE70898C07C0A
:10C3000000EE100AB8EE400A099880ED050A0AB05E
:10C3100080BD00BF00000046DB0FC9400000804622
:10C32000DB0FC9C0FFE7FEE788B0079006910592D2
:10C33000079800F0070004900498C0F10700052852
:10C3400003D3FFE70420019004E00498C0F1070044
:10C350000190FFE70198039004980430062803D861
:10C36000FFE70020009003E0049803380090FFE707
:10C370000098029006980399012202FA01F101390E
:10C380000840029B984005999A40013A11400843A1
:10C3900008B0704780B590B00E908DED0D0ACDEDD0
:10C3A0000C0A8DED0B1ACDED0A1A002028B9FFE713
:10C3B0000D9803F0CBFB58B943E00D980BF024FC2B
:10C3C00041EC100B51EC100B03F0A4FBC8B3FFE7DA
:10C3D000002028B9FFE70C9803F0B8FB58B930E00B
:10C3E0000C980BF011FC41EC100B51EC100B03F00E
:10C3F00091FB30B3FFE7002028B9FFE70B9803F06B
:10C40000A5FB58B91DE00B980BF0FEFB41EC100B9F
:10C4100051EC100B03F07EFB98B1FFE7002028B928
:10C42000FFE70A9803F092FB78B90AE00A980BF04C
:10C43000EBFB41EC100B51EC100B03F06BFB20B944
:10C44000FFE70E9880690F9016E19DED0D0ADDED76
:10C450000C0A0E98406890ED071AF8F73DFD8DED37
:10C46000090A9DED090A0E98406890ED001A20EE29
:10C47000010A8DED080A0E98406890ED000A9DEDC6
:10C480000C1A20EE010A8DED070A0E981C309DED66
:10C49000070AFEF7EDFA8DED060A0E9800780146C0
:10C4A000019110B3FFE70198012804D0FFE701983C
:10C4B000022817D01CE09DED060A0E9890ED021A96
:10C4C00090ED052A30EE420A9DED0A2AB4EE412A8B
:10C4D000F1EE10FAC8BFB0EE421A80EE010A8DEDFF
:10C4E000050A05E00B98059002E000200590FFE7A3
:10C4F00009980E99086106980E994861002028B99C
:10C50000FFE7059803F022FB70B90AE005980BF0ED
:10C510007BFB41EC100B51EC100B03F0FBFA18B94C
:10C52000FFE700200590FFE79DED080A0E984068A0
:10C5300090ED011A90ED032A20EE010A9DED051AF7
:10C5400021EE021A30EE410A8DED040A0E9890EDAC
:10C55000030A9DED081A9DED0A2A21EE021A30EE1B
:10C56000010A8DED030A9DED030A0E98406890EDD7
:10C57000021A20EE010A8DED020A0E98406890ED35
:10C58000020A9FED3F1AB4EE410AF1EE10FA39DDCE
:10C59000FFE7002028B9FFE7039803F0D7FA58B95E
:10C5A0002FE003980BF030FB41EC100B51EC100B1B
:10C5B00003F0B0FA28B3FFE79DED040A9DED021ADF
:10C5C00030EE010AB0EEC00A0E98406890ED051AF0
:10C5D000B4EE410AF1EE10FA12DCFFE79DED030A1A
:10C5E000B0EEC00A0E98406890ED041AB4EE410A0D
:10C5F000F1EE10FA04DCFFE703980E99C860FFE73C
:10C60000FFE7FFE79DED021A9DED040A30EE010AF7
:10C610008DED040A002028B9FFE7049803F096FA8C
:10C6200058B925E004980BF0EFFA41EC100B51ECEF
:10C63000100B03F06FFAD8B1FFE70E98406890ED49
:10C64000050A9FED0F1AB4EE410AF1EE10FA0BDD68
:10C65000FFE79DED040A0E984068D0ED050AF5F756
:10C6600099FA8DED040AFFE704980E998861FFE7B7
:10C670000E9880690F90FFE79DED0F0A10B080BD06
:10C68000BD37863580B586B004908DF80F108DEDDE
:10C69000020A0192049820B9FFE7FF208DF81700E5
:10C6A000B7E0002030B9FFE70198406803F04EFA88
:10C6B00080B90BE0019840680BF0A6FA41EC100B32
:10C6C00051EC100B03F026FA20B9FFE7FF208DF89C
:10C6D00017009EE0002030B9FFE70198806803F062
:10C6E00035FA80B90BE0019880680BF08DFA41ECC7
:10C6F000100B51EC100B03F00DFA20B9FFE7FF20EF
:10C700008DF8170085E0002030B9FFE70198C06878
:10C7100003F01CFA80B90BE00198C0680BF074FAC2
:10C7200041EC100B51EC100B03F0F4F920B9FFE7CA
:10C73000FF208DF817006CE0002030B9FFE701986A
:10C74000006903F003FA80B90BE0019800690BF06F
:10C750005BFA41EC100B51EC100B03F0DBF920B944
:10C76000FFE7FF208DF8170053E0002030B9FFE706
:10C770000198406903F0EAF980B90BE0019840693B
:10C780000BF042FA41EC100B51EC100B03F0C2F924
:10C7900020B9FFE7FF208DF817003AE001980499CF
:10C7A00048609DED021AB7EE000A80EE010A8DED99
:10C7B000000A002028B9FFE7009803F0C7F958B92C
:10C7C0000EE000980BF020FA41EC100B51EC100B2E
:10C7D00003F0A0F920B1FFE700980499886003E016
:10C7E000FF208DF8170014E0049901F11C009DED65
:10C7F000020A4968D1ED060AFEF796F99DF80F0086
:10C8000004990870049800F009F800208DF81700CA
:10C81000FFE79DF9170006B080BD000080B584B029
:10C820000290029820B9FFE7FF208DF80F0013E077
:10C83000029900200190C86002990861029948613C
:10C840000299886102981C309FED050AFEF70AFAEA
:10C8500001988DF80F00FFE79DF90F0004B080BD2F
:10C860000000000082B00090009820B9FFE7FF2090
:10C870008DF8070005E000990020C8608DF80700DA
:10C88000FFE79DF9070002B07047000000000000BC
:10C89000EFF30980BFF36F8F154B1A681EF0100F6E
:10C8A00008BF20ED108A20E9F04F10602DE9090043
:10C8B0004FF0500080F31188BFF34F8FBFF36F8F9D
:10C8C00006F050F84FF0000080F31188BDE8090031
:10C8D00019680868B0E8F04F1EF0100F08BFB0EC00
:10C8E000108A80F30988BFF36F8F704700BF00BFC5
:10C8F0003816002080B582B004F0D4F841F62071DB
:10C90000C2F20001086020B9FFE7FE208DF80700A1
:10C9100017E04CF64922C0F60002002000900321E7
:10C92000F6F79CFD009840F26461C2F200010876BF
:10C9300048610861C8608860486008608DF8070039
:10C94000FFE79DF9070002B080BD000080B584B00C
:10C95000029001910092029820B9FFE7FE208DF825
:10C960000F006DE0009820B9FFE7FE208DF80F0062
:10C9700066E00199022008700098F8F759FC0098C9
:10C9800001998068C86100980199C06808620098A0
:10C990000199006848610098019940688861009891
:10C9A000B0F91000FEF73CF8019981F824000098D6
:10C9B000B0F91200FEF734F8019981F825000098CB
:10C9C000B0F91400FEF72CF8019981F826000098C0
:10C9D000B0F91600FEF724F8019981F827000098B5
:10C9E000B0F91800FEF71CF8019981F828000098AA
:10C9F000B0F91A00FEF714F8019981F8290000989F
:10CA0000B0F91C00FEF70CF8019981F82A00009893
:10CA1000B0F91E00FEF704F8019981F82B00009888
:10CA2000B0F91C0040F29F61884205D1FFE70098F1
:10CA30000199F8F7CBFBFFE700208DF80F00FFE727
:10CA40009DF90F0004B080BD80B541F62070C2F2A0
:10CA500000000068012103F045FF80BD80B582B071
:10CA60000020F6F79BFC40F26461C2F2000119223B
:10CA7000FDF7EEFE20B9FFE700208DF8070003E088
:10CA8000FF208DF80700FFE79DF9070002B080BD89
:10CA900080B582B00190019A0121084603F074FF2D
:10CAA0000138B0FA80F0400902B080BD80B582B094
:10CAB00001900198806B009000980168486820F010
:10CAC000030048600099486D40F0100048650099E7
:10CAD000012081F851000098FBF788FE02B080BD6C
:10CAE00080B582B001900198806B00900098FCF7AF
:10CAF0000FFA02B080BD000080B582B001900198AD
:10CB0000806B00900098FCF735FF02B080BD0000FC
:10CB100080B582B001900198806B00900098FCF77E
:10CB20007DFF02B080BD000080B584B00390039803
:10CB3000806B0290FBF760F8019003980068006832
:10CB400000F48070B0F5807F39D0FFE7029801686B
:10CB5000486820F0200048600298806868B9FFE7C4
:10CB600002984068B0F5827F07D1FFE7029801681C
:10CB7000486820F00300486006E0029801684868B1
:10CB800020F001004860FFE70298019A642100F05C
:10CB9000B5F820B1FFE7029920204865FFE7029928
:10CBA0000020C8870299012081F851000298406D49
:10CBB00020B1FFE70298FBF719FE04E0FFE70298B7
:10CBC000FCF77CF9FFE704B080BD000080B584B0BD
:10CBD00003900398806B0290FBF70EF80190039886
:10CBE0000068006800F48070B0F5807F3BD0FFE7FC
:10CBF00002980168486820F02000486002980168A7
:10CC0000486820F0020048600298019A642100F010
:10CC1000E7F830B1FFE70299486D40F02000486521
:10CC2000FFE70298806870B9FFE7FFE700200090F7
:10CC300002980068C06800900298006880680090C0
:10CC40000098FFE7FFE702990020C88602990120BB
:10CC500081F851000298406D20B1FFE70298FBF780
:10CC6000C5FD04E0FFE70298FCF760FEFFE704B0B3
:10CC700080BD000080B584B003900398806B029063
:10CC8000FAF7BAFF019003980068006800F480701A
:10CC9000B0F5807F2BD0FFE702980168486820F04C
:10CCA000200048600298019A642100F099F830B1A0
:10CCB000FFE70299486D40F020004865FFE70298C1
:10CCC0000168486820F00300486002990020C88687
:10CCD0000299C8870299012081F851000298406D9D
:10CCE00020B1FFE70298FBF781FD04E0FFE702981F
:10CCF000FCF76AFEFFE704B080BD000080B586B097
:10CD000004900391029204984068B0F5827F13D199
:10CD1000FFE704988068B0F5004F06D0FFE704985D
:10CD20008068B0F5806F07D1FFE704980168086854
:10CD300020F040000860FFE704984068B0F5827F6B
:10CD400031D1FFE704988068B0F5806F15D0FFE718
:10CD50000498039B02996A4611608021002200F02A
:10CD6000BDF848B1FFE70499486D40F020004865E0
:10CD700003208DF817002FE014E00498039B02991C
:10CD80006A4611600121002200F0A8F848B1FFE7CF
:10CD90000499486D40F02000486503208DF8170085
:10CDA0001AE0FFE714E00498039B02996A461160B9
:10CDB0000121002200F092F848B1FFE70499486D84
:10CDC00040F02000486503208DF8170004E0FFE7DD
:10CDD00000208DF81700FFE79DF8170006B080BD12
:10CDE00080B586B00490039102920498039B029947
:10CDF0006A4611600221012200F070F848B1FFE795
:10CE00000499486D40F02000486503208DF8170014
:10CE100048E040F20000C2F2000000684AF6AB2190
:10CE2000CAF6AA21A0FB011000094DF68361C4F2E5
:10CE30001B31A0FB0110800C4FF47A714843019024
:10CE400004984068B0F5827F15D1FFE70498039BF2
:10CE500002996A4611608021002200F03FF848B133
:10CE6000FFE70499486D40F02000486503208DF8E5
:10CE7000170017E012E0FFE7019808B9FFE70CE0A0
:10CE8000019801380190FFE7049800688068C1B2FA
:10CE90000020B0EBD11FEFD1FFE7FFE700208DF8B6
:10CEA0001700FFE79DF8170006B080BD82B0009024
:10CEB0000098006843F20001C4F20101884204D1E5
:10CEC000FFE700208DF8070003E002208DF807003F
:10CED000FFE79DF8070002B07047000080B58AB0F8
:10CEE000DDF830C0089007918DF81B200593059858
:10CEF0000190FAF781FE024601980C99891A0844BC
:10CF00000390FAF779FE0290039840F20001C2F212
:10CF100000010968C1F3CB3148430490FFE708984A
:10CF20000068806807990840401AB0FA80F040090C
:10CF30009DF81B1088425FD0FFE70598013000285C
:10CF400059D0FFE7FAF758FE0299401A0399884230
:10CF500004D2FFE70398002842D1FFE70898016850
:10CF6000486820F0E000486008984068B0F5827F8B
:10CF700013D1FFE708988068B0F5004F06D0FFE7AF
:10CF800008988068B0F5806F07D1FFE708980168BE
:10CF9000086820F040000860FFE70898806AB0F554
:10CFA000005F0FD1FFE7FFE708980168086820F4E9
:10CFB0000050086008980168086840F40050086054
:10CFC000FFE7FFE70899012081F85100FFE7089982
:10CFD000002081F85000FFE703208DF827000FE0C4
:10CFE000049818B9FFE70020039003E00498013883
:10CFF0000490FFE7FFE792E700208DF82700FFE7A6
:10D000009DF827000AB080BD00000000000000006D
:10D01000074B19680868B0E8F04F80F30988BFF340
:10D020006F8F4FF0000080F31188704700BF00BF82
:10D030003816002080B56FF00400002102F018FEC1
:10D0400080BD000084B003900291039890ED000A27
:10D05000029890ED001A30EE010A8DED010A9DED67
:10D06000010AB7EE001AB4EE410AF1EE10FA1BDD28
:10D07000FFE79DED011AB7EE000A80EE010A8DED83
:10D08000000A9DED001A039890ED000A20EE010AB7
:10D0900080ED000A9DED001A029890ED000A20EE46
:10D0A000010A80ED000AFFE704B0704700000000AD
:10D0B00080B586B004908DF80F10049828B9FFE76A
:10D0C0000020CBF68070059065E0049880690078B8
:10D0D0000146009120B1FFE70098012805D009E042
:10D0E0000020C4F24820029007E00020C4F2C830BB
:10D0F000029002E0002005904DE0049882699DF8BE
:10D100000F1002EB810292ED020A90ED3E1A20EE22
:10D11000010A00EB011090ED091A30EE410A10EE01
:10D12000100A0AF071FD41EC100B51EC100B9FED51
:10D130001C0B52EC103BD20F62F3DF7141EC100B71
:10D1400051EC100B09F03AFE01909DED010A9DEDA6
:10D15000021AB4EE410AF1EE10FA12DAFFE79DED81
:10D16000010A20EE000A9DED021A21EE011A80EE5E
:10D17000011AB7EE000A30EE410A049880ED2D0A3C
:10D1800004E004990020C1F8B400FFE70498D0F847
:10D19000B4000590FFE79DED050A06B080BD00BF15
:10D1A000000000000000000080B586B004900391EC
:10D1B000049828B1FFE70498B0F8BC0020B9FFE755
:10D1C000FF208DF817004FE0049890ED000A90EDD5
:10D1D0002E1A30EE410A8DED020A0498D0ED300A85
:10D1E00090ED3F0A9FED221AF7F776FE8DED010ACA
:10D1F0009DED020A0498806990ED052AB7EE001AA9
:10D2000081EE021AB4EE410AF1EE10FA28DBFFE7D4
:10D210000398C078C00718B3FFE79DED010AB7EE89
:10D22000001AB4EE410AF1EE10FA19DCFFE7049996
:10D230000868C1F8B800049901F1FC00896991ED12
:10D24000040AB8EE400ADFED0A0A80EE800AF7F71A
:10D2500001FE0499B1F8BC000138A1F8BC00FFE759
:10D2600000208DF81700FFE79DF9170006B080BD7C
:10D27000DB0FC94084B002908DED010A029820B9FD
:10D28000FFE7FF208DF80F001DE00298806900780D
:10D290000146009120B1FFE70098012808D00EE078
:10D2A000029942F20000C4F2CB50C1F8F80006E047
:10D2B00002990020C4F27A50C1F8F800FFE700207C
:10D2C0008DF80F00FFE79DF90F0004B070470000D4
:10D2D00080B586B004900391049818B1FFE70398D5
:10D2E00020B9FFE7FF208DF8170035E0F6F700F8CA
:10D2F0000AF0DFFC00EE100A9FED191A8DED011AFD
:10D3000080EE010A049880ED000AF5F7F1FF049A17
:10D3100002929368D268C01A91410AF0CAFC9DED4E
:10D32000011A0146029800EE101A80EE010A80ED03
:10D33000040AF5F7DDFF0A460499CA60886004987C
:10D340009FED080AFFF796FF0498039900F0E8F8AC
:10D3500000208DF81700FFE79DF9170006B080BD8B
:10D36000002474490000694380B58AB00890079191
:10D370008DED060A089858B1FFE7079840B1FFE71E
:10D380009DED060AB5EE400AF1EE10FA04DCFFE767
:10D39000FF208DF82700BEE0079840688DF8170041
:10D3A000079808998861F5F7A7F800200490FFE72F
:10D3B00004989DF81710884248DAFFE70798049907
:10D3C00001EB810100EB41002830FEF717FA0898C5
:10D3D0000499C1EB011100EB810000F580709DED17
:10D3E000060A079901F1440201210391FFF74AF966
:10D3F00003990898049AC2EB021200EB820000F530
:10D40000BC709DED060A079A6432FFF73BF9089954
:10D41000049801EB401000F51A709DED060A896929
:10D42000D1ED410AFDF780FB0899049801EB40100B
:10D4300000F52A709DED060A8969D1ED420AFDF7D3
:10D4400073FBFFE7049801300490B1E707983C3084
:10D45000FEF7D4F90898806990F8400001460291DF
:10D46000D8B1FFE7029801282ED1FFE7089800F510
:10D47000F8709DED060A079901F1C402012101919E
:10D48000FFF700F90199089800F50B709DED060A69
:10D49000079AE432FFF7F6F81AE0089800F5F870FA
:10D4A0009DED060A079901F1840201210091FFF721
:10D4B000E9F80099089800F50B709DED060A079AA7
:10D4C000A432FFF7DFF803E0FC208DF8270022E00C
:10D4D000089901F53A709DED060A8969D1ED430A74
:10D4E000FDF722FB089901F542709DED060A896956
:10D4F000D1ED440AFDF718FB08990020C1F8C800D7
:10D50000C1F8C400C1F8C000C1F8BC00C1F8B8003F
:10D510008DF82700FFE79DF927000AB080BD0000C5
:10D5200080B584B002900191029820B9FFE7FF20F6
:10D530008DF80F00C1E002988069007FC0070028C5
:10D5400000F0AB80FFE7029890F89C000146009144
:10D55000032800F29C800099DFE801F0022054715A
:10D56000029890ED140A9FED591A80EE010A806925
:10D5700090ED081AB4EE410AF1EE10FA09DDFFE76A
:10D580000299012081F89C0002990868C1F898006E
:10D59000FFE70298019900F091F97DE0029890ED83
:10D5A000140A9FED4A1A80EE010A806990ED081A6C
:10D5B000B4EE410AF1EE10FA05DAFFE70299002015
:10D5C00081F89C0068E0029890ED000A90ED261A20
:10D5D00030EE410A806990ED091AB4EE410AF1EE8D
:10D5E00010FA09DBFFE70299012081F89400029903
:10D5F000022081F89C004FE0FFE70298019900F0BB
:10D600005DF949E002990020A1F8BC00029890ED74
:10D61000300A816991ED041AB8EE412A9FED291A6A
:10D6200081EE021A30EE010A80ED3F0A02990320D2
:10D6300081F89C0002990868C1F89800FFE70298F9
:10D64000019900F03BF9029890ED000A90ED261A3E
:10D6500030EE410A9FED1C1AB4EE410AF1EE10FAC9
:10D6600014DBFFE7029890ED140A9FED181A80EE84
:10D67000010AB3EE041AB4EE410AF1EE10FA05DA2B
:10D68000FFE70299002081F89C00FFE704E002997F
:10D69000002081F89C00FFE70BE00299002081F850
:10D6A0009C00029981F894000298019900F006F913
:10D6B000FFE700208DF80F00FFE79DF90F0004B091
:10D6C00080BD00BFDB0FC9C09A99993E00007A4423
:10D6D00080B586B00490049820B9FFE7FF208DF84C
:10D6E00017005AE00498806940688DF80F00002008
:10D6F0000290FFE702989DF80F1088422FDAFFE7AB
:10D7000004980299C1EB011100EB810000F58070D3
:10D71000FFF784F804980299C1EB011100EB810036
:10D7200000F5BC70FFF77AF80498029900EB4110FD
:10D7300000F51A709FED1B0A8DED010AFDF792FAB4
:10D740009DED010A0498029900EB411000F52A7042
:10D75000FDF788FAFFE7029801300290CAE70498C3
:10D7600000F5F870FFF75AF8049800F50B70FFF712
:10D7700055F8049800F53A709FED0A0A8DED000AFD
:10D78000FDF770FA9DED000A049800F54270FDF770
:10D7900069FA00208DF81700FFE79DF9170006B021
:10D7A00080BD00BF0000000080B584B002900298E8
:10D7B00020B9FFE7FF208DF80F0034E00298806960
:10D7C00040688DF8070000200090FFE700989DF862
:10D7D0000710884219DAFFE702980099C1EB01119E
:10D7E00000EB810000F58070FFF73CF8029800998B
:10D7F000C1EB011100EB810000F5BC70FFF732F8BE
:10D80000FFE7009801300090E0E7029800F5F8701B
:10D81000FFF728F8029800F50B70FFF723F80020B7
:10D820008DF80F00FFE79DF90F0004B080BD0000E8
:10D8300084B00290029820B9FFE7FF208DF80F0016
:10D8400038E00298806940688DF807000020009059
:10D85000FFE700989DF8071088421EDAFFE702985C
:10D86000009900EB81010020C1F8CC000299009AD8
:10D8700001EB8201C1F8D4000299009A01EB820108
:10D88000C1F8DC000299009A01EB8201C1F8E400C2
:10D89000FFE7009801300090DBE702990020C1F813
:10D8A000EC000299C1F8F0000299C1F8F4008DF87B
:10D8B0000F00FFE79DF90F0004B0704780B598B0E6
:10D8C00016901591169818B1FFE7159820B9FFE743
:10D8D000FF208DF85F004DE31698806940688DF851
:10D8E00053001698007F48BBFFE700201390FFE726
:10D8F00013989DF8531088420FDAFFE71698806955
:10D90000139901EB810100EB41002830FEF706F886
:10D91000FFE7139801301390EAE7169880693C30CE
:10D92000FDF7FCFF169890ED300A80ED3F0A40F2BB
:10D930006450C2F2000080ED000AF8E2169890F8F8
:10D9400090000146099150B1FFE70998012800F0C5
:10D95000AB80FFE70998022800F0DB81E1E20020BC
:10D960001290FFE712989DF85310884251DAFFE7B2
:10D9700016981299C1EB011100EB810000F580703F
:10D98000FEF770FF1699129AC2EB021001EB8000AD
:10D9900000F5807001EB8202D2ED2A0AD1ED041A63
:10D9A0009FEDE31AB0EE410AFEF7F4FC16981299C7
:10D9B00000EB810080ED330A1698129900EB81018B
:10D9C000D1F8CC00C1F8DC001699129A01EB421094
:10D9D00000F52A7001EB820191ED370AFDF748F856
:10D9E0001698129900EB810080ED390A1699886922
:10D9F000129A02EB820300EB4300283001EB820114
:10DA000091ED390AFDF796FFFFE712980130129069
:10DA1000A8E7169901F5F87040F26452C2F20002CC
:10DA200092ED000AD1ED041AD1ED300A9FEDC01A33
:10DA30008DED081AFEF7AEFC9DED081A169880EDE4
:10DA40003B0A169901F50B70D1ED041AD1ED320A9B
:10DA500091ED3B0AFEF79EFC169880ED3C0A169964
:10DA600001F5427091ED3C0AFDF702F8169880ED41
:10DA70003D0A169988693C3091ED3D0AFDF75AFF41
:10DA800015988078C00770B1FFE71698FFF720FE61
:10DA90001698FFF789FE1698FFF7CAFE169901201F
:10DAA00081F89000FFE741E200201190FFE7119814
:10DAB0009DF85310884280F2AC80FFE71698806989
:10DAC000119901EB810100EB410090F83000013821
:10DAD0008DF84300169881699DF8432001EB82017F
:10DAE00091ED020A90ED3E1A20EE010A9FED911A87
:10DAF00080EE010A8DED0F0A16989DF84410FFF78D
:10DB0000D7FA8DED0E0A1699119AC2EB021001EBAD
:10DB1000800000F580709DED0F0A01EB8202D2EDCE
:10DB20002A0AD1ED041A9FED821A8DED061AFEF72E
:10DB300031FC9DED061A1698119900EB810080EDDD
:10DB4000330A9DED0E0A8DED070A1699119BC3EB62
:10DB5000031001EB800000F5BC7001F1A002D1F8C8
:10DB600018C003EB830E0CEB4E0C9CF830C002EB9C
:10DB70008C0C9CED030A02EB8302D2ED020AD1ED7C
:10DB8000041AFEF707FCB0EE401A9DED070A20EEDE
:10DB9000010A1698119900EB810080ED350A16985C
:10DBA000119900EB810101F1CC00D431FFF74AFA61
:10DBB0001698119900EB810090ED330A90ED351A1B
:10DBC00030EE010A80ED370A1699119A01EB4210E6
:10DBD00000F52A7001EB820191ED370AFCF748FF4E
:10DBE0001698119900EB810080ED390A1699886921
:10DBF000119A02EB820300EB4300283001EB820113
:10DC000091ED390AFDF796FEFFE71198013011906A
:10DC10004DE7169901F5F87040F26452C2F2000225
:10DC200092ED000AD1ED041AD1ED300A9FEDD31A1E
:10DC30008DED051AFEF7AEFB9DED051A169880EDE9
:10DC40003B0A169901F50B70D1ED041AD1ED320A99
:10DC500091ED3B0AFEF79EFB169880ED3C0A169963
:10DC600001F5427091ED3C0AFCF702FF169880ED39
:10DC70003D0A169988693C3091ED3D0AFDF75AFE40
:10DC800015988078C00758B9FFE71698FFF720FD70
:10DC90001698FFF7CDFD1699002081F8900037E027
:10DCA00041F23850C2F200000078C00778BBFFE7AD
:10DCB0001598C078C00750B3FFE71699022081F885
:10DCC00090001698007F01460491012808D0FFE7D4
:10DCD0000498022809D0FFE7049803280BD010E02D
:10DCE00016990120A1F8BC0010E016998869806996
:10DCF000A1F8BC000AE0169941F60A20A1F8BC0080
:10DD000004E016990020A1F8BC00FFE7FFE7FFE759
:10DD10000CE116981599FFF747FA00200D90FFE7E0
:10DD20000D989DF85310884280F2B18004E000BF46
:10DD30000000000000C0DA45169880690D9901EBDB
:10DD4000810100EB410090F8300001388DF833007C
:10DD5000169881699DF8332001EB820191ED020A4A
:10DD600090ED3E1A20EE010A9FED851A80EE010A21
:10DD70008DED0B0A16989DF83410FFF799F98DED8B
:10DD80000A0A16990D9AC2EB021001EB800000F509
:10DD900080709DED0B0A01EB8202D2ED2A0AD1EDD3
:10DDA000041A9FED761A8DED021AFEF7F3FA9DED37
:10DDB000021A16980D9900EB810080ED330A9DED53
:10DDC0000A0A8DED030A16990D9BC3EB031001EBB4
:10DDD000800000F5BC7001F1A002D1F818C003EB7F
:10DDE000830E0CEB4E0C9CF830C002EB8C0C9CEDBF
:10DDF000030A02EB8302D2ED020AD1ED041AFEF708
:10DE0000C9FAB0EE401A9DED030A20EE010A1698F9
:10DE10000D9900EB810080ED350A16980D9900EB05
:10DE2000810101F1CC00D431FFF70CF916980D995E
:10DE300000EB810090ED330A90ED351A30EE010AC7
:10DE400080ED370A16990D9A01EB421000F52A7001
:10DE500001EB820191ED370AFCF70AFE16980D9945
:10DE600000EB810080ED390A169988690D9A02EB62
:10DE7000820300EB4300283001EB820191ED390A67
:10DE8000FDF758FDFFE70D9801300D9048E7169912
:10DE900001F5F870D1ED041AD1ED300A91ED3F0A89
:10DEA0009FED361A8DED011AFEF774FA9DED011AF9
:10DEB000169880ED3B0A169901F50B70D1ED041A06
:10DEC000D1ED320A91ED3B0AFEF764FA169880ED27
:10DED0003C0A169901F5427091ED3C0AFCF7C8FD29
:10DEE000169880ED3D0A169988693C3091ED3D0AFF
:10DEF000FDF720FD1598C078C00788B9FFE716998F
:10DF0000012081F890001698D0F8C00040F26451CA
:10DF1000C2F20001086016990020A1F8BC00FFE7DA
:10DF200004E01699002081F89000FFE7FFE71698BB
:10DF300080692830FDF7C4FA169880694068052882
:10DF400006D3FFE7169880695030FDF7B9FAFFE76E
:10DF5000169880693C30FDF7B3FA1598C07800F048
:10DF6000010041F23851C2F20001087000208DF822
:10DF70005F00FFE79DF95F0018B080BD0000000062
:10DF800000C0DA4583B001908DF80310019820B9E4
:10DF9000FFE7FF208DF80B0007E09DF803000199D3
:10DFA000087700208DF80B00FFE79DF90B0003B008
:10DFB0007047000080B588B00690069820B9FFE74A
:10DFC000FF208DF81F0058E10698806940688DF8A1
:10DFD000170000200490FFE704989DF8171088426E
:10DFE00080F29680FFE706988069049901EB810131
:10DFF00000EB41002830FDF72BFD0698806904995D
:10E0000001EB810100EB41002830FDF793FB039009
:10E010000398A0B1FFE70698049900EB0111DDF821
:10E020000CC0DCF82C00DCF83020DCF83430DCF8F4
:10E0300038C0C1F82CC08B624A620862FFE70699BB
:10E04000049A01EB421000F51A7001EB021191EDF8
:10E05000090AFCF70DFD0698049900EB810080ED9C
:10E06000280A0698049900EB810090ED280A9FED9C
:10E07000881A80EE010A80ED2A0A0698049900EBBE
:10E08000810090ED2A0AB7EE001AB4EE410AF1EED3
:10E0900010FA09DDFFE70698049900EB81014FF0C3
:10E0A0007E50C1F8A800FFE70698049900EB8100B4
:10E0B00090ED2A0ABFEE001AB4EE410AF1EE10FA12
:10E0C0000ADAFFE70698049900EB81010020CBF6FD
:10E0D0008070C1F8A800FFE7069901F1A000049A3A
:10E0E00000EB820393ED021A896902EB820201EBD5
:10E0F000420191F8301000EB810090ED030A30EE00
:10E10000010A80ED030AFFE704980130049063E7F9
:10E1100001200290FFE70298002815DCFFE706982F
:10E12000029900EB810090ED2C0A9DF8171001EE8A
:10E13000101AB8EEC11A80EE010A80ED2C0AFFE732
:10E14000029801300290E6E7069880693C30FDF7BE
:10E150007FFC069800F14001019180693C30FDF799
:10E16000E9FA014601985022F2F77BF90698816995
:10E1700091ED030A90ED221A20EE010A80ED300A9B
:10E18000FFE7069890ED300AB5EE400AF1EE10FA7E
:10E190000ADAFFE7069890ED300A9FED3A1A30EE62
:10E1A000010A80ED300AECE7FFE7069890ED300AAF
:10E1B0009FED341AB4EE410AF1EE10FA0ADBFFE7E4
:10E1C000069890ED300A9FED311A30EE010A80ED8D
:10E1D000300AEAE7069890F86800C00750B1FFE7F8
:10E1E000069890ED301A9FED270A30EE410A80ED37
:10E1F000300AFFE7069901F53A7091ED130AFCF732
:10E2000037FC069880ED310A069890ED130A9FEDD1
:10E210001E1A80EE010A80ED320A069890ED320A4D
:10E22000B7EE001AB4EE410AF1EE10FA06DDFFE790
:10E2300006994FF07E50C1F8C800FFE7069890EDB0
:10E24000320ABFEE001AB4EE410AF1EE10FA07DA14
:10E25000FFE706990020CBF68070C1F8C800FFE701
:10E26000069890ED090A90ED0D1A30EE410A80ED06
:10E27000CA0A00208DF81F00FFE79DF91F0008B0B3
:10E2800080BD00BFDB0FC9400080BB45DB0FC9C0AC
:10E2900000C0DA4580B582B0019002F003FC02F0C4
:10E2A000B7FC02B080BD000080B582B0009000983D
:10E2B0000138B0F1807F03D3FFE70120019019E01E
:10E2C000009801384EF21401CEF2000108604FF0C0
:10E2D000FF300F2101F0AAFC4EF21801CEF200012E
:10E2E000002008604EF21002CEF2000207211160F9
:10E2F0000190FFE7019802B080BD000080B5F9F7FA
:10E3000081FC05F023FD012803D0FFE704F03AFC6F
:10E31000FFE780BD80B594B008A83021F2F7DBF8A4
:10E32000002007900690059004900390FFE70020DE
:10E33000029043F64000C4F20200016841F08051AF
:10E340000160006800F0805002900298FFE7FFE74C
:10E350000020019047F20000C4F20000016841F47F
:10E3600080410160006800F4804001900198FFE75F
:10E37000012008904FF48030099002200E904FF455
:10E3800080010F9106211091A82111911290042073
:10E39000139008A8F9F7CAFE18B1FFE7F7F7CEF80F
:10E3A000FFE70F20039002200490002005904FF417
:10E3B000A05006904FF48050079003A80521F9F76C
:10E3C000E5FC18B1FFE7F7F7B9F8FFE714B080BD37
:10E3D0004EF68851CEF20001086840F470000860E3
:10E3E0007047000083B0029001910298006800908D
:10E3F00002980021C4F20101884225D0FFE702986B
:10E40000B0F1804F20D0FFE7029840F20041C4F203
:10E410000001884218D0FFE7029840F60001C4F2DC
:10E420000001884210D0FFE7029840F60041C4F294
:10E430000001884208D0FFE7029840F20041C4F290
:10E44000010188420AD1FFE7009820F07000009097
:10E4500001984168009808430090FFE70298002166
:10E46000C4F20101884255D0FFE70298B0F1804F15
:10E4700050D0FFE7029840F20041C4F20001884208
:10E4800048D0FFE7029840F60001C4F2000188423C
:10E4900040D0FFE7029840F60041C4F200018842F4
:10E4A00038D0FFE7029840F20041C4F201018842EF
:10E4B00030D0FFE7029844F20001C4F20101884223
:10E4C00028D0FFE7029844F20041C4F201018842DB
:10E4D00020D0FFE7029844F60001C4F2010188420F
:10E4E00018D0FFE7029841F60001C4F2000188420B
:10E4F00010D0FFE7029841F60041C4F200018842C3
:10E5000008D0FFE7029842F20001C4F200018842FD
:10E510000AD1FFE7009820F4407000900198C1688C
:10E52000009808430090FFE7009820F080000199D0
:10E53000496908430090019880680299C86201986F
:10E5400000680299886202980021C4F201018842A1
:10E5500008D0FFE7029840F20041C4F2010188426E
:10E5600005D1FFE70198006902990863FFE7029966
:10E57000086840F004000860029901204861009892
:10E580000299086003B0704784B003900291019231
:10E59000029800F01F01012088400090009A039922
:10E5A000086A904308620198029901F01F0100FA7D
:10E5B00001F20399086A1043086204B07047000032
:10E5C00085B0049003910498006A01900499086A48
:10E5D00020F0010008620498406800900498806967
:10E5E0000290029820F070000290029820F0030040
:10E5F000029003980168029808430290019820F065
:10E6000002000190039881680198084301900498E2
:10E610000021C4F20101884208D0FFE7049840F2CB
:10E620000041C4F2010188420ED1FFE7019820F0B9
:10E63000080001900398C16801980843019001986F
:10E6400020F004000190FFE704980021C4F20101CA
:10E65000884208D0FFE7049840F20041C4F201016B
:10E66000884213D1FFE7009820F480700090009852
:10E6700020F40070009003984169009808430090CE
:10E6800003988169009808430090FFE70098049977
:10E690004860029804998861039840680499486327
:10E6A00001980499086205B07047000085B0049095
:10E6B00003910498006A01900499086A20F0100000
:10E6C000086204984068009004988069029002985B
:10E6D00020F4E0400290029820F4407002900398E9
:10E6E0000168029840EA01200290019820F0200081
:10E6F000019003988168019840EA01100190049804
:10E700000021C4F20101884208D0FFE7049840F2DA
:10E710000041C4F2010188420FD1FFE7019820F0C7
:10E72000800001900398C168019840EA01100190AF
:10E73000019820F040000190FFE704980021C4F206
:10E740000101884208D0FFE7049840F20041C4F27A
:10E750000101884215D1FFE7009820F48060009005
:10E76000009820F40060009003984169009840EA06
:10E770008100009003988169009840EA8100009030
:10E78000FFE700980499486002980499886103980B
:10E7900040680499886301980499086205B070473D
:10E7A00085B0049003910498006A01900499086A66
:10E7B00020F4807008620498406800900498C06952
:10E7C0000290029820F070000290029820F003005E
:10E7D000029003980168029808430290019820F47F
:10E7E0000070019003988168019840EA012001902F
:10E7F00004980021C4F20101884208D0FFE7049880
:10E8000040F20041C4F2010188420FD1FFE70198B4
:10E8100020F4006001900398C168019840EA01204B
:10E820000190019820F480600190FFE70498002196
:10E83000C4F20101884208D0FFE7049840F2004189
:10E84000C4F20101884215D1FFE7009820F48050FE
:10E850000090009820F400500090039841690098BF
:10E8600040EA0110009003988169009840EA011085
:10E870000090FFE700980499486002980499C861E5
:10E88000039840680499C86301980499086205B028
:10E890007047000085B0049003910498006A0190CD
:10E8A0000499086A20F48050086204984068009037
:10E8B0000498C0690290029820F4E0400290029807
:10E8C00020F44070029003980168029840EA012009
:10E8D0000290019820F400500190039881680198FB
:10E8E00040EA0130019004980021C4F201018842FD
:10E8F00008D0FFE7049840F20041C4F201018842C9
:10E900000BD1FFE7009820F4804000900398416904
:10E91000009840EA81100090FFE700980499486051
:10E9200002980499C86103984068049908640198A2
:10E930000499086205B0704780B588B0079001F06F
:10E94000BDFC4EF6E120C0F6000048F29012C0F681
:10E9500001020021049102F0ADF8049941F64462ED
:10E96000C2F20002069210604FF27910C0F6000069
:10E9700048F24422C0F6010202F09CF80499069A7B
:10E9800050604EF6A150C0F6000048F2B412C0F636
:10E99000010202F08FF80499069A90604EF6A16089
:10E9A000C0F6000048F2D812C0F6010202F082F868
:10E9B0000499069AD0604EF6C970C0F6000048F27D
:10E9C000FC12C0F6010202F075F80499069A106173
:10E9D0004FF24920C0F6000048F26822C0F601025A
:10E9E00002F068F8049A06994861022005900F2108
:10E9F00001F052FD049A069B0146059819623121E7
:10EA000001F04AFD049A069B0146059859622021AF
:10EA100001F042FD049A069B0146059899620C217B
:10EA2000019101F039FD0199049ADDF818C00346FF
:10EA30000598CCF8343001F02FFD049A069B01466E
:10EA4000059819631021029101F026FD049A069B96
:10EA5000014605989963282101F01EFD049A069B42
:10EA600001460598D9631C2101F016FD0299049A0C
:10EA7000DDF818C003460598CCF8403001F00CFDD5
:10EA8000049A069B014605985964042101F004FD8F
:10EA9000049A069B014605985965582101F0FCFC33
:10EAA000049A069B01460598D9641921039101F047
:10EAB000F3FC0399049ADDF818C003460598CCF8D6
:10EAC000503001F0E9FC0699886501F04DFC01F039
:10EAD000E9FF02F09DF808B080BD000000000000D2
:10EAE00080B58CB00B9001F0C1FB08F05FFC41ECED
:10EAF000100B9FEDA51B53EC112B51EC100B08F0E4
:10EB00004BFA41EC100B51EC100B08F00BFC0A9087
:10EB10000020089001F026FB01F094FB099040F2E0
:10EB20000860C2F20000079040F20801C2F2000142
:10EB3000F3F7B0F80798F3F785F840F2D450C2F233
:10EB4000000041F22451C2F20001F1F7E5FD0899FD
:10EB500041F2E440C2F2000040F22432C2F200026C
:10EB60009FED8B0AFDF78EFD0898F4F7A1FA08983F
:10EB700041F6B961C0F60101F4F782F90898F4F79B
:10EB800029F9FFE70A99099808440990F3F772FAFE
:10EB9000F3F740F8F3F74EF8F3F766F8F3F772F887
:10EBA00001F08CFB40F20860C2F200000690F3F71F
:10EBB00035F90698F3F7ACF941F23450C2F200008F
:10EBC000006801286AD1FFE740F20861C2F2000143
:10EBD00091ED071A41F2C000C2F2000090ED000A68
:10EBE00030EE010A80ED000A91ED081A90ED010A5D
:10EBF00030EE010A80ED010A91ED091A90ED020A4A
:10EC000030EE010A80ED020A40F24E60C2F20000CE
:10EC1000018801310180008841F2883188423CDB63
:10EC2000FFE741F2C000C2F2000090ED000A9FED44
:10EC3000591A80EE010A40F20801C2F2000181ED8A
:10EC4000000A90ED010A80EE010A81ED010A90EDC3
:10EC5000020A80EE010A81ED020A40F25062C2F21D
:10EC600000020020107041F23452C2F20002106023
:10EC700040F20860C2F200000590F3F70BF8059827
:10EC8000F2F7E0FF40F2D450C2F2000041F224510A
:10EC9000C2F20001F1F740FDFFE7FFE740F25060EC
:10ECA000C2F20000007801281BD0FFE740F20860A4
:10ECB000C2F2000000F1100100F11C0240F2D45039
:10ECC000C2F20000049041F22453C2F20003F1F7B3
:10ECD0006FFE049941F2D840C2F20000F1F76EFCD9
:10ECE000FFE701F041FB41F2D841C2F200010868A0
:10ECF0004A688B6841F29801C2F2000100914B61B1
:10ED00000A61C86040F20863C2F200030293D86946
:10ED10001A6A5B6A8B604A60086040F2D45CC2F297
:10ED2000000CDCF80000DCF80420DCF80830DCF82B
:10ED30000CC0C1F824C00B62CA61886141F644600E
:10ED4000C2F200000190C06B01F088FC00990198AC
:10ED5000C06B002303931A4601F01EFC0298D0ED0D
:10ED60000A0A41F2E440C2F200009FED0B0ADFED17
:10ED70000B1AB0EE611AFDF70DFB0398F4F7F8F8E3
:10ED8000099801F009FAFDE60000000000407F400C
:10ED90000000FA4300409C450000204200000000B3
:10EDA00080B590B00F9001F061FA08F0FFFA41ECE5
:10EDB000100B9FED371B53EC112B51EC100B08F08F
:10EDC000EBF841EC100B51EC100B08F0ABFA0E9085
:10EDD000002001F0C7F901F035FA0D90F6F7CAF8F6
:10EDE000014640F28060C2F200009FED2B0A00F065
:10EDF0007FFFFFE70E990D9808440D9041F644609F
:10EE0000C2F200000490406C40F28061C2F2000146
:10EE1000FC31002303931A4601F0DEFA039B0498A9
:10EE2000806A40F6D841C2F200011A4601F0D4FAD5
:10EE300080B9FFE740F28060C2F200000290F5F76F
:10EE40005BFF02980D9A40F6D841C2F20001F4F738
:10EE50006FFD12E0002001900C900B900A90099039
:10EE600008900790069005900D9A40F28060C2F2DB
:10EE7000000005A9F4F75CFDFFE740F28060C2F2F4
:10EE80000000F4F777FF0D9801F086F9B2E700BFB4
:10EE90000000000000407F400000FA430000000036
:10EEA00080B588B0079001F0E1F908F07FFA41ECF5
:10EEB000100B9FED431B53EC112B51EC100B08F082
:10EEC0006BF841EC100B51EC100B08F02BFA06908C
:10EED000002001F047F901F0B5F9059040F6B8407F
:10EEE000C2F2000040F68451C2F20001F4F704FCC3
:10EEF000FFE7069905980844059001F0DFF941F60F
:10EF00004460C2F20000406A41F6B821C2F200013A
:10EF100000231A4601F060FA78B9FFE740F6B840DE
:10EF2000C2F2000041F6B821C2F2000140F684525C
:10EF3000C2F20002F4F7EEFBFFE740F6B840C2F27F
:10EF40000000009041F6B821C2F2000140F6845260
:10EF5000C2F20002019241F6E923C2F200030293D9
:10EF6000F4F7FCFA01F000FA41F64460C2F2000046
:10EF70000490806A01F072FB00990498806A002373
:10EF800003931A4601F008FB0498006C01F066FB3D
:10EF90000199039B0498006C1A4601F0FDFA04984D
:10EFA000406D01F05BFB0299039B0498406D1A468B
:10EFB00001F0F2FA059801F0EFF89AE700BF00BF00
:10EFC0000000000000407F4080B58CB00B9001F045
:10EFD0004DF908F0EBF941EC100B9FED631B53EC7E
:10EFE000112B51EC100B07F0D7FF41EC100B51EC3B
:10EFF000100B08F097F90A90002001F0B3F801F027
:10F0000021F90990F5F7B6FF00F1D40140F6A050C0
:10F01000C2F200009FED560AF6F7F6FCFFE70A99E8
:10F0200009980844099041F64460C2F20000079034
:10F03000C06B41F27001C2F20001059100230693FA
:10F040001A4601F0C9F9059940F6A050C2F2000035
:10F05000F6F7B0FE069B0798006D40F2E851C2F249
:10F06000000108911A4601F0B7F9069B0798006C59
:10F0700040F6F841C2F200011A4601F0ADF90898D5
:10F08000007868B9FFE741F27000C2F2000002693F
:10F0900040F6F841C2F200018A61C0684861FFE7AA
:10F0A00040F2E850C2F20000007801280FD1FFE7DB
:10F0B00040F2E850C2F20000D0F8052040F6F841D6
:10F0C000C2F200018A61D0F801004861FFE740F216
:10F0D000E850C2F20000007802280FD1FFE740F2AA
:10F0E000E850C2F20000D0F8052040F6F841C2F224
:10F0F00000018A61D0F801004861FFE740F6A050A6
:10F10000C2F200000490F6F7EBFD41F64460C2F253
:10F1100000000390406C01F0A1FA04990398406C40
:10F1200001F52871002302931A4601F035FA04997B
:10F13000039801F51E710191C06C01F08FFA0199DD
:10F14000029B0398C06C1A4601F026FA049840F618
:10F15000F841C2F20001F6F7F5F90498F6F714FD4C
:10F16000099801F019F85AE70000000000407F40BC
:10F170000000FA430000000080B586B0059001F061
:10F1800075F808F013F941EC100B9FED2D1B53ECB3
:10F19000112B51EC100B07F0FFFE41EC100B51EC62
:10F1A000100B08F0BFF80490002000F0DBFF01F026
:10F1B00049F80390FDF79EFBFFE704990398084484
:10F1C0000390FDF74BFC1420FDF762FC78B1FFE7DC
:10F1D00040F65050C2F2000040F61451C2F2000155
:10F1E00040F66452C2F20002FDF7B0FB12E040F6B6
:10F1F0005050C2F2000040F61451C2F200010291D8
:10F20000F5F7BAFF029940F66450C2F20000F5F734
:10F21000DDFFFFE741F64460C2F200000190406A62
:10F2200001F01CFA0198406A40F61451C2F2000144
:10F2300000231A4601F0B0F9039800F0ADFFBCE7D7
:10F240000000000000407F4080B588B0079001F0CA
:10F250000DF808F0ABF841EC100B9FED2D1B53ECB3
:10F26000112B51EC100B07F097FE41EC100B51ECF9
:10F27000100B08F057F80690002000F073FF00F024
:10F28000E1FF0590F5F776FE00F5E67141F6F02016
:10F29000C2F2000004909FED200AFEF765F8049882
:10F2A0000121FEF76FFEFFE70699059808440590D7
:10F2B00041F64460C2F200000190406D41F63961B0
:10F2C000C2F200010291002300931A4601F084F873
:10F2D000009B0198806D41F62061C2F200011A4640
:10F2E00001F07AF841F6F020C2F200000390FEF738
:10F2F00061FE029903980978FEF744FE029903988B
:10F30000FDF7E6FF059800F047FFCDE700BF00BF1F
:10F310000000000000407F400000FA4380B582B04A
:10F3200001900198806B009000990020C88500989A
:10F33000FAF72AFE02B080BD80B584B003900020A9
:10F3400002900398806B0190019800684069C0B2F8
:10F35000C0090290019890F8410021280AD1FFE7E6
:10F36000029838B1FFE701990020C884019800F0A5
:10F3700013F9FFE7019800684069C0F3801002901C
:10F38000019890F8420022280AD1FFE7029838B18C
:10F39000FFE701990020C885019800F09FF8FFE77A
:10F3A0000199486C40F0100048640198FAF7ECFDB0
:10F3B00004B080BD80B586B005900598806B049040
:10F3C000059800680068C00500285AD4FFE7049932
:10F3D0000020C885FFE7FFE70498006850E8030FA6
:10F3E00020F480700390FFE703990498026842E8D4
:10F3F00003100028F0D1FFE7FFE7FFE7FFE70498DD
:10F40000006850E8050F20F001000290FFE7029924
:10F410000498026842E805100028F0D1FFE7FFE7F2
:10F42000FFE7FFE70498006850E8050F20F0400070
:10F430000190FFE701990498026842E8051000284E
:10F44000F0D1FFE7FFE70499202081F842000498FB
:10F45000006B012814D1FFE7FFE7FFE7049800687D
:10F4600050E8030F20F010000090FFE70099049887
:10F47000026842E803100028F0D1FFE7FFE7FFE74A
:10F48000FFE70499002048630498006B012805D128
:10F49000FFE70498818DFAF771FD03E00498FBF70C
:10F4A00003FAFFE706B080BD80B582B001900198F5
:10F4B000806B00900099012048630098006B012840
:10F4C00006D1FFE70098818D4908FAF757FD03E060
:10F4D0000098FBF713FAFFE702B080BD84B00390F9
:10F4E000FFE7FFE70398006850E8030F20F49070EF
:10F4F0000290FFE702990398026842E8031000288F
:10F50000F0D1FFE7FFE7FFE7FFE70398006850E867
:10F51000050F20F001000190FFE7019903980268B0
:10F5200042E805100028F0D1FFE7FFE70398006BE1
:10F53000012814D1FFE7FFE7FFE70398006850E8D0
:10F54000030F20F010000090FFE700990398026875
:10F5500042E803100028F0D1FFE7FFE7FFE7039937
:10F56000202081F8420003990020086304B070470E
:10F5700080B582B0019001980168C86820F0400011
:10F58000C8600199202081F841000198FBF7E0F95B
:10F59000002002B080BD000082B00190FFE7FFE7CD
:10F5A0000198006850E8030F20F0C0000090FFE7CA
:10F5B00000990198026842E803100028F0D1FFE7A3
:10F5C000FFE70199202081F8410002B07047000058
:10F5D00082B000900098006844F60001C4F2000177
:10F5E000884204D1FFE700208DF807001DE0009855
:10F5F000006841F20041C4F20101884204D1FFE7F2
:10F6000001208DF8070010E00098006841F2000129
:10F61000C4F20101884204D1FFE702208DF80700FF
:10F6200003E004208DF80700FFE79DF8070002B013
:10F630007047000080B586B00490002003900290CF
:10F64000049890F84200222840F0A080FFE7049838
:10F650008068B0F5805F13D1FFE70498006978B93E
:10F66000FFE70498806A02900498006840686FF38E
:10F670005F20029908800499886A0230886223E03A
:10F680000498806A039004988068B0F5805F08D081
:10F69000FFE70498806850B9FFE70498006930B923
:10F6A000FFE70498006840680399087007E0049831
:10F6B0000068406800F07F0003990870FFE7049934
:10F6C000886A01308862FFE70499C88D0138C885CF
:10F6D0000004002856D1FFE704980168C86820F0AC
:10F6E0002000C86004980168C86820F48070C86071
:10F6F00004980168486920F00100486104992020BD
:10F7000081F842000499002048630498006B0128A6
:10F7100030D1FFE7049900200863FFE7FFE7049872
:10F72000006850E8030F20F010000190FFE70199F6
:10F730000498026842E803100028F0D1FFE7FFE7D1
:10F74000049800680068C00600280ED5FFE7FFE7B0
:10F7500000200090049800680068009004980068F9
:10F76000406800900098FFE7FFE70498818DFAF762
:10F7700005FC03E00498FBF797F8FFE700208DF8FD
:10F78000170007E000208DF8170003E002208DF835
:10F790001700FFE79DF8170006B080BD80B586B062
:10F7A000059005980068006920F44050059A11689A
:10F7B000D26810430861059988680B694A69C9696C
:10F7C000184310430843049005980068C06849F244
:10F7D0000C6188430499084305990968C860059835
:10F7E0000068406920F44070059A116892691043DE
:10F7F00048610598006841F20001C4F201018842A5
:10F8000009D0FFE70598006841F20041C4F2010108
:10F81000884204D1FFE7F8F703FC039003E0F8F710
:10F82000EDFB0390FFE70598C069B0F5004F29D1C3
:10F83000FFE703981921A0FB0101059A13680293C1
:10F8400053685A00DB0FF0F731FD0299864648F203
:10F850001F53C5F2EB13AEFB0320420910014FF01A
:10F86000640C02FB1CEC322202EBCC02A2FB033242
:10F87000F82303EA521300EB4300C2F34212104490
:10F88000886026E003981921A0FB0101059A1368FE
:10F89000019353689A009B0FF0F708FD0199844685
:10F8A00048F21F52C5F2EB12ACFB02304309642050
:10F8B00003FB10CC322000EB0C10A0FB0202F02066
:10F8C00000EA521000EB0310C2F3431210448860A8
:10F8D000FFE706B080BD000080B58AB008900791B0
:10F8E000ADF81A20079808998862BDF81A0008999F
:10F8F0008885089900204864089A222182F84210DD
:10F900000899CA6B4FF2B531C0F60001D16308996E
:10F91000CA6B4FF2A941C0F6000111640899CA6B85
:10F920004FF23931C0F60001D1640899C96B0865FE
:10F9300007A8059008980168C06B0431059A126801
:10F94000BDF81A30F7F778FE58B1FFE70899102094
:10F9500048640899202081F8420001208DF8270092
:10F960004EE0FFE7002004900898006800680490CB
:10F9700008980068406804900498FFE708980069B8
:10F98000A0B1FFE7FFE7FFE70898006850E8030F22
:10F9900040F480700390FFE703990898026842E8FA
:10F9A00003100028F0D1FFE7FFE7FFE7FFE7FFE7DD
:10F9B0000898006850E8050F40F001000290FFE74A
:10F9C00002990898026842E805100028F0D1FFE784
:10F9D000FFE7FFE7FFE70898006850E8050F40F0F1
:10F9E00040000190FFE701990898026842E805107D
:10F9F0000028F0D1FFE7FFE700208DF82700FFE7A0
:10FA00009DF827000AB080BD83B00190019890F85E
:10FA1000410021283AD1FFE701988068B0F5805F66
:10FA200013D1FFE70198006978B9FFE70198006AF0
:10FA30000090009800886FF35F2001990968486082
:10FA40000199086A0230086208E0019A106A411CB4
:10FA500011620078019909684860FFE70199C88C34
:10FA60000138C884000468B9FFE701980168C868D4
:10FA700020F08000C86001980168C86840F040002C
:10FA8000C860FFE700208DF80B0003E002208DF82E
:10FA90000B00FFE79DF80B0003B0704780B582B004
:10FAA00041F2FC30C2F200000190FAF797FA019897
:10FAB000F3F79EFC02B080BD80B582B041F24440B5
:10FAC000C2F200000190FAF789FA0198F3F790FC6E
:10FAD00002B080BD80B582B041F28C40C2F200001D
:10FAE0000190FAF77BFA0198F3F782FC02B080BD2F
:10FAF000FFE7FEE782B041EC100B8DED000B0198A3
:10FB0000C0F30A5040F2FF71401A18BF012002B042
:10FB10007047000082B041EC100B8DED000B019896
:10FB2000C0F30A5040F2FF71401A18BF012002B022
:10FB30007047000081B000EE100A00900098C0F3FA
:10FB4000C750FF3818BF012001B0704781B000EEE8
:10FB5000100A00900098C0F3C750FF3818BF01206A
:10FB600001B0704784B041EC100B8DED020B039A8D
:10FB700000200021CFF6E071B1EB420F019006D1D9
:10FB8000FFE70298B0FA80F040090190FFE7019882
:10FB900000F0010004B0704781B000EE100A009040
:10FBA00000994FF0807000EB4100B0FA80F04009FE
:10FBB00001B0704781B08DF803009DF90300002863
:10FBC00012D4FFE79DF9031001F01F0201209040BD
:10FBD0004A094EF28011CEF2000141F82200BFF333
:10FBE0004F8FBFF36F8FFFE701B0704781B08DF883
:10FBF00003009DF9030000280ED4FFE79DF90310D0
:10FC000001F01F02012090404A094EF20011CEF28D
:10FC1000000141F82200FFE701B070474EF60C509A
:10FC2000CEF200000068C0F30220704782B08DF869
:10FC3000070000919DF9070000280AD4FFE700980B
:10FC400000019DF907104EF20042CEF200028854E6
:10FC50000BE0009800019DF8071001F00F014EF62F
:10FC60001452CEF200028854FFE702B07047000041
:10FC700082B08DF8070000919DF9070000280AD492
:10FC8000FFE7009800019DF907104EF20042CEF206
:10FC9000000288540BE0009800019DF8071001F065
:10FCA0000F014EF61452CEF200028854FFE702B064
:10FCB0007047000083B00290029800F007000090A7
:10FCC0004EF60C51CEF200010868019001984FF6F3
:10FCD000FF02104001900198009A40EA02200022A1
:10FCE000C0F2FA52104301900198086003B07047C7
:10FCF00080B58EB00C900B918DED0A0A0C9858B11E
:10FD0000FFE70B9840B1FFE79DED0A0AB5EE400A08
:10FD1000F1EE10FA04DCFFE7FF208DF837001FE159
:10FD20000B980C99C1F870040C99032008720C9977
:10FD3000D1F87004D0F8C800C1F828060C99D1F8A1
:10FD40007004D0F8CC00C1F82C060C99D1F87004DE
:10FD5000D0F8D000C1F83006F2F7CEFB00200990B1
:10FD6000FFE7099803280EDCFFE70C98D0F8700431
:10FD7000099900EBC1008030FBF740FDFFE70998CF
:10FD800001300990EDE700200890FFE7089803286C
:10FD90000EDCFFE70C98D0F87004089900EBC10066
:10FDA000A030FBF72BFDFFE7089801300890EDE746
:10FDB00048F28C23C0F60103186859689A68DB681A
:10FDC00007930692059104900C990498059A069B56
:10FDD000DDF81CC0C1F86CC4C1F86834C1F86424F3
:10FDE000C1F8600400200390FFE70398032816DCA5
:10FDF000FFE70C990398C0EB001001EB800000F5C1
:10FE00003B709DED0A0AD1F8701401F14002002107
:10FE1000FCF738FCFFE7039801300390E5E700208A
:10FE20000290FFE70298032825DCFFE70C9902986F
:10FE3000C0EB001001EB800000F5FE709DED0A0A9A
:10FE4000D1F8702401210191FCF71CFC01990C9A56
:10FE50000298C0EB001002EB800000F586709DED6B
:10FE60000A0AD2F870242032FCF70CFCFFE7029853
:10FE700001300290D6E70C9901F577709DED0A0AE2
:10FE8000D1F8701401F160020121FCF7FBFB0C9822
:10FE900000F294409DED0A0AF3EE040ACDED000A4B
:10FEA000FAF742FEDDED000A0C9800F2B4409DED39
:10FEB0000A0AFAF739FEDDED000A0C9800F2D44088
:10FEC0009DED0A0AFAF730FEDDED000A0C9800F20B
:10FED000F4409DED0A0AFAF727FEDDED000A0C98C2
:10FEE00000F214509DED0A0AFAF71EFEDDED000A3D
:10FEF0000C9800F234509DED0A0AFAF715FEDDED7C
:10FF0000000A0C9800F254509DED0A0AFAF70CFE14
:10FF1000DDED000A0C9800F274509DED0A0AFAF724
:10FF200003FEDDED000A0C9800F294509DED0A0AE4
:10FF3000FAF7FAFDDDED000A0C9800F2B4509DEDE1
:10FF40000A0AFAF7F1FDDDED000A0C9800F2D45030
:10FF50009DED0A0AFAF7E8FD00208DF83700FFE76B
:10FF60009DF937000EB080BD82B08DED010ACDED58
:10FF7000000A01980099C90F61F3DF7001909DEDAF
:10FF8000010A02B07047000080B588B0069006985C
:10FF90000190019858B9FFE74FF0500080F31188A5
:10FFA000BFF36F8FBFF34F8F0790FFE7FEE7019816
:10FFB00041F23861C2F200010968884204D1FFE7CA
:10FFC00000208DF8170056E002F090F80198406983
:10FFD000049041F24060C2F200000068039041F2D8
:10FFE0004860C2F200000068029002F0ABF804988A
:10FFF0000399884205D0FFE704980299884204D10A
:020000040801F1
:10000000FFE702208DF8170034E0049842F6E06123
:10001000C2F20101884218D1FFE70198806A78B9DD
:10002000FFE7019890F85800012804D1FFE702206B
:100030008DF8170003E003208DF81700FFE703E0B9
:1000400002208DF81700FFE713E0049842F6F461F0
:10005000C2F20101884203D0FFE7049820B9FFE70C
:1000600004208DF8170003E001208DF81700FFE74A
:10007000FFE7FFE7FFE79DF8170008B080BD00002D
:1000800086B08DED050ACDED040A8DED031A0290C0
:100090009DED030A9DED041A30EE410A8DED010A33
:1000A000049800909DED050A9DED001A30EE410A7E
:1000B000029901208840013801EE100AB8EEC11AF9
:1000C00020EE010A9DED011A80EE010ABDEEC00A84
:1000D00010EE100A06B0704780B582B00020019083
:1000E000F7F79EFDFEF716F9FBF742FEFBF7C2FDA0
:1000F000FBF770FDFBF796FDFBF72EFFFBF7BCFF50
:10010000FBF7E0FFFBF750FFFBF796FF00F0B2F8BC
:10011000FBF70EFE00F0FEF8FFE7FEE785B08DED81
:10012000040ACDED030A8DED021ACDED011A8DED15
:10013000002A9DED040A9DED033A30EE430A9DED41
:10014000002A9DED011A32EE412A20EE020A9DEDB1
:10015000022A32EE432A80EE020A30EE010A05B08E
:100160007047000080B584B00290EFF305800390E3
:10017000039820B1FFE76FF00500019009E000202F
:100180000190029820B1FFE7029802F029F9FFE7F9
:10019000FFE7019804B080BD80B586B00490EFF30E
:1001A00005800590059820B1FFE76FF005000190EC
:1001B0001BE00020019003F0E5FD039004980399F3
:1001C000401A0290029858B1FFE702990020B0EB64
:1001D000D17F05D1FFE7029903A802F039F903E0C6
:1001E0006FF003000190FFE7FFE7019806B080BDC4
:1001F00080B582B003F0AAFD0146009158B1FFE737
:10020000009801280AD0FFE70098022807D1FFE7ED
:100210000220019012E0032001900FE0FFE740F27E
:100220004050C2F200000068012803D1FFE701201E
:10023000019002E000200190FFE7FFE7019802B083
:1002400080BD000080B582B0EFF305800190019879
:1002500020B1FFE703F0A0FD009003E003F092FD62
:100260000090FFE7009802B080BD00004FF47A7064
:100270007047000082B0EFF305800190019820B133
:10028000FFE76FF00500009014E040F24050C2F22A
:100290000000006848B9FFE740F24051C2F2000197
:1002A000012008600020009003E04FF0FF30009034
:1002B000FFE7FFE7009802B07047000080B584B008
:1002C000EFF305800390039820B1FFE76FF005007E
:1002D00002901BE003F03AFD0146019140B1FFE7B7
:1002E000019801280CD0FFE70198022803D008E00C
:1002F0000120029009E002F02DFB0020029004E0B2
:10030000FFE74FF0FF300290FFE7FFE7029804B0ED
:1003100080BD000080B582B0EFF3058001900198A8
:1003200020B1FFE76FF00500009019E040F2405067
:10033000C2F20000006801280DD1FFE7FCF77AFE49
:1003400040F24051C2F200010220086002F092FA2D
:100350000020009003E04FF0FF300090FFE7FFE740
:10036000009802B080BD000080B584B0EFF3058036
:100370000390039820B1FFE76FF00500029027E09B
:1003800003F0E4FC0146019140B1FFE70198012828
:1003900018D0FFE70198022811D014E00120029044
:1003A00003F0BEFF012809D0FFE703F0CFFC20B91E
:1003B000FFE74FF0FF300290FFE7FFE707E0002084
:1003C000029004E0FFE74FF0FF300290FFE7FFE705
:1003D000029804B080BD000080B588B006900591F9
:1003E000049203930698029000200190EFF3058099
:1003F0000790079868B3FFE7029830B1FFE70598C8
:1004000018B1FFE7039820B1FFE76FF003000190F8
:100410001EE000200090029805996A4602F0FEFF57
:10042000012804D0FFE76FF0020001900FE0009870
:1004300060B1FFE74EF60451CEF200014FF080505C
:100440000860BFF34F8FBFF36F8FFFE7FFE7FFE752
:100450001FE0029818B1FFE7059820B9FFE76FF099
:100460000300019014E002980599039A02F0E8FE57
:1004700001280CD0FFE7039820B1FFE76FF00100DF
:10048000019003E06FF002000190FFE7FFE7FFE754
:10049000FFE7019808B080BD80B588B0069005914F
:1004A000049200200390EFF305800790079800283E
:1004B0006ED1FFE7069800286AD0FFE7059800286C
:1004C00066D0FFE74FF0FF300290049868B3FFE773
:1004D00004988068A0B1FFE70498C06850280FD343
:1004E000FFE70498006958B1FFE70498406906994E
:1004F000059A5143884203D3FFE70120029013E09D
:100500000498806878B9FFE70498C06858B9FFE795
:100510000498006938B9FFE70498406918B9FFE703
:1005200000200290FFE7FFE702E000200290FFE7D3
:10053000029801280ED1FFE706980599049A93685E
:100540001269EE464FF0000CCEF800C002F0A0FB9E
:1005500003900AE0029838B9FFE70698059900224F
:1005600002F05CFB0390FFE7FFE7039878B1FFE739
:10057000049820B1FFE704980068019002E0002091
:100580000190FFE70398019901F0CEFEFFE7FFE736
:10059000039808B080BD000080B588B00690059132
:1005A0008DF8132003930698029000200190EFF33A
:1005B00005800790079868B3FFE7029830B1FFE71E
:1005C000059818B1FFE7039820B1FFE76FF003002B
:1005D00001901EE000230093029805996A4602F0FC
:1005E00053FD012804D0FFE76FF0020001900FE0F7
:1005F000009860B1FFE74EF60451CEF200014FF0D3
:1006000080500860BFF34F8FBFF36F8FFFE7FFE7A6
:10061000FFE720E0029818B1FFE7059820B9FFE74F
:100620006FF00300019015E002980599039A0023EA
:1006300002F014FC01280CD0FFE7039820B1FFE77B
:100640006FF00100019003E06FF002000190FFE7FE
:10065000FFE7FFE7FFE7019808B080BD80B584B0F1
:10066000029002980190EFF305800390039820B167
:10067000FFE76FF0050000900DE0019820B9FFE75B
:100680006FF00300009005E000210091019802F056
:1006900087FBFFE7FFE7009804B080BD80B586B018
:1006A00004900391049820F001000290049800F057
:1006B0000100009000200190EFF30580059005985F
:1006C00020B1FFE76FF00500019033E0029820B9F8
:1006D000FFE76FF0030001902BE00098A0B1FFE767
:1006E0000298039903F034F801280CD0FFE703982F
:1006F00020B1FFE76FF00100019003E06FF002000E
:100700000190FFE7FFE713E00298039902F00AFF68
:1007100001280CD0FFE7039820B1FFE76FF001003C
:10072000019003E06FF002000190FFE7FFE7FFE7B1
:10073000FFE7FFE7019806B080BD000080B588B0F4
:10074000069000200590EFF3058007900798002899
:1007500040F08580FFE7069820B1FFE706984068E3
:10076000049002E000200490FFE79DF81000C0070D
:1007700018B1FFE70120039002E000200390FFE79B
:10078000049800F00800082868D0FFE74FF0FF3019
:1007900002900698C8B1FFE70698806840B1FFE76D
:1007A0000698C068502803D3FFE7012002900BE0B1
:1007B0000698806838B9FFE70698C06818B9FFE75F
:1007C00000200290FFE7FFE702E000200290FFE731
:1007D0000298012812D1FFE7039838B1FFE7069885
:1007E0008168042002F000FA059006E0069881680E
:1007F000012002F0F9F90590FFE711E0029870B9C5
:10080000FFE7039828B1FFE7042002F0D9F905902B
:1008100004E0012002F0D4F90590FFE7FFE7FFE7CD
:10082000059878B1FFE7069820B1FFE706980068C1
:10083000019002E000200190FFE70598019901F086
:1008400073FDFFE7059840B1FFE7039828B1FFE784
:10085000059840F001000590FFE7FFE7FFE70598E6
:1008600008B080BD80B586B00490049820F00100E7
:100870000390049800F00100019000200290EFF333
:1008800005800590059820B1FFE76FF00500029004
:1008900024E0039820B9FFE76FF0030002901CE00A
:1008A000019858B1FFE7039802F094FC012804D0A6
:1008B000FFE76FF002000290FFE70DE003980023CE
:1008C00019461A4602F0CAFA012804D0FFE76FF071
:1008D00002000290FFE7FFE7FFE7FFE7029806B09C
:1008E00080BD000080B58AB00890079108980690F6
:1008F000069830B1FFE79DF81F000006002804D5D8
:10090000FFE76FF0030005903BE04FF0FF300590EC
:10091000EFF305800990099820B3FFE700230393C4
:10092000049306980799EC4604AACCF8002001220B
:1009300003F020F9039A069869460A6005AB114650
:1009400003F018F9049860B1FFE74EF60451CEF2B7
:1009500000014FF080500860BFF34F8FBFF36F8FDF
:10096000FFE70DE00698079901220023029303F0A8
:1009700045F8029A069805AB114603F03FF8FFE7E9
:10098000FFE705980AB080BD80B58CB00A90099148
:100990000892EFF305800B900B9820B1FFE76FF002
:1009A000050007907AE09DF82B000006002804D58A
:1009B000FFE76FF0030007906FE09DF824008007C9
:1009C000002803D5FFE70020059002E00A98059073
:1009D000FFE7002007900898029003F0D3F90490F5
:1009E000FFE70599029B002006AA03F0C7FA0190D1
:1009F000019801283FD1FFE70A990798084007901E
:100A000006990798084307909DF82400C00780B115
:100A1000FFE70A9907980840884201D1FFE73BE0C9
:100A2000089820B9FFE76FF00200079034E0FFE775
:100A30000EE00A980799084201D0FFE72CE00898D9
:100A400020B9FFE76FF00200079025E0FFE7FFE71E
:100A500003F098F90499401A039003980299884288
:100A600003D9FFE70020029004E003990298401A9E
:100A70000290FFE70BE0089820B9FFE76FF0020053
:100A8000079003E06FF001000790FFE7FFE7FFE743
:100A900001980028A5D1FFE7FFE7FFE707980CB012
:100AA00080BD000080B582B003F046F90190019846
:100AB00002B080BDB0B58EB00B900A9109920020B3
:100AC0000690EFF305800D900D98002840F0998076
:100AD000FFE70B98002800F09480FFE78020079044
:100AE00018200590002008904FF0FF3004900998DE
:100AF00000284DD0FFE70998006820B1FFE709986A
:100B000000680890FFE70998806920B1FFE709981D
:100B100080690590FFE7059848B1FFE705983828F8
:100B200005D8FFE709980079C00718B1FFE7002052
:100B30000C9069E00998406928B1FFE7099840697D
:100B400080080790FFE70998806880B1FFE709985F
:100B5000C0685C280BD3FFE70998006938B1FFE74C
:100B60000998406918B1FFE7012004900FE0099847
:100B7000806858B9FFE70998C06838B9FFE7099855
:100B8000006918B9FFE700200490FFE7FFE702E0E3
:100B900000200490FFE70498012817D1FFE70B9885
:100BA0000899079A0A9BDDF814C0DDF824E0DEF806
:100BB0000850DEF81040EE46CEF80850CEF804405B
:100BC000CEF800C002F0B2FE069019E00498B0B969
:100BD000FFE70B980899BDF81C200A9BDDF814C0AC
:100BE000EE4606ACCEF80440CEF800C002F04EFE51
:100BF000012803D0FFE700200690FFE7FFE7FFE7AB
:100C0000FFE706980C90FFE70C980EB0B0BD00000F
:100C100080B586B0049004980390EFF305800590AA
:100C2000059820B1FFE76FF0050002901CE00398E3
:100C300020B9FFE76FF00300029014E00398FFF77C
:100C4000A3F98DF807009DF80700042806D0FFE7F8
:100C500000200290039801F085FC03E06FF0020091
:100C60000290FFE7FFE7FFE7029806B080BD0000B3
:100C700080B586B08DED040B9DED040B9FED261B1A
:100C800004F0CAFA51EC100B9FED250B53EC102B1E
:100C900006F018FC41EC100B8DED000B9DED040BE4
:100CA0009FED211B04F0B8FA51EC100B9FED200BC7
:100CB00053EC102B06F006FC9DED001B41EC100BD5
:100CC00051EC110B53EC102B06F0AAF841EC100B71
:100CD0008DED020B049805999FED170B53EC102B2B
:100CE00006F0F0FB9DED021B41EC100B51EC110BDB
:100CF00053EC102B06F094F841EC100B51EC100B58
:100D00009FED0F0B53EC102B06F08AF841EC100B03
:100D100006B080BD00BF00BF00000000000008401A
:100D20005F09A4C4AEEDDA3F0000000000000040FF
:100D3000412B3064752B02C04CFDBCA94885104086
:100D4000BC5CC47762D6FFBF80B584B003900291CB
:100D500042F60870C2F201000068009041F238606B
:100D6000C2F200000068043001F0F2F808B9FFE7B1
:100D700000E0FFE70398013080B9FFE7029868B10F
:100D8000FFE741F23860C2F200000068011D42F640
:100D9000E060C2F2010001F081F93DE000980399A2
:100DA00008440190019841F23861C2F200010968DB
:100DB00048600198009988420ED2FFE741F24860EE
:100DC000C2F20000006841F23861C2F20001096815
:100DD000043101F02DF91EE041F24060C2F2000042
:100DE000006841F23861C2F200010968043101F083
:100DF0001FF9019842F66C61C2F20101096888424C
:100E000007D2FFE7019842F66C61C2F20101086067
:100E100000E0FFE7FFE7FFE704B080BD80B582B0E8
:100E2000019001F063F942F24071C2F201010868D9
:100E30000130086041F23860C2F20000006898B9E1
:100E4000FFE7019841F23861C2F20001086042F206
:100E50004070C2F201000068012803D1FFE700F0F2
:100E600021FB00E0FFE71CE042F6D460C2F2010083
:100E70000068A0B9FFE741F23860C2F200000068E4
:100E8000C06A0199C96A884207D8FFE7019841F210
:100E90003861C2F20001086000E0FFE700E0FFE710
:100EA000FFE742F24C70C2F20100016801310160BB
:100EB0000068019948640198C06A42F25071C2F218
:100EC00001010968884208D9FFE70198C06A42F227
:100ED0005071C2F201010860FFE70199C86A00EB96
:100EE000800241F25060C2F2000000EB8200043147
:100EF00001F0D4F801F026F942F6D460C2F2010004
:100F00000068C8B1FFE741F23860C2F20000006833
:100F1000C06A0199C96A88420CD2FFE74EF60451B3
:100F2000CEF200014FF080500860BFF34F8FBFF347
:100F30006F8F00E0FFE700E0FFE702B080BD000038
:100F400080B584B001F0D2F842F60C70C2F2010014
:100F50000068002840D1FFE742F60C60C2F20100B1
:100F6000029001F045F842F62060C2F201000390C1
:100F700001F03EF80299039841F23C62C2F200028D
:100F8000116041F24C61C2F2000108606946002024
:100F9000086041F24452C2F2000241F2E453C2F24C
:100FA00000030A20102101F073FE014642F60C7086
:100FB000C2F201000160006860B1FFE742F60C7008
:100FC000C2F20100006848F2D121C0F6010101F02F
:100FD000ABF900E0FFE700E0FFE701F0B3F804B091
:100FE00080BD000080B582B0FFE742F24470C2F2DB
:100FF0000100006808B3FFE701F078F842F6F460FA
:10100000C2F20100C068C06801900198043000F08D
:101010009FFF42F24071C2F2010108680138086086
:1010200042F24471C2F2010108680138086001F01F
:1010300089F8019800F08CF8D7E702B080BD000075
:1010400080B582B0019000910198006CB8B1FFE7C3
:101050000199C8680A6C1044C86001988168C0682A
:10106000884204D3FFE701990868C86000E0FFE701
:101070000098019AD168126CEFF7AEF9FFE702B061
:1010800080BD000080B586B00590049103920020D9
:1010900002900598806B01900598006C78B9FFE785
:1010A0000598006848B9FFE70598806802F0D2FF0C
:1010B000029005990020886000E0FFE741E0039876
:1010C000B8B9FFE7059A04995068126CEFF784F9F4
:1010D000059948680A6C1044486005994868896811
:1010E000884204D3FFE705990868486000E0FFE7FD
:1010F00026E0059A0499D068126CEFF76DF905990E
:10110000C8680A6C801AC86005980168C06888427F
:1011100006D2FFE7059988680A6C801AC86000E06B
:10112000FFE70398022809D1FFE7019820B1FFE704
:1011300001980138019000E0FFE700E0FFE7FFE7DA
:10114000FFE70198013005998863029806B080BDD9
:1011500080B582B00090009890F8590040B9FFE740
:101160000098006B01F014F8009801F011F81CE0F1
:10117000009890F85900012804D1FFE7009801F089
:1011800007F811E0009890F8590002280BD0FFE70B
:101190004FF0500080F31188BFF36F8FBFF34F8F74
:1011A0000190FFE7FEE7FFE7FFE702B080BD000028
:1011B00082B001900198406A38B1FFE70198006B56
:1011C0000068C0F13800009002E000200090FFE7C6
:1011D000009802B07047000082B0019041F23C607C
:1011E000C2F2000000680068B0FA80F0400901997E
:1011F00008600198006848B9FFE741F23C60C2F21C
:1012000000000068C0680068009002E000200090C4
:10121000FFE7009802B0704784B04FF48030009030
:1012200042F23470C2F2000001909DF804004007C1
:1012300088B1FFE7019807300190019820F007007E
:101240000190019A42F23471C2F200010098891AA9
:1012500008440090FFE701980290029942F6D86096
:10126000C2F201000160002141600298009A10441E
:101270000190019808380190019820F00700019032
:10128000019A41F24460C2F20000026002685160BB
:1012900002681160029903910199039A891A5160B9
:1012A0000068039908600398406842F66861C2F2DA
:1012B000010108600398406842F66061C2F20101D2
:1012C000086042F63461C2F201014FF0004008604C
:1012D00004B0704780B582B00190FFE7FFF782FE4F
:1012E00041F25060C2F20000006802280CD3FFE710
:1012F0004EF60451CEF200014FF080500860BFF36B
:101300004F8FBFF36F8F00E0FFE7E7E780B582B054
:101310000190019868B1FFE701980023836001986C
:1013200003600198C360019819461A4601F096FDC2
:1013300000E0FFE702B080BD80B584B0DDF818C0E2
:101340000390029101928DF80330029818B9FFE7DB
:101350000698006003E0019806990860FFE703988B
:101360000699C8630298069908640698012101F05D
:1013700017FD9DF80300069981F84C0004B080BD6C
:1013800080B588B0DDF834C0DDF830C0DDF82CC0A1
:10139000DDF828C006900591049203930C98006B29
:1013A00004998900A522EFF78EF80C98006B049938
:1013B00000EB810004380290029820F007000290B0
:1013C0009DF80800400758B1FFE74FF0500080F348
:1013D0001188BFF36F8FBFF34F8F0790FFE7FEE7D2
:1013E0000598F8B1FFE700200190FFE701980F286A
:1013F00013D8FFE70598019A805C0C99114481F895
:10140000340005980199405C08B9FFE705E0FFE763
:10141000FFE7019801300190E8E70C99002081F87E
:10142000430004E00C99002081F83400FFE70A989B
:10143000382803D3FFE737200A9000E0FFE70A9837
:101440000C99C8620A980C99C8640C990020009005
:1014500008650C98043000F0E3FD0C98183000F09B
:10146000DFFD00980C9909610A99C1F138010C9AC5
:1014700091610C9949620C9948650C9981F8580062
:1014800002980699039A00F0E7FC0C9908600B9803
:1014900020B1FFE70C980B99086000E0FFE708B067
:1014A00080BD000080B584B000200390FFE7039862
:1014B000372810D8FFE7039800EB800141F2506015
:1014C000C2F2000000EB810000F092FDFFE70398FC
:1014D00001300390EBE742F63860C2F20100019060
:1014E00000F086FD42F64C60C2F20100029000F06E
:1014F0007FFD42F68060C2F2010000F079FD42F605
:10150000F460C2F2010000F073FD42F6E060C2F246
:10151000010000F06DFD0199029841F24062C2F2B3
:101520000002116041F24861C2F20001086004B09B
:1015300080BD000083B0029042F6D860C2F2010084
:101540000190FFE7019800680299884205D2FFE701
:10155000FFE7019800680190F4E701980090009877
:101560000199496808440299884209D1FFE7029825
:10157000426801994868104448600198029000E070
:10158000FFE7029800900098029949680844019981
:101590000968884220D1FFE70198006841F2446160
:1015A000C2F20001096888420DD0FFE70198006887
:1015B00042680299486810444860019800680068D1
:1015C0000299086007E041F24460C2F2000000683E
:1015D00002990860FFE704E001980068029908603A
:1015E000FFE701980299884204D0FFE70298019929
:1015F000086000E0FFE703B07047000080B586B0E8
:10160000059004910392029300200190049805999B
:1016100048600598006104980399884216D8FFE74E
:1016200003980299401A05998969884203D3FFE714
:101630000120019009E041F24C60C2F20000006814
:101640000599043100F0F4FCFFE717E003980299D4
:10165000884208D2FFE704980299884203D3FFE743
:101660000120019009E041F23C60C2F200000068F4
:101670000599043100F0DCFCFFE7FFE7019806B0B4
:1016800080BD000080B582B0019000F02FFD019870
:10169000806B18B9FFE70120009002E00020009065
:1016A000FFE700F04FFD009802B080BD80B582B02A
:1016B000019000F01BFD0198806B0199C96B884275
:1016C00003D1FFE70120009002E000200090FFE737
:1016D00000F038FD009802B080BD000008480068A6
:1016E000006880F308884FF0000080F3148862B629
:1016F00061B6BFF34F8FBFF36F8F00DF00BF00BF36
:1017000008ED00E080B586B00490039141F23C60A2
:10171000C2F200000068C068C068019001980430FF
:1017200000F016FC019890F828004007002823D507
:10173000FFE70198049B81691944039AFFF75EFF54
:10174000C0B1FFE70198049A694600230B6019466F
:1017500002F0F4FE0290029858B9FFE74FF05000F3
:1017600080F31188BFF36F8FBFF34F8F0590FFE7B2
:10177000FEE700E0FFE707E0019991F8280000F09C
:10178000FE0081F82800FFE70198016A884706B04B
:1017900080BD000080B58EB0FFE742F60C70C2F24B
:1017A0000100006807A9002201F04AFD002800F0AE
:1017B000B880FFE70798B0F1FF3F17DCFFE707A805
:1017C00004300290029858B9FFE74FF0500080F3C0
:1017D0001188BFF36F8FBFF34F8F0B90FFE7FEE7CA
:1017E00002990A6848688968904700E0FFE707980F
:1017F000002800F19580FFE7099806900698406957
:1018000028B1FFE70698043000F0A2FB00E0FFE7F4
:1018100005A800F0FBF8039007980190092800F252
:101820007D800199DFE801F00505053D4566050568
:101830003D45069991F8280040F0010081F8280004
:101840000698089B81691944039AFFF7D7FE30B3C5
:10185000FFE70698016A8847069890F82800400735
:1018600000281AD5FFE70698089982690A44694654
:1018700000230B60194602F061FE0490049858B9E9
:10188000FFE74FF0500080F31188BFF36F8FBFF375
:101890004F8F0C90FFE7FEE700E0FFE700E0FFE777
:1018A0003DE0069991F8280000F0FE0081F828003C
:1018B00035E0069991F8280040F0010081F82800F1
:1018C0000898069988610698806958B9FFE74FF033
:1018D000500080F31188BFF36F8FBFF34F8F0D90CF
:1018E000FFE7FEE70698039B816919441A46FFF754
:1018F00085FE14E0069890F828008007002804D49C
:10190000FFE7069800F044FC07E0069991F82800EC
:1019100000F0FE0081F82800FFE700E0FFE7FFE7A6
:101920003BE70EB080BD000080B584B0039002910B
:1019300001F010F8684600F069F801900098D8BBF3
:10194000FFE7029860B9FFE703980199884207D83A
:10195000FFE702F0E5FC03980199FFF7D3FE2AE0C8
:10196000029858B1FFE741F24C60C2F200000068F3
:101970000068B0FA80F040090290FFE742F60C7070
:10198000C2F2010000680399019A891A029A00F0D4
:10199000F5FC02F0C5FC60B9FFE74EF60451CEF24B
:1019A00000014FF080500860BFF34F8FBFF36F8F7F
:1019B00000E0FFE7FFE702E002F0B2FCFFE704B05F
:1019C00080BD000081B041F24060C2F200000068BA
:1019D000006840B9FFE742F66C61C2F201014FF0C6
:1019E000FF3008600FE041F24060C2F20000006882
:1019F000C068C06800900098406842F66C61C2F20E
:101A000001010860FFE701B07047000080B582B0B7
:101A1000019002F0B7F90090009841F23461C2F2EF
:101A200000010968884206D2FFE700F011F8019929
:101A30000120086003E0019900200860FFE700989A
:101A400041F23461C2F200010860009802B080BD2A
:101A500080B588B0FFE741F23C60C2F20000006848
:101A6000006800284ED0FFE741F23C60C2F200005F
:101A70000168C968096806910068C068C068039079
:101A80000398043000F064FA0398016A88470398C9
:101A900090F828004007002832D5FFE70698039900
:101AA0008969084405900598069988420FD9FFE78F
:101AB0000598039948600398006141F23C60C2F2C6
:101AC000000000680399043100F0B2FA17E00398AF
:101AD000069A694600230B60194602F02FFD02901A
:101AE000029858B9FFE74FF0500080F31188BFF318
:101AF0006F8FBFF34F8F0790FFE7FEE7FFE700E030
:101B0000FFE7A8E741F23C62C2F2000210680490CD
:101B100041F24C61C2F2000108681060049808604C
:101B200008B080BD83B00020009040F24C30C2F27B
:101B300000000068013058B1FFE74FF0500080F31B
:101B40001188BFF36F8FBFF34F8F0190FFE7FEE760
:101B50004FF0500080F31188BFF36F8FBFF34F8FAA
:101B60000290FFE7009808B9FFE7FBE703B0704772
:101B700080B584B00390FFE701A8FFF72DFB02902A
:101B800002980199FFF7D0FEFFF704FEF4E700008A
:101B900080B582B0019000F0A9FA019890F8450054
:101BA0008DF80300FFE79DF90300012816DBFFE72E
:101BB0000198406A58B1FFE70198243002F048FBD1
:101BC00018B1FFE700F068FD00E0FFE700E005E086
:101BD0009DF8030001388DF80300E4E70199FF2028
:101BE00081F8450000F0AEFA00F080FA019890F814
:101BF00044008DF80200FFE79DF90200012816DB82
